:020000040000FA
:1000000040EF0720FDF0020001F1020003F10200C1
:1000100005F1020007F1020009F10200AA6AE6DF19
:100020000000000000000000000000000BF10200D2
:100030000DF10200000000000FF1020011F10200BA
:1000400013F102009DF8020013F102008F55030026
:1000500013F10200653F030013F1020001420300A7
:1000600013F102006546030013F1020013F10200D0
:1000700013F1020013F1020013F1020013F1020068
:1000800013F1020013F1020013F1020013F1020058
:1000900013F1020013F1020013F1020013F1020048
:1000A000F577030013F1020013F1020013F10200CF
:1000B00013F1020013F1020013F1020013F1020028
:1000C00013F1020013F1020013F1020000F002F834
:1000D00000F086F80AA090E8000C82448344AAF15C
:1000E0000107DA4501D100F07BF8AFF2090EBAE85A
:1000F0000F0013F0010F18BFFB1A43F0010318475C
:10010000CCE00400FCE004000A444FF0000C10F8BE
:10011000013B13F0070408BF10F8014B1D1108BF85
:1001200010F8015B641E05D010F8016B641E01F825
:10013000016BF9D113F0080F1EBF10F8014BAD1C75
:100140000C1B09D16D1E58BF01F801CBFAD505E093
:1001500014F8016B01F8016B6D1EF9D59142D6D3ED
:10016000704700000023002400250026103A28BF15
:1001700078C1FBD8520728BF30C148BF0B60704719
:1001800069293CF01B8164293CF0188175293CF0F9
:1001900015816F293CF0AC8178293CF0D38103684C
:1001A000DB0928BF41F0800163293CF07C8573297D
:1001B0003CF08185E3293CF08C85002070471FB519
:1001C0009DE803003CF0A6FC3CF0FEFD040000208E
:1001D00000213DF09BF9401C60601FBD10B510BDB3
:1001E0003CF0CDFD1146FFF7EAFF00F01FF93CF0AF
:1001F000EFFD03B4FFF7F2FF03BC3CF01FFE00006D
:1002000010B5782119483CF03CFC19494FF0FF30FB
:10021000088010BD16480188491C09B201800A29CE
:100220000CD001EB41021149436841F8223001EB47
:10023000820183684B60C06888607047FEE70C49A4
:1002400010B5B1F90000421C0ED0084A00EB400383
:10025000401E52F8234002EB83024C6053688B60CF
:100260009268CA60088010BDFEE7000090C60720B3
:1002700008C0072030B502464FF6FF7318460E4CF3
:1002800008E000BF12F8015B85EA1025655D85EA8C
:10029000002080B2491E89B2F4D2584030BD0246D7
:1002A00010B5FF20002905D0044B545C4440491E82
:1002B000185DFAD110BD000002E8030054C0072009
:1002C0000A4900EB4000084410F8030C7047074946
:1002D00000EB4000084410F8020C7047034900EBA3
:1002E0004000084410F8010C704700002408040086
:1002F00000487047DCDE072070477047FFFFFFFFB4
:100300007FB5054603A805F083FB264C000640D4C4
:100310009DF80C00012832D00026022809D0872041
:10032000206021480660784620490860872004B094
:1003300070BD00200BF05CFE00062AD42888ADF8C2
:1003400004006888ADF8060028798DF808008DF85B
:10035000096001A80AF08CFD00061AD469462B201A
:100360001BF0BAFA000614D411489DF8001000786A
:10037000C90704D0012802D001208DF80C0003A881
:1003800005F04DFB000604D4284608F019F90006D4
:1003900001D52068CBE703208DF80C0003A805F0F9
:1003A0002DFBC4E70CC0072010C0072014C0072095
:1003B000CAC3072038B50546684605F029FB0D4C31
:1003C000000611D49DF80000032809D087200A49AF
:1003D000206000200860784608490860872038BD02
:1003E0000BF0DEFD000601D5206838BD284608F078
:1003F0002FFA38BD0CC0072010C0072014C00720FA
:10040000D26770CE601B01B53CF01BFA01BD70478E
:100410004170722031392032303136000000000046
:1004200031363A30343A32350000000088B0C24CE0
:100430000027039720883E4640F002002080BF48F6
:100440002DF023FFBE48007802281CD1FFF7E2FE02
:1004500003A82EF04DFF000601D502F076FDFFF750
:10046000EEFE0398B0F58C7F0DDAFFF7D3FE002186
:10047000B4A036F0CAFA000601D502F066FDFFF717
:10048000DEFE02F062FDAD4D288830F4504010D001
:100490000127FFF7BFFE32201AF049FA012011F0C0
:1004A00041FB10B1082036F09BFCFFF7C8FE02F0BC
:1004B0004CFD2888810B06D001270FF0F3FD0006C4
:1004C00001D502F042FDAA482E80007828B12EF016
:1004D00097FA10B1A7A036F062FC26F005F90006E5
:1004E00001D502F032FD01F093F906F022FB00067F
:1004F00001D502F02AFDA54DAE6805A82DF0C0FD7E
:1005000001F03EF910B1012702F01FFD01F0C2F920
:10051000DFF87C82C0B1FFF77DFE01F013FBFFF72F
:100520008EFED8F80000062802D0002199A004E031
:100530009D490220087000219CA036F066FA2088B0
:1005400040F0020020800CE001F0C1FB38B1FFF761
:1005500061FE01F0F7FAFFF772FE02F0F6FC01F01F
:100560003FFE9748A968891B8142FBD306A82DF05E
:1005700087FD944EDFF85092307800EB400159F837
:1005800031008047000601D502F0DFFC01F061FE7A
:10059000000601D502F0D9FC9DF81A009DF816104E
:1005A000884201D0012000E0002001F094FE00B15B
:1005B000012701F0EEFE00F0A5FC02A953201BF07C
:1005C0008BF9000601D502F0C0FC9DF8080000F090
:1005D00001008DF808006FB9B0B1012011F0A2FA46
:1005E000000601D502F0B1FC10F0F6FD000601D5C1
:1005F00002F0ABFC9DF8080030B1012011F092FA36
:10060000000601D502F0A1FC2FF0FAF94F46E946A9
:10061000307800EB400007EBC000C0688047000660
:1006200001D502F092FC307800EB400007EBC000EF
:1006300040688047000601D502F087FC307800EB67
:10064000400007EBC00080688047000601D502F03B
:100650007CFC002035F0ACFED8F800000C2805D05A
:1006600004F08EFE000601D502F06FFC20784007F2
:100670001ED5012035F09CFED0B9684605F053FA2E
:1006800050B909F1020005F05FFA28B909F1040038
:1006900005F06BFA000601D502F057FC4B499DF8B6
:1006A00004000870684606F05BFC08B907F0BCFA65
:1006B000207810F0B80F35D0012035F079FE000613
:1006C00030D4A8684249AA68121A8A42FBD320781B
:1006D000000701D510F029FE2088010614D58106F7
:1006E00012D4C00613D410F07AFE000601D502F031
:1006F0002CFC002007F082FB000601D502F025FC4F
:10070000208820F0810020802078C00601D506F0E6
:10071000C9FB2078800605D5012009F07DF801206D
:1007200011F000FA2FF0CEF9000601D502F00DFC11
:1007300036F040FC6CE7000002C0072004C0072030
:1007400088C407208E9888818A802081809280903A
:100750008588209780918E820A8E819080928892DF
:1007600085919C20822096928E0A0A0A0A00000037
:1007700089C50720C0E2F2EEEEF2F0E5E7F7E8EA1D
:1007800020E2FBEAEBFEF7E5ED0A0000000009407D
:1007900010C007208E9888818A80208F808C9F923D
:1007A00088208F840A0A000000C00720878D208DD2
:1007B000852082828584858D0A0A0A0A0A00000043
:1007C000E0C81000CAC30720CCC3072071C30720AC
:1007D000A08601002DE9F047FD4DFE4EFE4F9046EC
:1007E000C3B15C1E0BD4DFF8F493642200233BF00A
:1007F000B5FC19F8023008F80430641EF5D508433A
:1008000010D0892028600420306078463860892024
:10081000BDE8F0878820286009203060784638607D
:100820008820F5E700202860306078463860002096
:10083000EEE710B500220BE0835C03F00F04092CF7
:1008400003D803F0F003902B01D9002010BD521CF7
:100850008A42F1D3012010BD2DE9FF4FDC4CDD4D64
:10086000DD4E83B08246082A30D872B30020CDE92D
:10087000000001214FF0860B4FF0200E0AEB02031F
:1008800013F8019C09F00F03092B14DCA1FB03787A
:100890004FEAD37C00FB038301FB0C33DDE9008CC2
:1008A00018EB07074CEB030CCDE9007C4FEA191954
:1008B000B9F1090F12DDC4F800B07846C5F800E0C0
:1008C0003060862007B0BDE8F08FFFE78820206009
:1008D00009202860784630608820F3E74FF00A0C42
:1008E000A1FB0C3800FB0C80002701FB0700A3FBD9
:1008F000091800FB09874FEAE97C03FB0C77DDE967
:10090000008C18EB01014CEB070CCDE9001C4FF0FB
:100910000A0CA3FB0C18002700FB0C8003FB07004C
:10092000521EABD10698DDE90023C10001208840AA
:10093000401EC117801A994107D2892020600420E7
:100940002860784630608920BCE76946069A04989A
:100950003BF077FF00202060286078463060002060
:10096000B0E730B500B90120401E80B240F2B55367
:10097000B0FBF3F2B0FBF3F403FB14009206401C4F
:10098000120E80B24FF4B77398420BD9521CD2B2F8
:10099000A0F5B77003E0521CD2B2A0F26D1080B285
:1009A0009842F8D2202801D2012319E01F3880B2E2
:1009B000930701D01C2300E01D23984201D8022395
:1009C0000EE0C01A854D002380B2643503E0001BA1
:1009D0005B1C80B2DBB2EC5C8442F8D3DB1CDBB284
:1009E0000A704B7088707A49002008607949086065
:1009F000784679490860002030BD10B5027840F291
:100A00006D135A430A80754C43786E3434F81330B2
:100A10001A440A8083781A4493B20B8002789407B0
:100A200005D14078022802D803EB920003E00120B0
:100A300000EB920018440880654900200860654971
:100A40000860784664490860002010BD10B58178C0
:100A50004FF0FF32C9B143780D2B18D2DFE803F015
:100A600017070D070A070A07070A070A07001F29C1
:100A70000BD80FE01E2908D80CE00078800702D0C0
:100A80001C2902D806E01D2904D9104610BD6FF0BC
:100A9000010010BD002010BD18B502880024B2F579
:100AA000FA6F0ED9C2788DF8022082788DF8012075
:100AB0000078A0F5FA608DF800006846FFF79DFF0A
:100AC00000E00C8042480460424804607846424995
:100AD0000860002018BD2DE9F04F884600213C4DEC
:100AE0003C4E3D4F82464FF08609B3EB420F15D383
:100AF00001201EE0A2EB000B1AF80B4004F00F04DB
:100B0000092C0BDCA3EB400E0EEB080C30348CF8F8
:100B100001401AF80B402409092C06DDC5F80090A5
:100B20007846316038608620CDE6303408F80E40D3
:100B3000401C9042DED9012000EB4200302204E04C
:100B4000A3EB000C401C08F80C209842F8D929604F
:100B50007846316038600020B5E67CB50D4601A9C5
:100B6000FFF7FFFE1A4C000601D520687CBD9DF8FA
:100B7000040000909DF805309DF8062018A1284635
:100B80003BF088FB1349002020600860784612493A
:100B9000086000207CBD3C2310B5B0FBF3F2B0FB35
:100BA000F3F403FB1403D2B20A20B2FBF0F43034A6
:100BB0000C70B2FBF0F400FB142230324A703A227F
:100BC0008A70B3FBF0F23032CA70B3FBF0F20FE080
:100BD0000CC0072010C0072014C00720EEE403005B
:100BE000253032752D253032752D253032750000B7
:100BF00000FB1230303008713D49002008603D494B
:100C0000086078463C490860002010BD3C2310B5C0
:100C1000B0FBF3F2B0FBF3F403FB1400374BD2B29A
:100C20009A5C0A70185C48703149002008603149AC
:100C30000860784630490860002010BD18B50C46A1
:100C40006946FFF78EFE2A49000601D5086818BDDF
:100C50009DF802202948825C22709DF80120825C68
:100C600062709DF80020805CA0700020086021491F
:100C70000860784620490860002018BD70B5044619
:100C800011B93BF0B3FD0146002220230DE0A05C2A
:100C9000F02801DB103802E0C02802DB4038A05405
:100CA00002E0802800DBA354521C8A42EFDB0020C4
:100CB00070BD70B5044611B93BF098FD01460020A7
:100CC000202311E0225CF02A01DB23540BE0E02A10
:100CD00001DB103206E0B02A01DB403A02E0802A54
:100CE00001DB40322254401C8842EBDB002070BD07
:100CF0000CC0072010C0072014C00720EEE403003A
:100D0000F8B56A4E0D4607460222694630462FF076
:100D100073FA674C000615D4BDF800002A4640F06F
:100D2000804039462FF073FA00060BD4BDF800005E
:100D300002222844ADF80000694630462FF067FAD9
:100D4000000601D52068F8BD5A49002020600860DF
:100D50007846594908600020F8BD08B50020ADF874
:100D600000000222694651482FF051FA08BD0146A1
:100D700002224E482FF040BA2DE9F04188B00025FC
:100D8000022201A949482FF037FA494C00064ED4F7
:100D9000012035F02FFD000649D448490888420655
:100DA00006D520F04000088019F03FFE00063ED432
:100DB000002705A8059705F0ABFB000637D406A869
:100DC000069705F0B4FB000631D43D4902200870B7
:100DD00004A962201AF080FD000628D400264FF0F6
:100DE000200829E046F08040012203A92FF004FAF0
:100DF0009DF81000400714D49DF80C0043280DD036
:100E0000F3280BD0F42809D0F5280AD16D1CEDB2D7
:100E10008DF80C80022D04D1002502E00DB18DF873
:100E20000C80012103A835F0FAFA000603D52068EA
:100E300008B0BDE8F081761CBDF804008642D1D32D
:100E40001C482760076078461B4908600020EFE7D0
:100E500010B5FFF782FF164C000604D4052035F0CC
:100E6000C9FC000601D5206810BD12490020206091
:100E70000860784610490860002010BD10B50C4C81
:100E800018B1FFF76AFF000604D4012035F0B2FC68
:100E9000000601D5206810BD0649002020600860CA
:100EA000784605490860002010BD0000480F00206A
:100EB0000CC0072010C0072014C0072002C0072064
:100EC00000C00720F8B516460D46044689480122A1
:100ED00069462FF091F9000602D587480068F8BDF1
:100EE0009DF80000204000D001202870022C06D080
:100EF0008048401C022231462FF07EF9F8BD7D4823
:100F0000C01CF7E710B5A2B01EA80BF03AF87A4C57
:100F100000064BD41DAA1FA90120FFF7D3FF00062E
:100F200044D49DF87C0028B1BDF87400BDF8781059
:100F3000884209D9714900202060086078467049CC
:100F40000860002022B010BD022035F0EFFA000644
:100F50002CD46C4835F023FF000627D469481430A0
:100F600035F01DFF000621D41DAA1FA90220FFF79E
:100F7000A9FF00061AD49DF87C00C8B120A9BDF8CD
:100F80007400FFF7EEFC000610D49DF880005D4968
:100F900000909DF881309DF88220263101A83BF019
:100FA00079F901A835F0FBFE000601D52068C9E7F4
:100FB0005548018841F0020101805449022008701F
:100FC000012010F0AFFDBDE7FEB501A80AF0D9FF82
:100FD000494C000632D46A4602A90220FFF772FF8C
:100FE00000062BD49DF80800444D454E28B1BDF8AD
:100FF0000000BDF80410884206D900202060286057
:10100000784630600020FEBD022035F08FFA0006E1
:1010100014D43C4835F0C3FE00060FD439481430D0
:1010200035F0BDFE000609D43748018841F00201C1
:101030000180012010F076FD000601D52068FEBD7C
:1010400091202060BE202860784630609120FEBD4F
:101050004FF0A0430146042218462FF0CDB84FF0C0
:10106000A0430146042218462FF0D1B8F7B5044634
:10107000204882B00E460546012269462FF0BCF892
:101080001D4F00060ED49DF800000EB1204300E075
:10109000A0438DF800000122694628462FF0B7F8DA
:1010A000000602D5386805B0F0BD022C06D0114804
:1010B000401C022204A92FF0AAF8F4E70D48C01C36
:1010C000F7E738B500200122014600901046FFF7EF
:1010D000CDFF094C000606D4012200210220FFF7B3
:1010E000C5FF000601D5206838BD6846FFF7B7FF89
:1010F00038BD0000040000500CC0072010C00720BD
:1011000014C0072076E5030002C0072000C00720B6
:101110002DE9F04F99B0012400250C94841A08950C
:1011200071EB030404DA16461C4607460D4603E03D
:101130000C46064617461D4600218B46059116E0D3
:1011400002220023304621463BF07FF806460C463B
:1011500002220023384629463BF077F80D4601224B
:1011600005991BEB020B41F1000107460591F007C1
:1011700001D1F807E4D001200021CDE9220124AA01
:101180000846279482E84300711E64F10000CDE90F
:101190001610CDE91475CDE9127500BFDDE9260101
:1011A00080468946C00729D1DDE92201C20702D164
:1011B000249AD2070AD03A1845EB0100CDE9222043
:1011C000DDE9241071186041CDE92410DDE9220128
:1011D000022200233BF039F8CDE92201DDE92401A8
:1011E000022200233BF031F8CDE924010222002342
:1011F000404649463BF029F8CDE92601DDE91201D8
:10120000C20704D0DDE92632181A8A410BDA14A984
:1012100022A800F066FA16A924A800F062FA12A922
:1012200026A800F05EFADDE9260110900D91C007B6
:10123000B4D00DF15008DDF85C2098E80B009E4614
:10124000DDE922C3E1469A46BCEB000C8B4106DB8C
:10125000DDE9248CB8EB0E037CEB020C0DDA17EB06
:10126000090345EB0A0CCDE9223CDDE9243CF318E7
:1012700044EB0C0CCDE9243CE2E7B9EB00006AEB4F
:101280000103CDE922032598B8EB0E0160EB0200C3
:10129000CDE92410DDE91210109B0D9A5B1A62EB68
:1012A0000002CDE926320023591A73EB0002FFF643
:1012B00075AF14E0DB1B60EB05004FF0000CB3EBE7
:1012C0000C0C70F1000C17DBCDE92230901B61EBA8
:1012D0000401021E71F100020EDBCDE92401DDE9FB
:1012E0002230D91B70EB050106DBDDE92421B6EBCA
:1012F000020C74EB010CDDDB002108461AE000BF94
:10130000DDE922720C9B089DA3FB07C805FB07853E
:1013100003FB0252CDE922C2DDE92672A3FB07C816
:10132000089D491C05FB078503FB0252CDE926C237
:1013300040F10000059AB1EB0B0370EB0202DFDB1A
:10134000DDE9261081F00101014304D04FF0FF30A8
:1013500019B0BDE8F08FDDE92410711A64EB0004C8
:101360002898C0E900140020F2E72DE9FF5F9CB047
:101370000020CDE90200CDE9040092462E9907AA8B
:101380000A20CDE90002994614AB0122491C1AF04B
:1013900097FE00287DD114AB08AA195C0C0902F84D
:1013A000104001F00F0402EB4001401C4C70082873
:1013B000F3DB9DF82F70DFF8408311460E2000BF4D
:1013C00058F82740461C255CA45D801E4E5D11F830
:1013D00004C001F805C00E55F2D5002002EB400410
:1013E00012F810106478904644EA01111954401C18
:1013F0000828F3DB19460020079B0DE01C1A0C445B
:101400000A5C14F8015D2E0146EA15150D5415010C
:1014100045EA12122270401CB0EB530FEED30823A2
:1014200012A914A8079AFFF717FA0028B2D114A935
:101430000FF02CF80028ADD10C2114A8FFF7F9F912
:1014400000287DD0DDE91501CDE90801082208A9B1
:101450000020131A0B440C5C13F8015D0D54401C62
:101460001C70B0EB520FF4D300252C462F462E46AD
:101470002846C3464FF00A0E1BF80010724630395A
:1014800001EBC101B1FBF2F3B1FBFEFC0EFB1C1141
:1014900000E0AEE04FF0640CA5FB0C2801EB8101ED
:1014A00003EB410104FB0C84002305FB03445518A6
:1014B0005C4107910A23A7FB031C06FB03C3002220
:1014C00007FB02321BF8003000F10100303B5F18CF
:1014D00042EBE3760828CFDBDDE91201401B61EB2C
:1014E0000401864A0023CDE912013AF037FECDE926
:1014F000122350EA01027CD01AAA0692CDE90054C8
:10150000DDE91C23FFF704FE002872D1DDE91A5043
:10151000A7FB051206FB052207FB00248346DDE935
:101520001C23084621463AF019FE14469846DDE988
:101530001223A2FB050603FB056302FB0B3100E04F
:101540006CE0DDE91C233AF009FE15469B4654EA9F
:10155000080203D0DDE92A01012618E0012000215C
:101560001AE000BFDDE92A72A0FB073C01FB07C1BE
:1015700000FB02111846BAEB000379EB010205D219
:1015800052464B463AF0EAFD10461946761CF317D0
:10159000371B73EB0803E5DBCDE91A0180460C46E7
:1015A00055EA0B0003D0DDE92C01012617E00120EC
:1015B000002119E0DDE92C72A0FB073C01FB07C10B
:1015C00000FB02111846BAEB000379EB010205D2C9
:1015D00052464B463AF0C2FD10461946761CF317A8
:1015E000771B73EB0B03E5DBA0FB085301FB083112
:1015F00000E012E000FB041152464B4628463AF048
:10160000ADFD10461946DDE91C233AF0A7FDDDE9E2
:10161000120150405940084303D0002020B0BDE8DB
:10162000F09F0120FAE7F0B5411E85B01E2932D2A5
:10163000012404FA00F111F0500F2CD0304FBE6895
:10164000401E2D4D8440083D69680C4229D1C1B22D
:1016500004912C49002301EBC001D1E90021CDE91F
:1016600002212849284A403901EBC001D1E9000193
:10167000CDE9000149F6BF601946FFF776FE002864
:10168000286801D0204300E0A0432860B8681F49C3
:10169000801B884202D3002005B0F0BD686820435B
:1016A000686028682040F7E7411E1E290ED20121FC
:1016B00001FA00F212F0500F08D0401E81400E488F
:1016C000083842688A434260012070470020704712
:1016D00000B501231846FFF7E7FF5B1C1E2BF9DD61
:1016E00000BD30B5D0E90023D1E90045C0E900458F
:1016F000C1E9002330BD000020C0072000E1F5054E
:1017000000000940F8E503007FF81A03404B4C0045
:1017100038B50446684604F05AF99DF800002040A8
:1017200038BD38B50446684604F051F9000602D5C4
:10173000FD48006838BD9DF8000020438DF800008A
:10174000684604F03BF938BD38B50446684604F0F5
:101750003EF9000602D5F448006838BD9DF8000047
:10176000A0438DF80000684604F028F938BD01B5A3
:10177000FEF750FD684604F041F9FEF760FD08BD34
:101780007CB5684604F044F9E74C000638D49DF86F
:1017900000000025082809D009280DD0E34825605D
:1017A00005607846E249086000207CBD684604F088
:1017B00040F9000624D40BE001A804F065FE000601
:1017C0001ED49DF8040001281CD013208DF80000C1
:1017D000684604F013F9000612D48DF8045001A8ED
:1017E00004F048FE00060BD48DF8045001A804F064
:1017F0004CF9000604D4432019F099F8000603D5EB
:1018000020687CBD0220E1E7012010F08BF97CBD4F
:101810002DE9F0410024022035F0FCFAC54DAE68F8
:10182000C54F4FF4FA7811E0A868801BB8420DD379
:1018300001202BF031FFC82140462EF0C5F80120D1
:101840002BF035FFAE68641C042C04DC00202BF068
:1018500015FF0028E8D1012C06D0022C07D0032C5C
:1018600009D0042C11D10EE001F0FAF80DE00220AD
:1018700028F095FA09E0B14C0120207002F082FCBA
:101880000020207001E02DF0A4FABDE8F041012015
:1018900035F0C0BA0EB568460EF073FD50B193280E
:1018A00003D1A2480068062801D00E2000E01120D4
:1018B000FFF75DFF9C4800680EBD2DE9F34F002740
:1018C00089B088460F703E4608A938460DF02AF8C0
:1018D000954C000639D49DF82000DFF85092DFF8CF
:1018E00050A2400607D407A804F081F800062CD4C3
:1018F0009DF81C0068B3694609980DF08FFD00063D
:1019000023D40125EB4605A9284604F07BFB0006FD
:101910001BD405EB85015944052205A8491F3AF05F
:1019200015FF00B101276D1CEDB2042DEBD9C7B135
:10193000834909980880452018F0F9FF000604D46F
:10194000012010F0EFF800060BD520680BB0BDE8C1
:10195000F08F26607946C9F800600020CAF80010B0
:10196000F4E788F80070F4E72DE9F34F85B0032021
:10197000002408700E462746214601200EF051FD36
:101980000106694802D5006807B0E0E70168DFF8A2
:101990009C91DFF89CA10025052913D08046EB46D9
:1019A000694601200EF017FD0006D8F80000EBD4C0
:1019B00005280DD005220BF1040005993AF0C6FE6A
:1019C00018B103E0357005600DE0671C641CE7E7A3
:1019D00037B1BC4201D1022000E00120307000E0AC
:1019E0003570C8F800507946C9F800500020CAF890
:1019F0000010C9E730B5044685B0002020800220E1
:101A00000EF025FD484D05280BD0694602200EF04A
:101A1000E2FC00061ED4BDF800002188884200D9EF
:101A2000208001200EF013FD052802D06946012018
:101A300006E000200EF00BFD05280BD069460020C3
:101A40000EF0C9FC000605D4BDF8000021888842CC
:101A500000D92080286805B030BD2DE9F04387B05B
:101A60000646694600200EF011FD2F4D000649D4B0
:101A700003A90B200CF056FF000643D40C2203A947
:101A800068463AF063FE0227DFF8A080DFF8A090F6
:101A9000002408B137703EE003A910200CF042FF8B
:101AA00000062FD4694604200EF0F0FC000629D46D
:101AB000BDF80000BDF80C108842EBD16946062045
:101AC0000CF030FF00061DD4BDF80000BDF80C106E
:101AD000401E8142DED169460E200CF023FF000635
:101AE00010D403A8FFF786FF00060BD4BDF8000052
:101AF000BDF80C108842CDD3694600200CF012FFCF
:101B0000000603D5286807B0BDE8F0839DF8000003
:101B10004007BFD534702C607946C8F800400020DB
:101B2000C9F80010EFE700000CC0072010C0072024
:101B300014C0072000000940C0C62D0048C007207F
:101B400094C10720FEB502A803F062FFFC4C00061A
:101B500037D49DF808000025FA4EFB4F1D2812D0FF
:101B600003F063FE08B103F0E2FD01A803F097FF64
:101B7000000626D49DF8040028B1012809D00228C7
:101B80000BD003280ED025607846356038600020E1
:101B9000FEBD012007F040FE01E008F083FC0006D6
:101BA0000FD410E08DF80050684604F063FC000686
:101BB00007D4432018F0BBFE000602D40CF07EFCD4
:101BC000EDE72068FEBD01200FF0ACFFFEBD2DE962
:101BD000F0418AB0002606A80EF0D3FBDFF8688338
:101BE000D74CD84D932806D1286808286DD00528F1
:101BF0006BD0062833D0002108460EF012FC0006F8
:101C000063D405A900200EF0D9FE00065DD4CF4FA5
:101C1000387858B1002101200EF003FC000654D49E
:101C200005A901200EF0CAFE00064ED409A804F052
:101C300048FF000649D49DF8240038B30021012054
:101C40000EF0EFFB000640D4694601200EF0C3FB06
:101C500005280DD00120397881430ED10AE00020FB
:101C6000206079462860C8F800100AB0BDE8F0810D
:101C70000020F0E73978884308D0932020600820BE
:101C8000794628609320C8F80010EEE702200EF095
:101C9000DEFB000619D4694602200EF09CFB00060C
:101CA00013D4002102200EF0BCFB00060DD405A9C0
:101CB00002200EF083FE2068932806D128680828A9
:101CC00003D1761CB6B2032EF1D32068CDE72DE9FF
:101CD000F04F97B012A803F08AFE994C00066ED41C
:101CE00013A804F0EEFE0006F9D4DFF86082102697
:101CF000DFF8549298F80000924D4FF0000A4FF030
:101D0000160B9227C0B107A80CF073FD40F3C0106A
:101D1000401C8DF8300011D09DF82D00010637D5FC
:101D20009DF84C1099B38DF80060684603F066FE8C
:101D3000032027602860ABE18DF830A09DF84C00AF
:101D400098F80010084217D02868032811D00428FA
:101D50000FD08DF800B000BF9DF80000FFF707FD21
:101D6000286809282BD9462018F0E1FD302027608B
:101D7000E0E78DF80060EFE7FFF7E4FE8EE100BFDB
:101D80008DF80000684603F039FE17B0DFE5FFE785
:101D9000C00603D50CF092FB0006A0D4FFF717FF96
:101DA000DFF8AC8193280BD09DF82D0000077DD57E
:101DB0000CA90AA8FFF7D8FD00285ED114E06CE159
:101DC000FFF7C0FE00068AD40E208DF8000068469A
:101DD00003F014FE000687D400215EA034F015FE47
:101DE000614902200870C8E19DF83000022804D043
:101DF00001287DD000287CD0E9E19DF82D00400726
:101E000078D501A80CF077FC002874D103E000BF5E
:101E1000FFF7ADFCD9E10FA904200EF037FB000657
:101E2000F8D4BDF83C00BDF80410401C81427CD1C0
:101E30009DF82D00800602D5FFF784FE11E015A85D
:101E400003F02DFE0006E5D49DF85400012815D0BE
:101E5000FFF778FE0006DDD412A803F0C8FD0006E7
:101E6000D8D4BDF8040014A9FFF727FD2068822804
:101E7000D0D0922863D093287AD133E110A803F010
:101E800052FE0006C6D410AEB01C03F05DFE000684
:101E9000C0D4301D03F069FE0006BBD433499DF861
:101EA00044000870684603F0B3FD00E06CE10006F2
:101EB000B0D49DF80000042809D005283AD01D2888
:101EC0002BD0FFF73FFE684603F0A2FDC7E703F003
:101ED000ACFC30B103F02BFC10A805F041F8000673
:101EE00098D4012600270EA9304603F054FF03E0E2
:101EF00099E0A3E08EE0F1E000068BD40E98761C0A
:101F0000F6B20744102EEED93FB11D208DF8000027
:101F1000684603F073FD000695D4B8F8001010A8C9
:101F200041F00401A8F8001000E022E005F018F8E4
:101F3000000688D405F078FE000684D4C3E753E099
:101F40000CC0072010C0072014C007201C0400008C
:101F500002C007208E9888818A80208F808C9F9273
:101F600088208F840A0A000000C0072071C3072060
:101F70003DE0FFF7E7FD000684D49DF82D009DF8B5
:101F8000481000F04000491E084306D1BDF83C103F
:101F9000BDF80400891C884214D00CF08FFA0006AA
:101FA0007BD414208DF80000684603F027FD00065E
:101FB00073D44E2018F0BBFC00066ED401200FF045
:101FC000B1FDE2E6401E80B214A9FFF776FC20685E
:101FD000822862D0922802D0932803D182E0286818
:101FE00008287DD11320CBE62868082878D19DF8F1
:101FF000500008B11520C3E6684603F009FD00064D
:102000004BD49DF800001D2869D047E00120B7E6B9
:102010000220B5E68DF80060684603F0EFFC00068C
:102020003BD4332007E08DF80060684603F0E6FCFF
:10203000000632D4412018F07AFC9EE0FFF782FDC2
:1020400000062AD49DF82D004FF0310610F0600FE5
:1020500029D09DF84C0008B38DF800B0684603F015
:10206000CDFC000619D4422018F061FC69465320CB
:1020700019F032FC000610D49DF8000010F00200A8
:102080008DF8000002D001200FF04CFD27602E607B
:1020900079469220C9F8001077E680E09DF8480064
:1020A0000028B5D0B2E701A80CF025FBB0B914A800
:1020B000FFF7D3FC822872D0922811D0932811D038
:1020C0009DF8500080B1022836D088202060022080
:1020D000794628608820C9F8001056E600E076E0CE
:1020E0000F2095E60E2093E60FF056FA01200FF030
:1020F00019FD5E2018F01BFC0CF05FFF000664D495
:10210000FE4D0121FD480FF096FD00060AD5FEF7B1
:1021100081F80CF0D3F9000657D4FEF790F8207838
:10212000000652D40CF085FF00064ED495F840000E
:102130000028E6D1182019E09DF84C0080B18DF8F8
:1021400000B0684603F05AFC00063ED4422018F066
:10215000EEFBB8F8001041F00201A8F8001092E779
:102160009DF8480008B1012000E002208DF8000031
:10217000684603F043FC000627D4B8F8001041F08D
:102180000201A8F8001019E7FFF7DCFC9DF84C00ED
:1021900000289DF848000DD010B10C2001E014E09B
:1021A0000D208DF80000684603F028FC00060CD4D2
:1021B000402040E708B1012000E002208DF8000037
:1021C000684603F01BFC000601D52068DDE5C4F875
:1021D00000A07946C5F800A00020C9F80010D4E599
:1021E00038B5C748C74C007820B10420FFF71BFA68
:1021F00040B125E00620FFF716FA08BB0420FFF7E0
:1022000012FAE8B90120FFF70EFAC8B9372018F022
:102210008EFB6946532019F05FFB000601D520684C
:1022200038BD9DF8000010F002008DF8000007D0C6
:10223000B548018841F00201018001200FF072FCD5
:10224000B2490020206008607846B149086000204B
:1022500038BD38B5684603F0DBFBAA4C000629D42C
:10226000AC4D2878752827D00220FFF751FA70B1BD
:102270007B202870684603F0D2FB00061AD41C208D
:102280008DF80000684603F0B9FB000612D4012067
:10229000FFF73EFA80B151202870684603F0BFFB7B
:1022A000000607D417208DF80000684603F0A6FB4F
:1022B000000601D5206838BD9DF800000F2801D127
:1022C0007E2028709149002020600860784690495F
:1022D0000860002038BD2DE9FC41804603202BF02A
:1022E00093FE8A4E8A4F874C002530B9B8F1000F13
:1022F00003D00420FFF70CFAE8B36946532019F025
:10230000EBFA9DF8000010F002008DF8000002D0FA
:1023100001200FF007FC3D2018F009FB9DF800009C
:1023200010B101200FF0FEFB7A4975200870684655
:1023300003F06EFB00061BD4684603F081FB000629
:1023400016D401A803F053FB000611D49DF8040035
:1023500008B1192000E01A208DF80000684603F04B
:102360004DFB000604D40420FFF7DBF9000603D57B
:102370002068BDE8FC8106E0822020607846356058
:1023800038608220F5E725607846356038600020A7
:10239000EFE72DE9F0438BB000273E4607A803F096
:1023A00037FB584C00067DD49DF81C00DFF85C819B
:1023B000DFF85C910025022803D0192801D01A28E3
:1023C00071D103A9352019F087FA00066AD49DF867
:1023D0000E0000F00F01000900EB800001EB40004F
:1023E00000F5FA60ADF814009DF80D0000F00F0143
:1023F000000900EB800001EB40008DF816009DF80D
:102400000C0000F00F01000900EB800001EB400020
:102410008DF8170009A905A8FEF73EFB03A9362091
:1024200019F05AFA00063DD49DF80E0000F00F0195
:10243000000900EB800001EB400000F5FA60ADF808
:1024400014009DF80D0000F00F01000900EB800062
:1024500001EB40008DF816009DF80C0000F00F0114
:10246000000900EB800001EB40008DF8170008A97F
:1024700005A8FEF711FB684609F083FD00067AD433
:1024800004A82BF0FDFD000675D4BDF82400A0B112
:10249000BDF80010814210D39DF8100017280CD20F
:1024A000012701E067E055E003AB35223946022001
:1024B000039519F04BFE00065DD4BDF8200088B1ED
:1024C000BDF8001081420DD39DF8100050B10126D7
:1024D00003AB362231460220039519F037FE000681
:1024E00049D4BFBB56EA070054D006A9342019F0DE
:1024F000F3F900063FD49DF818000DE008C7072047
:102500001C0400000CC0072002C0072010C00720D8
:1025100014C0072070C30720012827D0022804D048
:10252000032837D14D497D20087006A9532019F0A2
:10253000D3F900061FD49DF8180010F002008DF8A2
:10254000180004D001200FF0EDFA000613D416B1E4
:10255000482001E01EE0472018F0E9F99DF8180036
:1025600020B101200FF0DEFA000604D404A82BF0FD
:1025700087FD000603D520680BB0BDE8F0839DF809
:1025800010000EB1401E00E0401C8DF8100004A8A1
:102590002BF0DBFD25607946C8F800500020C9F813
:1025A0000010E9E738B50546684603F031FA2C4CCF
:1025B000000604D4284603F01AFA000601D5206864
:1025C00038BD9DF8001006290FD008DC01290CD079
:1025D00003290AD0042908D0052908D105E00729D4
:1025E00003D0132901D0152901D1012028701D49DC
:1025F00000202060086078461B490860002038BD34
:1026000038B50546684603F014FA154C000618D490
:102610009DF80010072916D006DC0DD2DFE801F086
:102620000C130C13131313000E290CD013290AD00A
:10263000152908D01B2906D0284603F0D8F9000632
:1026400003D5206838BD012028700649002020608D
:102650000860784604490860002038BD70C3072030
:102660000CC0072010C0072014C0072010B58AB086
:1026700005A834F0DFFACF4C000637D4684634F0B2
:10268000D9FA000632D40220ADF80A00ADF80200F3
:10269000ADF804000A20ADF806000021684634F0C9
:1026A00045F8000622D40021C3A034F0AEF900069C
:1026B0001CD40021C3A034F0A8F9000616D40121CF
:1026C000084633F0C9FF000610D40021BEA034F044
:1026D0009CF900060AD4002105A834F027F800066A
:1026E00004D4012033F022FF000602D520680AB08E
:1026F00010BD34F030FBFAE72DE9F04F83469DB072
:102700000D46084633F03EFFAA4C00067DD45846DD
:1027100033F0D9FF00067DD42B465A46B1A1684656
:1027200039F0B8FD0021684634F06FF9000671D425
:10273000B2482A22C589684629463AF078F90A2023
:102740000DF805000DF101014FF0000905F80190A9
:102750004946684634F059F900065BD434F009FC68
:10276000DFF89CA20646DFF89C829AF80000022857
:1027700005D000EB400108EBC10040688047A24F44
:10278000BD680021A14834F040F9000642D4002180
:102790009E4834F03AF900063CD4002189A034F078
:1027A00034F934F0E6FB861BB868411B4FF47A70AD
:1027B000B1FBF0F59AF80000022805D000EB4001CB
:1027C00008EBC1004068804706EB4600C0EBC6102E
:1027D00005EBC000401EB0FBF5F7ABF1010034F093
:1027E000CBFB4FF47A714E436843B6FBF0F2FF1D0A
:1027F000FB0887A1684639F04DFD684634F0CFFAF2
:10280000000607D400218AA000E003E034F0FDF8C0
:10281000000603D520681DB0BDE8F08F8549C4F8D7
:1028200000907846C1F80090834908600020F2E7E4
:1028300070B58AB0064605A834F0FCF95D4D000677
:102840003CD4684634F0F6F9000637D40121ADF8DF
:102850000210ADF80060BDF81400ADF80410ADF83A
:102860000A10ADF80610401E34F08DFBBDF82210A2
:1028700000FB01F4BDF80000401E34F084FB94FB23
:10288000F0F0ADF80E000121684633F04FFF00066E
:1028900014D40424032E02D10D2C00D10E24214681
:1028A0003046FFF729FF000608D4E41C0F2CF1D3B3
:1028B000002105A833F03AFF000602D528680AB0C7
:1028C00070BD5C4900202860086078465A4908605D
:1028D0000020F4E710B5002033F0F5FE354C00067B
:1028E00035D400213EA034F090F800062FD4012109
:1028F000084633F0B1FE000629D400214FA034F081
:1029000084F8000623D40221012033F0A5FE00063E
:102910001DD4002149A034F078F8000617D4012115
:10292000022033F099FE000611D4002143A034F0B8
:102930006CF800060BD40221084633F08DFE000629
:1029400005D400213DA034F060F8000601D52068D0
:1029500010BD38490020206008607846364908607C
:10296000002010BD10B5012033F0E0FD114C000631
:1029700019D40121084633F06FFE000613D4052058
:1029800033F000FE00060ED4204B1822A53364213C
:10299000002033F0FEFF000605D400212AA034F009
:1029A00034F8000601D5206810BDBDE810400120B4
:1029B00033F02CBF0CC00720465072696E742D3561
:1029C000350000000A00000084A5ACAEADE1E2E0F5
:1029D000A0E6A8AEADADA0EF20AFA5E7A0E2EC0A5F
:1029E000200A0000200A98908894922025752C20B7
:1029F0009F908A8E91929C2025750A0000DD072009
:102A0000CAC30720CCC3072000000940D8E6030052
:102A1000D1EAEEF0EEF1F2FC3A20257520D1D2D0C9
:102A20002FD12028257520CCCC2FD1290A000000D9
:102A30000A200A0010C0072014C0072031323520B8
:102A4000544543540A0000002034203630323234DA
:102A500032203030313733370A200A200A00000094
:102A600070B5AEB0022033F061FDAD4D00067CD4F0
:102A70000221084633F0F0FD0006F8D4A9A2ACA16B
:102A800002A839F007FC002102A833F0BEFF0121A3
:102A9000084633F0E1FD0006E9D4A6A034F07FF942
:102AA000012033F043FD9FA2A1A102A839F0F2FB5F
:102AB000002102A833F0A9FF02A801F076F802A8CD
:102AC00000F038FD002102A800F0F1FC02A801F09E
:102AD00081F8002102A800F04DFF02A801F0FDF8E6
:102AE000202220A998482DF087FB02AA95A197A043
:102AF00000F08FFC02A834F052F997A128A8209A80
:102B000039F0C8FB02AA28A995A000F082FC02A80F
:102B100034F045F990A128A8219A39F0BBFB02AA0C
:102B200028A994A000F075FC02A834F038F98AA115
:102B300028A8229A39F0AEFB02AA28A992A000F098
:102B400068FC02A834F02BF983A128A8249A39F054
:102B5000A1FB02AA28A990A000F05BFC02A834F017
:102B60001EF97DA128A8259A00E0CFE039F092FB5C
:102B700002AA28A98DA000F04CFC02A834F00FF99D
:102B800075A128A8269A39F085FB02AA28A98CA04D
:102B900000F03FFC02A834F002F9684633F0E6F892
:102BA0008BA128A8009A39F075FB02AA28A98AA04F
:102BB00000F02FFC02A834F0F2F802A800F005FDA6
:102BC0008AA034F0ECF82CA831F0B6F92C98012842
:102BD0002ED004282ED088A102AA89A000F019FCCA
:102BE00002A834F0DCF88A4C202202A8E18939F0EE
:102BF0001EFF0E2287A102A839F0AAFE2DA90120EE
:102C0000CDE9000101461EAB0222092019F058FA55
:102C100000067BD49DF8783001A80A22411E0A2BB9
:102C20004ED2DFE803F04D090D4D14181C2428493D
:102C30007CA1D1E77DA1CFE7E18908447CA102E036
:102C4000E18908447CA10968016002711DE0E18905
:102C500008447BA1F7E7E08908447BA102E0E08912
:102C600008447BA10A680260898881800DE0E089C0
:102C7000084479A1F6E7E1890DF10200084478A142
:102C80000B68036089888180827102A834F087F81C
:102C900002AA75A176A000F0BCFB02A834F07FF870
:102CA000784800788DF8780070B101280FD002289C
:102CB00002AA2ED023A10CE0E089084472A1D1E73A
:102CC000E189084472A1BEE702AA73A101E002AA49
:102CD00073A175A000F09DFB02A834F060F831F0FC
:102CE00006F8012033F092FD552017F020FE1FA8B2
:102CF00002F0E6FE000609D41FA802F0D9FA000689
:102D000004D41FA802F0D2FE000604D528682EB015
:102D100070BD6AA1DDE701200EF004FFF7E70000B7
:102D20000CC00720465072696E742D3535000000C6
:102D300025730A00C8CDD4CED0CCC0D6C8DF20CEF3
:102D400020CFC40A0000000008000020CDC0D0C081
:102D5000C1CED2CAC00000002531306C7500000021
:102D600020C02DCED2D0C5C7D72E2CC2D1C5C3CE40
:102D70000000000020C4C2C8C3C0D2C5CBDC2CC236
:102D8000D1C5C3CE0000000020C3CECBCEC2CAC086
:102D90002CC2D1C5C3CE000020C02DCED2D0C5C715
:102DA000D72E2CD1C1D0CED10000000020C4C2C883
:102DB000C3C0D2C5CBDC2CD1C1D0CED10000000025
:102DC00020C3CECBCEC2CAC02CD1C1D0CED1000040
:102DD0002532644300000000D2C5CCCFC5D0C0D29C
:102DE000D3D0C020C3CECBCEC2CAC800D1C2DFC7A9
:102DF000DC20D120CFCA0A00556E6B6E6F776E0053
:102E000020CAC0CDC0CB20CEC1CCC5CDC0000000F3
:102E100000DD072020D1CACED0CED1D2DC20C1DB4C
:102E2000CBC0000052532D323332000055534200C4
:102E3000313230300A000000323430300A000000F5
:102E4000393630300A00000031343430300A0000A6
:102E500033383430300A000035373630300A00005D
:102E60003131353230300A00343830300000000063
:102E700020D1CACED0CED1D2DC20C2D0C5CCC5CDD7
:102E8000CDCE0000CAC3072031393230300A0000ED
:102E9000343830300A000000C0D2CECB0000000031
:102EA000D8D2D0C8D500000020CFD0CED2CECACE46
:102EB000CB20CEC1CCC5CDC000000000C0D2CECB4F
:102EC00020CDCEC2DBC900002DE9F843F34DF44F0D
:102ED000DFF8D083002440B9694601202AF0AAFB1C
:102EE000000617D40098C0071DD0EF4E308880052B
:102EF00006D501220021104609F090FC000609D4F5
:102F00003078000609D501221146002009F086FC20
:102F1000000602D52868BDE8F883308810F4207FC9
:102F200008D1800406D42C6079463C600020C8F8A3
:102F30000010F0E74FF4FA74FA2120462CF044FD1B
:102F4000214600202CF040FDF6E72DE9F04F95B02A
:102F50004FF00009D14FDFF854B3CDF84890DFF8B7
:102F600040A33B68CBF80030DAF80000CE49DFF828
:102F70003483CBF804007F26CD4C0988D8F8002094
:102F80004D46892B10D010DC812BFBD006DC062BA4
:102F900077D2DFE803F0F7F776F7F7F7822B71D0F7
:102FA000862BEFD0872B6CD1ECE0932B14D00ADC6E
:102FB000A3F18A010929EBD2DFE801F0E46363633E
:102FC00063FBE4E43E00962B70D0A12BECD0A22B47
:102FD000FAD0A32BE7D12CE10A2819D008DC052868
:102FE00016D00628E0D0082812D0092806D10FE014
:102FF0000B280DD0802819D0812817D00090AD491A
:1030000001A839F047F9002101A833F0FEFC03E0E4
:1030100009B9A9A00DE00425AF4926700220087067
:103020004B2017F084FCFF2D3CD1EAE00029F2D1BF
:10303000AAA00EF042F9EEE7FDF7ECF813A803F0B2
:1030400040FDFDF7FCF89DF84C0000287DD0DAF833
:10305000000008282BD00ADC19D2DFE800F018287D
:103060002828282828283860CAF800003FE02A28A5
:1030700019D008DC09281AD0202814D0282806D115
:1030800011E0A8E040E0302838D0312836D00021C7
:103090009CA033F0BAFC26708F49022008704B20A8
:1030A00017F045FCA6E00EF0CAF82AE0BFE00EF0EB
:1030B000C6F88949CBF800900220CBF8049008703C
:1030C0004C4612A9532018F007FC00066FD4129842
:1030D00010F00200129007D09148018841F00201DF
:1030E000018001200EF01EFD3C60CAF800407946C8
:1030F0000020C8F8001015B0BDE8F08F082033F0AC
:103100006FFE7E202070C7E7252864D2DFE800F03C
:10311000631E1E2B2B256313296340323A634063E1
:103120006336633A3A6363631E2B3434633A6363F2
:103130003A5C5C632B0031B96749022008700021BA
:103140005DA033F062FC042553E06EE019B9002164
:1031500074A033F05AFC02254BE000217AA033F032
:1031600054FC012545E019B9002180A033F04DFC45
:1031700003253EE00A253CE009253AE08348007833
:103180000228F5D0CBF800904846CBF804906AE7C7
:1031900014A9622018F0A0FB000608D49DF8500086
:1031A0000007EFD5684602F09BFD000602D538689F
:1031B000A1E71AE09DF800000028E3D058480188F4
:1031C00041F080010180DDE719B9002170A033F0E2
:1031D0001CFC08250DE00090364901A839F05AF88A
:1031E000002101A833F011FC03E003281DD00728BB
:1031F0001BD026706D00FF2D03D012A9284600F0C9
:103200001DF80020FFF760FE694C6A4E207800EB45
:10321000400006EBC00040688047207800EB40008B
:1032200006EBC00080688047E5E748461BE70428B6
:10323000FBD079461846C8F800105CE770B504006A
:1032400008680D4605D0611E88420FD14FF4FA611F
:1032500010E05949584A363A31F9101032F9100045
:103260002CF063FB002818D11B240CE0C00703D00E
:103270004FF4FA71002002E0C8214FF416702CF0D0
:1032800054FB002809D101202AF02DFA2868401C9F
:103290002860A04201D10020286070BD0CC007202A
:1032A00010C0072014C0072004C007204CC007200E
:1032B00070C3072064D404008EE8A8A1AAA020AFA0
:1032C000A0ACEFE2A8208F84200A0A0A0A0A0A0AA0
:1032D0000A0A0A0A0A0A000000C0072091A1AEA942
:1032E00020AEA1ACA5ADA020E120AFA0ACEFE2ECF8
:1032F000EE208F84200A0A0A0A0A0A0A0A0A0A0A1F
:103300000A0A00008EE8A8A1AAA0209D8A8B870A3D
:103310000A0A0A0A0A0A0A0A0A0A0A0A0000000035
:1033200002C0072091A1AEA920AEA1ACA5ADA020FE
:10333000E1209D918F87930A0A0A0A0A0A0A0A0A5B
:103340000A0A0A0A000000008220E7A0E1A0E520A6
:10335000ADA5A2A5E0ADAEA520A2E0A5ACEF0A0AFE
:103360000A0A0A0A0A0A0A0A0A0A0A0091A1AEA966
:1033700020AEA1ACA5ADA020E1208E87930A0A0A59
:103380000A0A0A0A0A0A0A0A0A0A000088C4072066
:1033900091A1AEA920AEA1ACA5ADA020E1208F8F58
:1033A00087930A0A0A0A0A0A0A0A0A0A0A0A0A0081
:1033B000CAC30720CCC30720CCE703002DE9F041A6
:1033C000804633F0ECFC002821D04FF496764FF481
:1033D000FA77FE4CFE4D01202AF085F93146384639
:1033E0002CF0F2FA01202AF07EF9A068A168091AEF
:1033F000A942FBD333F0AFFC0028ECD10021F5A0AB
:1034000033F003FB4046BDE8F04133F0C8BCBDE8F3
:10341000F0812DE9F05F14468B46824639F0E6F9DB
:103420008146584639F0E2F9EB4D064609EB0600B5
:10343000E9890A274FF00008884217D22022204647
:1034400039F0F5FA4A465146204639F0FAF9E8894A
:103450003246801B2044594639F0F3F9E889275455
:10346000E989641C01F80480BDE8F09F012000EBAD
:1034700041012022204639F0DAFA4A4651462046D8
:1034800039F0DFF9E889324659462754E889C6EB16
:1034900040002044401C39F0D4F9E88904EB400096
:1034A0004770E98904EB410181F80280DCE730B51F
:1034B00085B00546002004900C4604A82BF018FFA8
:1034C000FCF7A8FE0499642091FBF0F200FB1212B5
:1034D0000A2392FBF3F391FBF0F2C0A1684638F0A7
:1034E000D9FE2A466946C0A0FFF793FF2846FFF79A
:1034F00065FFFCF7A4FEC348006814B111280ED084
:1035000010E011282A4608D0BFA1B6A0FFF781FF1E
:103510002846FFF753FF05B030BDBDA1F5E7206891
:10352000401C2060BCA16846226838F0B3FE2A46E1
:103530006946EAE770B5044688B0012032F0F6FF2C
:10354000A54E01252846FEF7AFF8002838D02A46B8
:10355000B4A1204638F09EFE2046FFF72FFFF189E8
:103560002022204639F063FA07A91420CDE9000192
:1035700002AB012229460A2018F0A2FD2846FEF7D8
:1035800052F850B1079A611C530002A8FDF7A3FA44
:10359000F189201F0844A7A109E00798582241009B
:1035A000601C39F044FAF189A01F0844A3A138F047
:1035B00071FEF289601C002111542046FFF7FEFEC7
:1035C0006D1C1E2DBEDB08B070BD10B504468CB05E
:1035D000012032F0ABFF9BA0FFF7F0FE9C490A8868
:1035E000A2F51940993820D09AA1684638F052FEC9
:1035F0002246694699A000BFFFF70BFF2046FFF760
:10360000DDFE09A90AA80DF0B4F9BDF8242091A1A6
:10361000684638F03FFE2246694691A0FFF7F9FE62
:103620002046FFF7CBFE0CB010BD8EA290A16846DD
:1036300038F030FE2246694688A0FFF7EAFE2046B1
:10364000FFF7BCFE8B4A8AA1684638F023FE22466B
:10365000694689A0FFF7DDFE2046FFF7AFFE884AE6
:1036600083A1684638F016FE2246694685A0C3E766
:1036700010B50420FEF755F80106844801D500680E
:1036800010BD002101605F480160784680490860F4
:10369000002010BD7F48002100F8081FFF2101769F
:1036A000017780F820107047F0B5074687B00C46C8
:1036B000002603202AF0A8FCD0B101263046FFF7EF
:1036C000D7FF002842D18DF800008DF801008DF859
:1036D000020040F2DA70ADF8140001208DF81600F7
:1036E0008DF8170005A82AF051FD68462AF02DFD37
:1036F00068462AF0C5FC35499DF802508868664A3C
:103700008B681B1A9342FBD368462AF0B9FC0EB1B2
:10371000FFF7C0FF9DF8020064B1A84202D1206803
:10372000401C20603CA101A8226838F0B3FD3A4655
:1037300001A905E0A8423A4601D033A100E034A136
:1037400056A0FFF766FE3846FFF738FE07B0F0BD1B
:1037500030B50C0054A187B00546D1E90001CDE990
:1037600000010DD02AF03CFD10B12068401C206003
:1037700029A102A8226838F08DFD2A4602A906E098
:103780002AF02EFD2A4608B121A100E01EA16846BC
:10379000FFF73FFE2846FFF711FE07B030BD30B5FA
:1037A00043A30C4605460FCB89B08DE80F0008A94E
:1037B00008460DF0DEF81348006828B109282A46AB
:1037C00003D03FA168467DE092E09AE00000094006
:1037D00020A107000A00000000DD072025752E2526
:1037E000303175C200000000C1C0D2C0D0C5DF209A
:1037F000D7C0D1CEC228322E32202D20332E3329ED
:103800000000000010C00720CDCED0CC000000008A
:10381000CDC5CDCED0CC00002530346420CED8C864
:10382000C1CECA00CACEC420C7C0D9C8D2DB2025A9
:10383000750A0000CDCED0CC0A000000CDC5CDCE9B
:10384000D0CC0A00494420D1C5D0C8C83A0A0000EB
:103850000404000025303475000000002031000011
:1038600020320000CED2CBC0C4CED7CDC0DF000006
:10387000257300001004000020C4E0F2E03A0000CC
:103880002004000020C2F0E5ECFF3A000CC0072045
:1038900014C0072000400240E0C81000D5CEC4206C
:1038A000D7C0D1CEC2000000CFCE20CFC4000000D0
:1038B000CFCE20CFC0CCDFD2C820CFC400000000C4
:1038C000CDC5D200FFF7A5FD6CB12068401C20607B
:1038D000AFF2BC0104A8226838F0DCFC2A4604A937
:1038E0006846FFF796FD2846FFF768FD09B030BD32
:1038F0002A46AFF2EC016846FFF78BFD002CE7D1BA
:10390000F1E7AFF2F4016846FFF783FD002CEAD03F
:103910002168491C2160DBE77FB50C46054618F09D
:103920006DFC88B1FD482A460068012809D0AFF235
:103930002011FBA0FFF76DFDC4B12068401C206082
:1039400009E0AFF28401F4E72A46AFF24411F4A093
:10395000FFF75FFD54B1AFF240116846226838F0BE
:1039600099FC2A466946EEA0FFF753FD2846FFF76B
:1039700025FD7FBD7FB50C4605462EF099F938B17F
:103980002A46AFF2C4010FE02068401C206018E016
:103990000BF041FF70B1E148016803290AD0042906
:1039A00008D02A46AFF29811DFA0FFF732FD002CB5
:1039B000EAD111E02A46AFF2B011DBA0FFF729FDF2
:1039C00054B1AFF2AC116846226838F063FC2A4665
:1039D0006946D5A0FFF71DFD2846FFF7EFFC7FBD28
:1039E00030B50546D2A085B000680C46049002F0C0
:1039F000C2FF000607D42A46AFF2F41104A8FFF76D
:103A000008FD74B918E0C5482A460068192817D07F
:103A1000AFF2541104A8FFF7FCFC6CB12068401C05
:103A20002060AFF20C216846226838F033FC2A4649
:103A3000694604A8FFF7EDFC2846FFF7BFFC6AE5DE
:103A4000AFF23421E6E72DE9F0438146B9A00C46F8
:103A50008BB007C801AB002683E80700012032F0D5
:103A600065FD08A80CF08DFCAC4D932803D12868A7
:103A7000062800D00126002108460CF0D2FC0027C1
:103A800012E02868082815D117B9ADA0FFF796FCF9
:103A9000BDF80020B1A14846521C38F0FBFB484657
:103AA000FFF78CFC01267F1C694600200CF086FF86
:103AB0000028E6D1DFF8AC82D8F80000932800D1C6
:103AC0000126002101200CF0ACFC002712E0286840
:103AD000082815D117B9A4A0FFF770FCBDF8002085
:103AE0009EA14846521C38F0D5FB4846FFF766FCBD
:103AF00001267F1C694601200CF060FF0028E6D1FA
:103B0000D8F80000932800D10126002102200CF0F3
:103B100088FC002712E02868082815D117B999A059
:103B2000FFF74CFCBDF800208CA14846521C38F031
:103B3000B1FB4846FFF742FC01267F1C6946022084
:103B40000CF03CFF0028E6D1D8F8000093280BD0F9
:103B50009EB14A46AFF2483101A8FFF75AFCF4B1D2
:103B60002068401C20600FE02868802801D0812850
:103B7000EFD14A46AFF2B821EEE74A46AFF27831CC
:103B800001A8FFF746FC54B1AFF2743104A82268D3
:103B900038F080FB4A4604A901A8FFF73AFC4846E2
:103BA000FFF70CFC0BB0BDE8F0833EB504462AF0ED
:103BB0001EFB00F00F03C0F3031278A1684638F033
:103BC00069FB2246694677A0FFF723FC2046FFF7F2
:103BD000F5FB3EBD70B58AB0064605A80CF0D1FBDA
:103BE00020B13F220C2105A838F021FF00258DF8D7
:103BF00020502022052105A838F019FF324605A9DA
:103C00006DA0FFF706FC3046FFF7D8FB00200CF054
:103C10001EFC544C20B9694600200CF0DCFB28B196
:103C20003F22142105A838F002FF08E00A230522EC
:103C300005A90DF10B00FCF74EFF00063AD48DF8F4
:103C40001E50324605A960A0FFF7E3FB3046FFF7A0
:103C5000B5FB9DF814003F2816D0BDF8000005A95B
:103C6000FCF77BFF000625D4324605A95CA0FFF7D0
:103C7000D0FB3046FFF7A2FB5E48007828B3012056
:103C80000CF0E5FB50B904E05BA105A838F08AFD13
:103C9000EAE7694601200CF09EFB20B156A105A879
:103CA00038F080FD09E0BDF8000005A9FCF755FFDC
:103CB000000602D520680AB070BD324605A951A0A1
:103CC000FFF7A7FB3046FFF779FB14482560056036
:103CD0007846514908600020EDE710B58CB00446E5
:103CE00018224EA105A838F033FE0BA802F0E9FE19
:103CF0009DF82C0008B14FA101E0AFF23C412246F3
:103D000005A8FFF786FB2046FFF758FB9DF82C001F
:103D1000002802D0694600208EE005E110C007208F
:103D2000DDD1CFCFC7D30000CFCFC7D30000000075
:103D3000CEC7D300CFE0ECFFF2FC20CFC4000000E0
:103D4000CFCEC2D0C5C6C4C5CDCDDBC520D4C8D169
:103D5000CAC0CBC8C7C0D6C8C83A0A002325303469
:103D6000750A00000CC00720CFCEC2D0C5C6C4C59E
:103D7000CDCDDBC520C0CAD2C8C2C8C7C0D6C8C84E
:103D80003A0A0000CFCEC2D0C5C6C4C5CDCDDBC572
:103D900020D1CCC5CDDB3A0A0000000025752E25C8
:103DA00075000000DDCBC5CAD2D0CECDCDDBC92099
:103DB000C1CBCECA00000000D1C5D0C8C9CDDBC977
:103DC00020CDCECCC5D00000D0C5C3C8D1D2D0C084
:103DD000D6C8CECDCDDBC920CDCECCC5D00000001D
:103DE000C4C0D2C020D0C5C3C8D1D2D0C0D6C8C8E4
:103DF000000000001C0400003F3F2D3F3F2D3F3FCF
:103E000000000000C4C0D2C020C7C0CCC5CDDB209C
:103E1000DDCACBC70000000014C00720CFC0CCDF34
:103E2000D2DC20CFC420C0CAD2C8C2C8C7C8D02ED6
:103E300000000000C4C000000CF06BFA002873D131
:103E4000BDF80020FCA101A8521E38F023FA22463A
:103E500001A9FBA0FFF7DDFA2046FFF7AFFABDF896
:103E60000000F5A1C0F1190201A838F013FA2246AA
:103E700001A9F8A0FFF7CDFA2046FFF79FFA69469F
:103E800002200CF046FA00284ED1BDF80020AFF217
:103E90003C6101A838F0FEF9224601A9F0A0FFF725
:103EA000B8FA2046FFF78AFA04A902200CF002FAB9
:103EB000002839D1BDF81000BDF80010421AAFF249
:103EC0006C6101A838F0E6F9224601A9E1A0FFF7EC
:103ED000A0FA2046FFF772FAE3480078002823D0C2
:103EE000694601200CF015FA00281DD1BDF800200C
:103EF000D1A101A838F0CEF9224601A9DBA0FFF735
:103F000088FA2046FFF75AFABDF80000CAA1C0F1AE
:103F1000400201A838F0BEF9224601A9CDA0FFF762
:103F200078FA2046FFF74AFA0CB010BDF0B5074604
:103F300095B00C46002503200AF095FDD04E0006F2
:103F400002D5306815B0F0BD0AF0A6FD000605D414
:103F500011A905200AF0E6FC00060AD514B1206874
:103F6000401C206001253F220A21684638F05FFD91
:103F700014E00A230522694611A8FCF7ACFD13A939
:103F800000200AF0CFFC000608D49DF84C00000683
:103F900004D514B12068401C2060012500208DF854
:103FA0000A006A46B7A105A838F074F944B1AFF227
:103FB00098710DA8226838F06DF93A460DA906E00F
:103FC00015B1AFF2B47101E0AFF2C4713A4605A881
:103FD000FFF71FFAFCF71EF93846FFF7EFF9FCF779
:103FE0002EF9AEE770B5AA4C0546B222E18938F049
:103FF0001EFDE1890A2068540321A6A032F09FFF2C
:1040000000240021284632F000FD641C0A2CF8D35D
:1040100032F0A1FEBDE87040082032F0E5BA70B57C
:1040200005460C469CA0FFF7C9F99DA0FFF7C6F90D
:1040300004F00F0003282ED09DA0FFF7BFF9E00782
:1040400008D02A46AFF638019FA0FFF7E2F92846CC
:10405000FFF7B4F9A00708D52A46AFF64C019CA09B
:10406000FFF7D7F92846FFF7A9F9600708D52A46D0
:10407000AFF6640198A0FFF7CCF92846FFF79EF948
:10408000200708D52A46AFF6780195A0FFF7C1F9B9
:104090002846FFF793F9C4F303100C2818D092A018
:1040A000FFF78CF9600608D42A46AFF69C018AA077
:1040B000FFF7AFF92846FFF781F9200608D42A4612
:1040C000AFF6B40186A0FFF7A4F92846FFF776F90A
:1040D000C4F303200A2818D088A0FFF76FF9600501
:1040E00008D52A46AFF6D8017BA0FFF792F92846FB
:1040F000FFF764F9200508D42A46AFF6EC0178A052
:10410000FFF787F92846FFF759F9C4F3033005286C
:1041100018D080A0FFF752F9600408D42A46AFF601
:1041200010116DA0FFF775F92846FFF747F9200435
:1041300008D52A46AFF6281169A0FFF76AF9284684
:10414000FFF73CF9C4F3034003281AD077A0FFF728
:1041500035F9600308D52A46AFF64C115EA0FFF78B
:1041600058F92846FFF72AF920030AD52A46AFF660
:1041700060115BA0FFF74DF92846BDE87040FFF7DE
:104180001DB970BD2DE9F043C1B0002438943994B5
:104190003A943B943C943D943E943F942AA8409496
:1041A00032F048FD364D00062CD40221ADF8B21095
:1041B00001212420ADF8AA10ADF8B600ADF8AC107E
:1041C000ADF8A8100821A0462046ADF8B440ADF8DF
:1041D000AE1032F0D8FE4FF4D874B4FBF0F0BDF856
:1041E000B610884208D2BDF8A800401E32F0CBFEBF
:1041F000B4FBF0F0ADF8B60001212AA832F096FA2F
:10420000000602D5286841B0CDE4022032F002FE5B
:104210004CA0FFF7D3F8012032F088F950A0FFF747
:10422000CDF8DFF8589199F8000018B154A0FFF7C5
:10423000C5F8C1E0AAE0000025303275000000009A
:1042400020CFC5D0C5D0C5C3C8D1D2D0C0D6C8C96B
:10425000000000002020D1C2CEC1CEC4CDCE0000CF
:1042600020D1CCC5CD0000001C04000020C0CAD263
:10427000C8C2C8C7C0D6C8C920DDCACBC7000000A5
:104280000CC00720DDCACBC72028257329000000F9
:1042900000DD07201B3300003F3F3F2000000000EF
:1042A000205749464920D7C0D1D2DC0A000000007F
:1042B00020C2D1C520D1C8C3CDC0CBDB20CDC0200A
:1042C000C2D5CEC40A0000002020CFC8CD203700C0
:1042D0002020CFC8CD2038002020CFC8CD203600E8
:1042E0002020CFC8CD20350020CFC8CD203720C812
:1042F00020CFC8CD203820C220300A0020CFC8CD22
:10430000203720C220302C20CFC8CD203820C2201A
:10431000310A000020CFC8CD203720C220312C2008
:10432000CFC8CD203820C220300A000020CFC8CD11
:10433000203720C220312C20CFC8CD203820C220E9
:10434000310A00003D20D2C5D5CDCECBCEC3C8D7D3
:10435000C5D1CAC8C920CFD0CEC3CECD203D0A001A
:10436000D2C5D1D220CDCEC6C020C0C2D2CECED2F0
:10437000D0C5C7D7C8CAC00A0000000089C5072039
:10438000CFD0CECFD3D9C5CD0A000000082032F05F
:1043900027FD00240021FDA032F037FB30B90120B9
:1043A00032F0E6FC10B932F0D6FC08B1FEF7CDFDD4
:1043B000641CA4B20A2CEDD3012032F0B7F8F4A0AB
:1043C000FEF7FCFF082032F00BFDF94F002600201D
:1043D00029F054F950B1022032F0A8F8AFF2600091
:1043E000FEF7ECFF012032F0A1F808E032F053FDB7
:1043F00038880643B6B27007E9D5B007E7D532F082
:104400004AFD38880028FAD1EA4CA068EA4DA16834
:10441000091AA942FBD3E9A0FEF7D0FF012032F030
:1044200085F822A80BF0ADFF20B13F220C2122A875
:1044300038F0FDFA8DF894802022052122A838F06A
:10444000F6FA03AA22A9E2A0FEF7E3FF03A8FEF70B
:10445000B5FF27A829F045FE18B928A829F010FEB5
:1044600020B1DCA103A838F09DF912E0BDF89C2032
:104470009DF8A1109DF8A000A2F5FA620092CDE986
:1044800001019DF89E309DF89F20D7A103A837F029
:1044900001FF032032F04AF803A8FEF78FFF012046
:1044A00032F044F803A8FFF745F8D6A2D8A103A834
:1044B00037F0F0FE002103A832F0A7FA03A8FFF7B7
:1044C00074FBD4A0FEF77AFF32F0E5FC387899F857
:1044D000001000F01000084303AA0DD0AFF6D04141
:1044E000CFA0FEF796FF03A8FEF768FFB00703AA68
:1044F00005D5AFF6EC4104E0AFF6F441F0E7AFF6D6
:10450000F041CCA0FEF785FF03A8FEF757FF700728
:1045100003AA02D5AFF6105101E0AFF60C51C7A0C7
:10452000FEF777FF03A8FEF749FFC6A0FEF746FF98
:10453000002108462FF095FF012100202FF091FF68
:1045400040B9022100202FF08CFF18B103AAAFF66A
:10455000485102E003AAAFF64851BEA0FEF759FF4A
:1045600003A8FEF72BFFBEA0FEF728FF082032F0BD
:1045700037FC002029F082F808B1012600E000266F
:10458000012100202FF06DFF30B1022100202FF01B
:1045900068FF08B1012700E000273E43E9D003206F
:1045A00031F0C4FF0FB1B1A000E0B3A0FEF706FFE9
:1045B000012031F0BBFF032100202FF052FF00202B
:1045C00029F05CF80028FAD1AEA0FEF7F7FE002132
:1045D00002202FF046FF012102202FF042FF40B9B8
:1045E000022108462FF03DFF18B103AAAFF6E851AB
:1045F00002E003AAAFF6E85196A0FEF70AFF03A86F
:10460000FEF7DCFE96A0FEF7D9FE082032F0E8FBAC
:10461000002029F033F808B1012700E0002701212C
:1046200002202FF01EFF30B1022108462FF019FFA3
:1046300008B1012600E000263743E9D0032031F01D
:1046400075FF0EB189A000E08BA0FEF7B7FE012038
:1046500031F06CFF032102202FF003FFA068A16856
:10466000091AA942FBD3002029F008F80028FAD142
:1046700088A0FEF7A3FE01202FF020FB002029F0E8
:1046800046FF03AA98B1AFF6786172A0FEF7C1FEAB
:1046900003A8FEF793FE72A0FEF790FE082032F00A
:1046A0009FFB002028F0EAFF20B1012703E0AFF6CE
:1046B000A861EAE70027012029F029FF08B10126B7
:1046C00000E0002636EA0700EBD1032031F02EFF90
:1046D000EEB369A0FEF772FE012031F027FF002043
:1046E00028F0CCFF0028FAD1002103A8FEF7DCFF58
:1046F000002103A8FEF7DBFE002103A8FFF728F83E
:10470000002103A8FFF74BF8002103A8FFF768F981
:10471000002103A8FFF700F9002103A8FFF72AF9F9
:10472000002103A8FFF78FF903A8FFF7D6FA0021AD
:1047300003A8FFF7FBFB2AF049F9A0F1C87118396B
:1047400008D02AF043F9B0F5881F03D0BBE0FFE79B
:1047500046A0BFE7202130A838F093F9AFF2C84057
:10476000006830902AF07EF84D4A0146219080186A
:1047700008D0A0F6C300B0F5804004D0494AD0422A
:1047800002D191E0EDE0E5E09AE000000A0A0A00BB
:10479000D2C5D1D220C4C0D2D7C8CACEC220CAD0B6
:1047A000DBD8CAC820C820C1D3CCC0C3C80A000007
:1047B000D4C507200000094020A107003D3D3D2051
:1047C00020CFD0CEC3CECD203120203D3D3D0A00AC
:1047D000CFC4000058582D58582D585858582058B4
:1047E000583A58580A000000253032752D253032CD
:1047F000752D2530327520253032753A25303275C9
:104800000A000000465072696E742D3535000000B4
:1048100025730A00C4C0D2D7C8CAC80A0000000065
:1048200020CDCEC620C0C2D2CECED2D0C5C7D7C82A
:10483000CAC0000020CAD0DBD8CAC80020C1D3CC6F
:10484000C0C3C80052533233322D310A200A200A25
:104850000000000020D0C0C7CCDBCAC0CDC8C50056
:1048600020C7C0CCDBCAC0CDC8C5000020CDCED08B
:10487000CC0A0A0A0000000020CDC5CDCED0CC0A5B
:104880000A0A000052533233322D320A200A200A1B
:10489000000000005553420A200A200A00000000D0
:1048A00000EEFCFFF77BF3FFF5A130A837F0BDFF6A
:1048B00003AAF6A1FEF7ADFD03A8FEF77FFD02E017
:1048C00003A8FFF7ACFB464621A91320CDF884804E
:1048D00017F0CDF808B164202190F0A122A8219A08
:1048E00037F0D8FC03AA22A9EDA0FEF792FD03A899
:1048F000FEF764FD32F02FFA03A8FFF773FBAFF267
:104900001C10FEF75BFD012031F010FEE7A0FEF762
:1049100055FD082032F064FAA768002028F0AEFEAA
:1049200000B1A768A068C01BA842F6D303AAE1495A
:10493000E1A0FEF76EFD03A8FEF740FDE1A0FEF743
:104940003DFD082032F04CFAA768002028F096FEC2
:1049500070B10EE0CAA130A837F067FF03AAD549AD
:10496000A8E7C7A130A837F060FF03AAD8A1A1E744
:10497000A768A068C01BA842E7D3032031F0D6FD8A
:10498000CC482C30FEF71AFD012031F0CFFD00207D
:1049900028F074FE0028FAD1D0A0FEF70FFD082001
:1049A00032F01EFAD04F06E028F09DFEA068A16804
:1049B000091AB942FBD3002028F060FE00284FF00E
:1049C0000300F1D028F073FE022028F065FE03AA50
:1049D000C6A1B1A0FEF71DFD03A8FEF7EFFCC5A020
:1049E000FEF7ECFC082032F0FBF94FF4FA77C8210F
:1049F00038462AF0E9FFA068A168091AA942FBD34A
:104A0000002028F03BFE0028F1D003AAB7A1A2A005
:104A1000FEF7FFFC03A8FEF7D1FC002028F02EFED5
:104A20000028FAD1012031F081FDB5A0FEF7C6FCC7
:104A3000032031F07BFD32F02EFAB74D2878400785
:104A400002D49C482C3001E09A483430FEF7B6FC82
:104A5000012031F06BFDB1A0FEF7B0FC082032F070
:104A6000BFF9B14F31F095FCA068A168091AB942AD
:104A7000FBD3002028F002FE0028F3D0022031F002
:104A800055FDAAA0FEF79AFC012031F04FFDAAA027
:104A9000FEF794FC082032F0A3F932F0FCF9032071
:104AA00031F044FD2878400702D582482C3001E0DF
:104AB00080483430FEF782FC03A8FEF786FD32F012
:104AC0004AF9ADF8A46029A9392016F0D0FFADF855
:104AD0007C601FA93A2016F0CAFF7649BDF87C20F9
:104AE0004C3122A837F0D6FB03AA22A995A0FEF7E5
:104AF00090FC03A8FEF762FCBDF8A42095A122A8B3
:104B000037F0C8FB03AA22A995A0FEF782FC03A8F0
:104B1000FEF754FC542015F00AFF2FA800F0D0FF38
:104B20002FA800F0C5FB2FA800F0C0FF01268F4D75
:104B30007DE0288840F00200288001200CF0F2FF80
:104B4000012031F0F3FCBDF87C30324688A103A887
:104B500037F0A0FB03A8FEF731FC27A829F0C1FA23
:104B600018B928A829F08CFA28B1AFF2983103A817
:104B700037F018FE13E0BDF89C209DF8A1009DF8C9
:104B8000A010A2F5FA620092CDE901109DF89E30C6
:104B90009DF89F20AFF2B03103A837F07BFB0320D4
:104BA00031F0C4FC03A8FEF709FC012031F0BEFC83
:104BB00032F0D1F803A8FFF715FAAFF2D830FEF7BC
:104BC000FDFB38A903A8FEF76FFD39A903A8FEF77E
:104BD0006EFC3AA903A8FEF7BBFD3BA903A8FEF7AC
:104BE000DEFD3DA903A8FEF7FBFE3EA903A8FEF7E4
:104BF00093FE3FA903A8FEF7BDFE3CA903A8FEF75C
:104C000022FF40A903A8FFF791F9A76803E000205D
:104C100028F034FD80B9A06843F60952C11BBDF8E5
:104C2000A4005043B1EB801FF1D3761CB6B2BDF89F
:104C30007C0086427FF67DAF552015F078FE2FA8C8
:104C400000F03EFF2FA800F033FB2FA800F02EFF4E
:104C5000288840F00200288001200CF063FF49A062
:104C6000FEF7ACFB032031F061FC4FA0FEF7A6FB82
:104C7000288840F00200288001200CF053FFFEE756
:104C80005749464920D7C0D1D2DC0000CDC5D2203B
:104C9000C7C0C3CBD3D8CAC8000000002575000028
:104CA000DFD0CACED1D2DC20D7CB0000CACDCECF48
:104CB000CAC00A0008380000D0C0C7CCDBCAC0CDCB
:104CC000C8C50000C7C0CCDBCAC0CDC8C50A0A0031
:104CD000CDC5D2202B332E3356000000C8CDC4C81A
:104CE000CAC0D2CED0DB0000400D0300CFD0CEC969
:104CF000C4C5CD00C4C8CDC0CCC8CA0A00000000DD
:104D0000C4C5CDC5C6CDDBC920DFD9C8CA0A20C7F6
:104D1000C0CAD0DBD20A0000D2C50720D2C5D1D28A
:104D200020C7C0CCCAC00A0000350C00CFD0CEC905
:104D3000C4C5CD0A0000000020CED2CAD0DBD20A02
:104D400000000000D7C8D1CBCE20D6C8CACBCEC277
:104D5000000000002530347520D1C5CA00000000D5
:104D6000C7C0C4C5D0C6CAC00000000002C007202A
:104D7000D6C8CACB202530347520C8C7202530348A
:104D8000750A00003DD2C5D5CDCECBCEC3C8D7C5A0
:104D9000D1CAC8C920D2C5D1D220C7C0C2C5D0D8B7
:104DA000C5CD3D0A0A0A0A0028CFCEC4CFC8D1DC3F
:104DB000290A0A00F0B5036802790D68002462F33D
:104DC0000704EB18002242EB0401FE4DFE4EDFF813
:104DD000FCC30C0A04D1FE4FE824FF1A8C4108D210
:104DE00089202860012030607846CCF800008920B6
:104DF000F0BD036001712A6078463260CCF8000093
:104E00000020F0BDF0B500230C681A460979057939
:104E100061F30702016865F3070361185A41E94C21
:104E2000E94DEA4E130A04D1E94FE8237F1A934172
:104E300007D28920206001202860784630608920D0
:104E4000F0BD01600271002020602860784630606B
:104E50000020F0BDF0B5036809680022CB18D94CDA
:104E6000D94DDA4E52EB020106D1DFF864C3E827D0
:104E7000BCEB030C8F4107D2892020600120286001
:104E8000784630608920F0BD0360226078462A6051
:104E900030600020F0BDF0B5036809680022CB182F
:104EA000C84CC94DC94E52EB020106D1DFF824C3EC
:104EB0000227BCEB030C8F4107D289202060012020
:104EC0002860784630608920F0BD03602260784613
:104ED0002A6030600020F0BD30B502680968B94B27
:104EE000B94CBA4D8A4207D289201860022020604E
:104EF00078462860892030BD511A01600020186072
:104F0000206078462860002030BDF0B5036809684D
:104F10000022CB18AB4CAC4DAC4E52EB020106D18B
:104F2000DFF8B0C20227BCEB030C8F4107D2892007
:104F3000206001202860784630608920F0BD036041
:104F4000226078462A6030600020F0BD30B50268EB
:104F500009689C4B9C4C9D4D8A4207D28920186061
:104F60000220206078462860892030BD511A0160F7
:104F700000201860206078462860002030BD10B501
:104F800002880988904B11448E4A904CB1F5803FBD
:104F900007D389201060012018607846206089209E
:104FA00010BD01800020106018607846206000204D
:104FB00010BD0021016001718248016082480160DA
:104FC0007846824908600020704700210160818096
:104FD00081717C4801607C48016078467B490860AB
:104FE000002070471CB50023CDE90033036800930F
:104FF0008388ADF8043080798DF8060000201060B9
:10500000DDE900340968CB1A70EB040301D2411EBC
:1050100005E0DDE90043611A834101D201211160FD
:105020006849086068490860784668490860002057
:105030001CBD2DE9FC410022CDE90022026800924E
:105040008288ADF8042082798DF80620DDE90043DE
:105050000A680021141941EB0302CDE90042150E44
:10506000584A594B594C08D1DDE90067DFF868C14F
:105070005A4DBCEB0606BD4108D2892010600120C4
:105080001860784620608920BDE8FC81009D05609D
:10509000BDF8045085809DF80650857111607846F2
:1050A000196020600020EFE72DE9FC410022CDE9E6
:1050B0000022026800928288ADF8042082798DF87F
:1050C0000620DDE900730A6800213E4C3E4D3F4E4C
:1050D000BF1A8B4107D289202060012028607846C2
:1050E00030608920D0E7DDE90073BA1A63EB010371
:1050F000CDE900230260BDF8042082809DF80620DF
:10510000827121607846296030600020BCE72DE97B
:10511000FC410022CDE900220B68097961F3070206
:10512000016800918188ADF8041081798DF806102E
:10513000DDE900145B186241CDE90032140E21490B
:10514000214A224B06D1DDE90056234F234C7D1B1B
:10515000B44107D2892008600120106078461860A9
:10516000892091E7009C0460BDF8044084809DF88C
:1051700006408471002008601060784618600020A6
:1051800082E72DE9F0410546006809680024A1FB8B
:10519000002304FB003001FB04014FF4FA701018E7
:1051A00041F100014FF47A72234636F0D7FF054AE9
:1051B000054B064EA9B9DFF81CC00227BCEB000C5A
:1051C0008F410DE00CC0072010C0072014C007203D
:1051D000FF0FA5D4FFE30B54FFFF63A7B3B6E00DA9
:1051E00008D289201060032018607846306089203A
:1051F000BDE8F0812860146078461C6030600020B3
:10520000F6E72DE9F0410546006809880024A1FB76
:10521000002304FB003001FB040141F28830101828
:1052200041F1000142F21072234636F097FF4E4AD8
:105230004E4B4F4E31B9DFF83CC10227BCEB000C9E
:105240008F4107D2892010600320186078463060B3
:105250008920CDE72860146078461C60306000200B
:10526000C6E7018842F20F72491C89B2018091425F
:1052700001D9012101803C49002008603B490860B8
:1052800078463B49086000207047018842F20F725F
:10529000491E89B20180914200D902803249002022
:1052A000086032490860784631490860002070473C
:1052B0000168314A491C0160914201D90121016014
:1052C0002949002008602949086078462849086073
:1052D000002070470168284A491E0160914200D9A8
:1052E0000260214900200860204908607846204972
:1052F0000860002070472DE9F0410446D1E9000123
:10530000D4E90023A0FB025601FB026100FB03115C
:10531000681949418018594142F21075401941F10C
:105320000001521943F1000392185B4136F016FF59
:105330000D4B0E4D0E4E0A0A04D1104FE8223F1AB3
:105340008A4107D28920186003202860784630609F
:1053500089204DE7C4E900010020186028607846E4
:105360003060002044E700000CC0072010C0072078
:1053700014C00720FFE30B54FFE0F505FF0FA5D491
:105380002DE9FF4717F0B8FE654C000615D402F072
:105390003DF8DFF89081DFF89091644F002668B106
:1053A000012820D087281DD0684601F06DF800063E
:1053B00003D49DF800000E287ED0AEE0684601F0D0
:1053C00063F8000679D403A801F085F8000674D4C8
:1053D0009DF800000E2805D1BDF80C00402801D131
:1053E0007120387089E0684601F04EF8000664D4F8
:1053F0009DF800001D2827D2DFE800F0260F2222AA
:10540000222214141414141414140F12121212124F
:105410000F24242424261212120025F0FDF803E0A4
:10542000202000E06020387002F09EF8000674D45E
:105430009DF800003E4D0E2811D0172812D014E020
:105440005020F0E73020EEE7882009212060C8F8DE
:1054500000107946C9F8001004B0BDE8F0870CF0E0
:105460002DFC05E02878022844D001200CF05AFBDE
:10547000000652D49DF80000172806D1287801288C
:1054800035D125F039F9000647D49DF800000E28E3
:1054900025D12878022826D10AF015FBD8B901A811
:1054A00006F06FFD000638D40DF1060006F04DFD44
:1054B000000632D41F4801E027E02EE000788DF886
:1054C000080017208DF8090001A801F055FF00061B
:1054D00023D4322038709DF800000E2803D0C0B2CB
:1054E000172804D009E02878032803D005E028789D
:1054F000022802D102F02DFA2E7026607946C8F8F3
:1055000000600020C9F80010A6E7FAF783FE25F036
:1055100083F8FAF794FE02F027F820689CE7000071
:105520000CC0072010C0072014C0072070C307203C
:105530005CC1072071C307202DE9F843CD4ECE4F43
:10554000CE4C05464FF08808B0F1004F06D0B5F1BB
:10555000104F03D00220C4F800800AE0684601F032
:1055600029F9000628D49DF8000040B10A20C4F8AB
:1055700000803060784638608820BDE8F8830122DA
:10558000694628462AF038FE000615D49DF800002A
:10559000FF2809D0FF208DF8000001226946284627
:1055A0002AF035FE000607D4280F8DF80000684663
:1055B00001F0F6F8000601D52068DEE7B0490120C9
:1055C0000870002048602060306078463860002015
:1055D000D3E7AB4900200870A8490860A5490860D6
:1055E0007846A549086000207047A5490120087049
:1055F000A249002008609F49086078469E490860DB
:1056000000207047F8B5684601F0D4F89B4D0006BD
:1056100018D49DF80000974E974FA8B198490024E0
:1056200000070C70FF218DF80010012269462AF056
:10563000EEFD000606D48DF80040684601F0B0F893
:10564000000609D52868F8BD882028600A20306047
:10565000784638608820F8BD2C6078463460386021
:105660000020F8BD2DE9F74F92B0144610A801F0C4
:10567000A1F8824D000649D49DF84000DFF8F4817E
:10568000DFF8F4918827B0B1060730462AF0CBFD49
:105690007B4A401E4FF0000A51680B195B1D98426F
:1056A0000ED22F60C8F800A079468820C9F80010F3
:1056B00015B0BDE8F08F0A212F60C8F80010F3E79D
:1056C00046EA01078DF800401298ADF801009346B4
:1056D0006E462246F01C139937F0B3F83019FF21BB
:1056E000C4700171221D711C781C2AF090FD000607
:1056F0000CD40920B0EB177F01D1621D00E001221C
:10570000694638462AF083FD000601D52868CFE7B0
:10571000DBF804102144091DCBF80410C5F800A0E3
:105720007946C8F800A00020C9F80010C0E72DE9AC
:10573000F04F524D4F4F99B0D5F8009016A8D7F8BA
:1057400000A001F037F8000664D49DF85800DFF897
:105750002881040700264FF0010B012201A92046F1
:105760002AF04AFD000655D49DF80400F0B3FF2846
:105770004AD00444241D04F070402AF054FD24F063
:105780007041401E884211D39DF8040040280DD876
:10579000761CE2E7641E012201A920462AF02CFDB6
:1057A000000637D49DF80400402808D988202860D6
:1057B0007946C7F800B0C8F8001019B079E7241A84
:1057C000A41E022215A920462AF016FD000621D4A7
:1057D000A41C9DF8042002A920462AF00DFD000615
:1057E00018D4BDF8540040F0005000E00CE09DF8E3
:1057F000042002A92AF00BFD00060BD49DF804003A
:1058000021180C1AE41E761E002EC3D1FFF7FAFEF3
:10581000000601D52868D0E7C5F800907946C7F89A
:1058200000A04846C8F80010C7E708B5684600F071
:10583000C1FF08B1002008BD9DF800000028FAD083
:105840000007012269462AF0D7FC000605D50B485F
:1058500000680028EFD0012008BD9DF8000008B1C5
:10586000FF28F8D100208DF80000684600F098FF6E
:10587000E0E7000010C0072014C007200CC007207C
:1058800054C107202DE9F0418046F84816461D46D0
:1058900000780F4680B11A4640462AF0ADFCF44C21
:1058A000000606D42A4639464046FFF7DBFE0006CE
:1058B00002D52068BDE8F0812A4631464046BDE861
:1058C000F0412AF0A4BC38B5022269464FF070407E
:1058D0002AF092FCE64C000602D5208885B201E051
:1058E000BDF8005001F05DF9E249E34A854206D176
:1058F00000202060086078461060002038BD8820B5
:1059000020601120086078461060882038BD2DE99D
:10591000FF4FD74CD74ED84F81B0994692468B4611
:1059200000254FF070484A46514601982AF06FFC16
:10593000000611D401F035F9ADF8000002226946E5
:1059400040462AF064FC000606D44A4659460198AF
:105950002AF052FC000603D5206805B0BDE8F08FA0
:105960004A465146584636F0F1FE10B9FFF7ABFFF4
:1059700058B16D1CADB2032DD5D3822020602220FA
:105980003060784638608220E7E700202060306091
:10599000784638600020E0E700B587B00246B74897
:1059A0001C236946FFF7B3FF07B000BDC0EBC00082
:1059B000401F40F0704007222AF01EBC38B5B04CA2
:1059C0000246012369462046FFF75CFF38BDAC4B19
:1059D0000146012218462AF00FBC38B5A84C0246F1
:1059E000641C012369462046FFF74CFF38BDA44BD9
:1059F00001465B1C012218462AF0FEBB38B5A04CBC
:105A00000246A41C012369462046FFF73BFF38BD30
:105A10009B4B01469B1C012218462AF0EDBB38B572
:105A2000974C0246E41C012369462046FFF72AFFF3
:105A300038BD934B0146DB1C012218462AF0DCBB23
:105A400038B58F4C0246241D012369462046FFF7D6
:105A500019FF38BD8A4B01461B1D012218462AF04A
:105A6000CBBB1CB5C0EBC00026300A4640F000504E
:105A700007236946FFF706FF1CBDC0EBC0002630B8
:105A800040F0005007222AF0B7BB38B57C4C0246E4
:105A90004B34012369462046FFF7F4FE38BD784BAE
:105AA00001464B33012218462AF0A6BB38B5744C88
:105AB00002464C34042369462046FFF7E3FE38BD16
:105AC0006F4B01464C33042218462AF095BB38B57B
:105AD0006B4C02465034022369462046FFF7D2FE43
:105AE00038BD674B01465033022218462AF084BB6A
:105AF00038B5634C02465234042369462046FFF70A
:105B0000C1FE38BD5E4B01465233042218462AF0CE
:105B100073BB38B55A4C02465634022369462046B8
:105B2000FFF7B0FE38BD564B0146563302221846E9
:105B30002AF062BB38B5524C0246583402236946FB
:105B40002046FFF79FFE38BD4D4B014658330222D9
:105B500018462AF051BB38B5494C02465A34012345
:105B600069462046FFF78EFE38BD454B01465A3345
:105B7000012218462AF040BB38B5414C02465B343E
:105B8000042369462046FFF77DFE38BD3C4B0146A5
:105B90005B33042218462AF02FBB832208B502EBA0
:105BA00080000A4640F0005004236946FFF76AFE71
:105BB00008BD832202EB800040F0005004222AF04E
:105BC0001BBB38B52E4C0246873404236946204659
:105BD000FFF758FE38BD2A4B01468733042218468A
:105BE0002AF00ABB38B5264C02468B34022369469C
:105BF0002046FFF747FE38BD214B01468B3302227A
:105C000018462AF0F9BA38B51D4C02468D340423E3
:105C100069462046FFF736FE38BD194B01468D33E5
:105C2000042218462AF0E8BA38B5154C02469134D9
:105C3000022369462046FFF725FE38BD104B01467A
:105C40009133022218462AF0D7BA38B50C4C0246D6
:105C50009334012369462046FFF714FE38BD084BF4
:105C600001469333012218462AF0C6BA54C10720D0
:105C70000CC0072010C0072014C00720020000F04D
:105C80002800002038B5FA4C024604236946204615
:105C9000FFF7F8FD38BD38B5F54C0246241D042346
:105CA00069462046FFF7EEFD38BD38B5F04C024698
:105CB0000834042369462046FFF7E4FD38BDEC4B69
:105CC00001460833042218462AF096BA38B5E84C43
:105CD00002460C34012369462046FFF7D3FD38BD48
:105CE000E34B01460C33012218462AF085BA38B539
:105CF000DF4C02460D34042369462046FFF7C2FDFF
:105D000038BDDB4B01460D33042218462AF074BA25
:105D100038B5D74C02461134022369462046FFF7B6
:105D2000B1FD38BDD24B01461133022218462AF08C
:105D300063BA38B5CE4C0246133402236946204676
:105D4000FFF7A0FD38BDCA4B0146133302221846A7
:105D50002AF052BACD2208B502EB80000A4640F084
:105D6000005004236946FFF78DFD08BDCD2202EBEC
:105D7000800040F0005004222AF03EBA40F20D129A
:105D800008B502EB80000A4640F000500423694643
:105D9000FFF778FD08BD40F20D1202EB800040F0E5
:105DA000005004222AF028BA38B5B14C0246953486
:105DB000042369462046FFF765FD38BDAC4B01461C
:105DC0009533042218462AF017BA38B5A84C024673
:105DD0009934042369462046FFF754FD38BDA44B8F
:105DE00001469933042218462AF006BA38B5A04C69
:105DF00002469D34012369462046FFF743FD38BD26
:105E00009B4B01469D33012218462AF0F5B938B55F
:105E1000974C02469E34042369462046FFF732FD24
:105E200038BD934B01469E33042218462AF0E4B94C
:105E300038B58F4C0246A234042369462046FFF74A
:105E400021FD38BD8A4B0146A233042218462AF0B0
:105E5000D3B938B5864C0246A63404236946204699
:105E6000FFF710FD38BD824B0146A63304221846C9
:105E70002AF0C2B938B57E4C0246AA3401236946DD
:105E80002046FFF7FFFC38BD794B0146AA330122BB
:105E900018462AF0B1B938B5754C0246AB34022326
:105EA00069462046FFF7EEFC38BD714B0146AB3327
:105EB000022218462AF0A0B938B56D4C0246AD341E
:105EC000042369462046FFF7DDFC38BD684B0146D8
:105ED000AD33042218462AF08FB938B5644C024617
:105EE000B134012369462046FFF7CCFC38BD604B36
:105EF0000146B133012218462AF07EB938B55C4C10
:105F00000246B234012369462046FFF7BBFC38BD88
:105F1000574B0146B233012218462AF06DB938B505
:105F2000534C0246B334022369462046FFF7AAFCCD
:105F300038BD4F4B0146B333022218462AF05CB9F4
:105F400038B54B4C0246B534042369462046FFF76A
:105F500099FC38BD464B0146B533042218462AF059
:105F60004BB938B5424C0246B93404236946204641
:105F7000FFF788FC38BD3E4B0146B9330422184672
:105F80002AF03AB938B53A4C0246BD340423694682
:105F90002046FFF777FC38BD354B0146BD33042260
:105FA00018462AF029B938B5314C0246C1340423C9
:105FB00069462046FFF766FC38BD2D4B0146C133CC
:105FC000042218462AF018B938B5294C0246C534BF
:105FD000012369462046FFF755FC38BD244B014696
:105FE000C533012218462AF007B91CB500EB800022
:105FF00000F27D100A4640F0005005236946FFF785
:1060000041FC1CBD00EB800000F27D1040F0005010
:1060100005222AF0F1B84FF4CA7208B502EB40002D
:106020000A4640F0005002236946FFF72BFC08BDEA
:106030004FF4CA7202EB400040F0005002222AF0F6
:10604000DBB84FF4CE7208B502EB40000A4640F0D0
:10605000005002236946FFF715FC08BD4FF4CE72CD
:1060600002EB400040F0005002222AF0C5B80000C8
:10607000BC0000201CB500EB800001EB810100EBAF
:10608000810000F28D1040F0005005236946FFF7B3
:10609000F9FB1CBD00EB800001EB810100EB8100EE
:1060A000134600F28D1040F00050052219462AF0E8
:1060B000A3B8090108B501EB800000F2D22040F03E
:1060C000005004236946FFF7DDFB08BD090101EB21
:1060D0008000134600F2D22040F0005004221946FE
:1060E0002AF08AB81CB500EB800001EB810100EBBF
:1060F000810000F2CD3040F0005005236946FFF7E3
:10610000C1FB1CBD00EB800001EB810100EB8100B5
:10611000134600F2CD3040F00050052219462AF017
:106120006BB838B5F84C0246042369462046FFF7A1
:10613000A9FB38BDF44B0146042218462AF05CB88E
:106140001CB500EB800000F225500A4640F00050DC
:1061500005236946FFF796FB1CBD00EB800000F2AB
:10616000255040F0005005222AF046B838B5E64CDC
:1061700002461834042369462046FFF783FB38BDE6
:10618000E14B01461833042218462AF035B81CB5F5
:1061900000EB800000F23D500A4640F0005005231D
:1061A0006946FFF76FFB1CBD00EB800000F23D501D
:1061B00040F0005005222AF01FB81CB500EB80000B
:1061C00000F251500A4640F0005005236946FFF79F
:1061D00059FB1CBD00EB800000F2515040F0005014
:1061E00005222AF009B81CB500EB800000F26550CA
:1061F0000A4640F0005005236946FFF743FB1CBDEB
:1062000000EB800000F2655040F00050052229F0BC
:10621000F3BF1CB500EB800001EB810100EB8100B6
:1062200000F2655040F0005005236946FFF72AFB55
:106230001CBD00EB800001EB810100EB81001346E7
:1062400000F2655040F000500522194629F0D4BFF5
:106250001CB500EB800001EB810100EB810000F236
:106260002D6040F0005005236946FFF70BFB1CBD75
:1062700000EB800001EB810100EB8100134600F28E
:106280002D6040F000500522194629F0B5BF1CB51D
:1062900000EB800001EB810100EB810000F60D00B6
:1062A00040F0005005236946FFF7ECFA1CBD00EBF7
:1062B000800001EB810100EB8100134600F60D0028
:1062C00040F000500522194629F096BF1CB500EB9E
:1062D000800000F679200A4640F000500523694608
:1062E000FFF7D0FA1CBD00EB800000F6792040F0EB
:1062F0000050052229F080BF40F6862208B502EB47
:1063000040000A4640F0005002236946FFF7BAFAFF
:1063100008BD40F6862202EB400040F00050022209
:1063200029F06ABF1CB500EB800001EB810100EB96
:10633000410000F67D2040F0005005236946FFF73C
:10634000A1FA1CBD00EB800001EB810100EB4100D4
:10635000134600F67D2040F000500522194629F032
:106360004BBF40F6EE2208B502EB40000A4640F073
:10637000005002236946FFF785FA08BD40F6EE2279
:1063800002EB400040F00050022229F035BF40F6F9
:10639000F62208B502EB40000A4640F00050022306
:1063A0006946FFF76FFA08BD40F6F62202EB40009F
:1063B00040F00050022229F01FBF38B5534C02466E
:1063C000022369462046FFF75DFA38BD4F4B014670
:1063D0000222184629F010BF38B54C4C0246A41CC6
:1063E000022369462046FFF74DFA38BD474B014668
:1063F0009B1C0222184629F0FFBE38B5434C0246CA
:10640000241D012369462046FFF73CFA38BD38B504
:106410003E4C0246641D022369462046FFF732FACD
:1064200038BD3A4B01465B1D0222184629F0E4BEF6
:1064300038B5364C0246E41D022369462046FFF774
:1064400021FA38BD314B0146DB1D0222184629F0E6
:10645000D3BE38B52D4C0246093401236946204687
:10646000FFF710FA38BD294B0146093301221846BF
:1064700029F0C2BE38B5254C02460A3401236946CC
:106480002046FFF7FFF938BD204B01460A330122B1
:10649000184629F0B1BE40F6093208B502EB4000BB
:1064A0000A4640F0005002236946FFF7EBF908BDA9
:1064B00040F6093202EB400040F00050022229F081
:1064C0009BBE38B5114C0246413402236946204632
:1064D000FFF7D8F938BD0D4B01464133022218466B
:1064E00029F08ABE38B5094C024643340223694676
:1064F0002046FFF7C7F938BD044B0146433302225B
:10650000184629F079BE000026050020000B002067
:1065100038B5FC4C0246042369462046FFF7B2F921
:1065200038BDF84B01460422184629F065BE38B53F
:10653000F44C0246241D042369462046FFF7A2F9C5
:1065400038BDF04B01461B1D0422184629F054BEED
:1065500038B5EC4C02460834042369462046FFF760
:1065600091F938BDE74B014608330422184629F05B
:1065700043BE1CB500EB800000F64C300A4640F0EC
:10658000005005236946FFF77DF91CBD00EB800034
:1065900000F64C3040F00050052229F02DBE38B5F1
:1065A000D84C02462034042369462046FFF76AF996
:1065B00038BDD44B014620330422184629F01CBEB6
:1065C00038B5D04C02462434012369462046FFF7F3
:1065D00059F938BDCB4B014624330122184629F026
:1065E0000BBE40F6663208B502EB80000A4640F06A
:1065F000005004236946FFF745F908BD40F66632AE
:1066000002EB800040F00050042229F0F5BD1CB5DB
:1066100000EB800001EB810100EB810000F66530AA
:1066200040F0005005236946FFF72CF91CBD00EB34
:10663000800001EB810100EB8100134600F665301C
:1066400040F000500522194629F0D6BD1CB500EBDC
:10665000800001EB810100EB810000F6C93040F0C1
:10666000005005236946FFF70DF91CBD00EB8000C3
:1066700001EB810100EB8100134600F6C93040F0C8
:1066800000500522194629F0B7BD40F61E5208B544
:1066900002EB80000A4640F0005004236946FFF7F1
:1066A000F1F808BD40F61E5202EB800040F00050A9
:1066B000042229F0A1BD38B5934C02460123694656
:1066C0002046FFF7DFF838BD8F4B01460122184600
:1066D00029F092BD38B58C4C0246641C04236946EF
:1066E0002046FFF7CFF838BD874B01465B1C0422DC
:1066F000184629F081BD38B5834C0246641D042339
:1067000069462046FFF7BEF838BD7F4B01465B1D4A
:106710000422184629F070BD38B57B4C0246093476
:10672000042369462046FFF7ADF838BD764B014695
:1067300009330422184629F05FBD38B5724C024671
:106740000D34042369462046FFF79CF838BD6E4B94
:1067500001460D330422184629F04EBD38B56A4C67
:1067600002461134022369462046FFF78BF838BDF4
:10677000654B014611330222184629F03DBD38B55C
:10678000614C02461334022369462046FFF77AF82B
:1067900038BD5D4B014613330222184629F02CBD4B
:1067A00038B5594C02461534012369462046FFF797
:1067B00069F838BD544B014615330122184629F0BB
:1067C0001BBD38B5504C024616340123694620469D
:1067D000FFF758F838BD4C4B0146163301221846D6
:1067E00029F00ABDC90008B501EB400000F557606B
:1067F00040F0005002236946FFF744F808BDC90085
:1068000001EB4000134600F5576040F000500222B3
:10681000194629F0F1BC40F6F85208B502EB4000E9
:106820000A4640F0005002236946FFF72BF808BDE6
:1068300040F6F85202EB400040F00050022229F0EE
:10684000DBBC40F62E6208B502EB40000A4640F081
:10685000005002236946FFF715F808BD40F62E6286
:1068600002EB400040F00050022229F0C5BC1CB5EC
:1068700000EB800001EB810100EB810000F64D6030
:1068800040F0005005236946FEF7FCFF1CBD00EBFD
:10689000800001EB810100EB8100134600F64D60A2
:1068A00040F000500522194629F0A6BC1CB500EBAB
:1068B000800001EB810100EB810000F69D6040F05B
:1068C000005005236946FEF7DDFF1CBD00EB80008C
:1068D00001EB810100EB8100134600F69D6040F062
:1068E00000500522194629F087BC40F6047208B50D
:1068F00002EB40000A4640F0005002236946FEF7D2
:10690000C1FF08BD450B0020620D002040F6047257
:1069100002EB400040F00050022229F06DBC40F62E
:10692000067208B502EB80000A4640F000500423CE
:106930006946FEF7A7FFE4E740F6067202EB800027
:1069400040F00050042229F057BC4FF4716208B5A2
:1069500002EB40000A4640F0005002236946FEF771
:1069600091FFCEE74FF4716202EB400040F000501F
:10697000022229F041BC2DE9F84304226946002097
:1069800029F07BFD954C00060FD49549009882278D
:10699000944D954E4FF0190888420DD10422694656
:1069A000104629F06AFD000602D52068BDE8F8838C
:1069B0008E490098884206D027607846C5F8008046
:1069C00030608220F2E70020206028607846306046
:1069D0000020EBE72DE9F043804EDFF80882DFF876
:1069E000089291B000254FF40057002461196846C1
:1069F00000F0EBF820226946204629F053FE0006FD
:106A00000ED42034BC42F1D300246119684600F052
:106A1000DCF8202208A9204629F02FFD000603D526
:106A2000306811B0BDE8F083202208A9684635F02F
:106A30008DFE40B1822019213060C8F800107946DF
:106A4000C9F80010EDE72034BC42DED3ED1DFF2D68
:106A5000CBD9002030607946C8F80000C9F8001092
:106A6000DFE770B58CB000208DF824005C480A90F8
:106A700024226946042029F000FD584D000617D451
:106A8000FFF7A8FF000613D400244FF4005601229C
:106A900009A9204629F006FE000609D4641CB44268
:106AA000F5D324226946042029F0FCFD000602D516
:106AB00028680CB070BD04220AA9002029F0F2FD5C
:106AC000F7E738B504466946002009F022FC0106C4
:106AD000424801D5006838BDBDF8001001B1012160
:106AE0002170002101603F48016078463E490860FE
:106AF000002038BDFF2009F046BD10B588B06846BB
:106B0000C11D06F027F8354C00060BD40DF10E0020
:106B1000FEF75BFA000605D40DF11500FEF755FAF5
:106B2000000602D5206808B010BD6846FEF734FFA5
:106B3000F9E738B5FEF7C7FE284C48B36846FFF7BB
:106B4000C0FF00061FD49DF80000F0B1702013F0C4
:106B5000EEFE000617D4712013F0E9FE000612D4F1
:106B60006F2013F0E4FE00060DD4FFF7C6FF000609
:106B700009D4722013F0DBFE000604D46F2013F05A
:106B8000D6FE000604D5206838BDFFF7B6FFF8E74B
:106B900014490020206008607846134908600020EE
:106BA00038BD00B589B01E226946D00629F024FB05
:106BB000000604D50948008880B209B000BD1C2138
:106BC0000DF10200F9F756FBF7E7002200F8011B70
:106BD000491C521C202AF9D3704700000CC0072022
:106BE000CC2C514010C0072014C00720CEFAADDED7
:106BF00038B504466846FEF70BFF01060A4801D582
:106C0000006838BD9DF80010032909D08721016074
:106C1000064900200860784605490860872038BD8D
:106C2000204601F007FF38BD0CC0072010C0072028
:106C300014C0072038B504466846FEF7E9FE010691
:106C40000A4801D5006838BD9DF80010032909D015
:106C500087210160064900200860784605490860E0
:106C6000872038BD204601F0DBFF38BD0CC007206F
:106C700010C0072014C0072038B504466846FEF748
:106C8000C7FE01060A4801D5006838BD9DF800100E
:106C9000032909D087210160064900200860784651
:106CA00005490860872038BD204602F06DF838BDE0
:106CB0000CC0072010C0072014C0072038B50446B8
:106CC0006846FEF7A5FE01060A4801D5006838BDF2
:106CD0009DF80010032909D0872101600649002092
:106CE0000860784605490860872038BD204602F0D4
:106CF00029F938BD0CC0072010C0072014C0072098
:106D000038B504466846FEF783FE01060A4801D5F9
:106D1000006838BD9DF80010032909D08721016063
:106D2000064900200860784605490860872038BD7C
:106D3000204602F0BBF938BD0CC0072010C0072068
:106D400014C0072038B504466846FEF761FE010608
:106D50000A4801D5006838BD9DF80010032909D004
:106D600087210160064900200860784605490860CF
:106D7000872038BD204602F075FA38BD0CC00720C8
:106D800010C0072014C0072038B504466846FEF737
:106D90003FFE01060A4801D5006838BD9DF8001085
:106DA000032909D087210160064900200860784640
:106DB00005490860872038BD204602F0E7FA38BD53
:106DC0000CC0072010C0072014C0072038B50446A7
:106DD0006846FEF71DFE01060A4801D5006838BD69
:106DE0009DF80010032909D0872101600649002081
:106DF0000860784605490860872038BD204602F0C3
:106E00007DFB38BD0CC0072010C0072014C0072030
:106E100038B504466846FEF7FBFD01060A4801D571
:106E2000006838BD9DF80010032909D08721016052
:106E3000064900200860784605490860872038BD6B
:106E4000204602F0EFFB38BD0CC0072010C0072021
:106E500014C0072038B56846FEF7DAFD0E4C000670
:106E600011D49DF80000032809D087200B49206029
:106E70000020086078460A490860872038BD02F083
:106E800089FC000601D5206838BD04208DF800007B
:106E90006846FEF7B3FD38BD0CC0072010C00720C0
:106EA00014C007202DE9FE43294C002620688228C3
:106EB00000D001266846FEF7ABFD00063AD49DF8E7
:106EC00000001D280DD101A800F04AF8000631D4B9
:106ED0002048018821F00201018000F0A5FE000693
:106EE00028D49DF8000000251B4FDFF87080032890
:106EF0000DD004280BD00E2809D01B2807D08720DE
:106F0000206079463D60C8F80010BDE8FE8300208F
:106F100002F082FC00060DD49DF800001B280BD067
:106F20006846FEF786FD000604D46846FEF766FD57
:106F3000000601D52068E8E716B101200AF0F2FD4D
:106F4000256079463D600020C8F80010DDE70000AC
:106F50000CC0072002C0072010C0072014C0072063
:106F60002DE9F04796B0824614A8FEF751FD504C2B
:106F7000000654D49DF85010002505264D4FDFF82B
:106F800038810DF1400904290AD01D2948D08720F5
:106F9000206079463D60C8F8001016B0BDE8F08763
:106FA00015A9504602F07BFD20B192282AD09328E3
:106FB00075D123E09DF85400002873D03F48007835
:106FC00000286FD01D208DF8500014A8FEF716FD84
:106FD000000664D44846FEF7DFFF00065FD413A81E
:106FE000FEF7EBFF00065AD40AF085FA60B325607D
:106FF00079463D600020C8F80010CEE7F9F70AF99D
:107000000E2005E03868312849D1F9F703F9162038
:107010008DF8500014A8FEF7F1FCF9F710F93EE0E6
:107020000EA807F0E6FB000639D413A9109807F064
:107030003FFE000633D44846FEF7A4FF00062ED4D8
:1070400013A8FEF7B0FFCDE70C208DF801001098D3
:10705000CDF802001398CDF80600684608F076FDDA
:1070600000061CD4684609F0D7FE000617D4FEF7C8
:10707000DCFB18B1FEF7ADFA000610D4684608F044
:1070800090FD00060BD4684609F0F1FE000606D418
:10709000FEF7CBFB28B1FEF7A8FA000602D5206860
:1070A0007BE7FFE78DF8506014A8FEF7A7FC74E7B4
:1070B0000CC0072010C0072014C007201C040000CB
:1070C00070B586B005460E4603A8FEF7A1FC2D4C10
:1070D00000064ED49DF80C001D280DD104A8FFF722
:1070E0003FFF000645D42848018821F002010180B5
:1070F00000F09AFD00063CD49DF80C1001292DD01B
:107100000020022909D087212160204908607846A3
:107110001F490860872006B070BD2988ADF80410AB
:107120006988ADF8061029798DF808108DF80900E6
:1071300001A803F09DFE00061BD469462B2014F025
:10714000CBFB000615D413489DF800100078C90742
:1071500004D0012802D001208DF80C0003A8FEF70E
:107160005EFC000605D43146284603F019F90006F6
:1071700001D52068CFE706208DF80C0003A8FEF7A4
:107180003DFCC8E70CC0072002C0072010C0072044
:1071900014C00720CAC3072038B56846FEF738FC7C
:1071A0000F4C000616D49DF80000062809D0872051
:1071B0000C4920600020086078460B490860872051
:1071C00038BD03F06FF9000604D46846FEF731FCC1
:1071D000000601D5206838BD6846FEF70FFC38BDB3
:1071E0000CC0072010C0072014C0072038B5054682
:1071F0006846FEF70DFC0F4C000612D49DF8000007
:10720000062809D087200C492060002008607846B5
:107210000A490860872038BD284603F07BF900063C
:1072200001D5206838BD07208DF800006846FEF7BC
:10723000E5FB38BD0CC0072010C0072014C0072094
:1072400038B504466846FEF7E3FB01060B4801D556
:10725000006838BD9DF8001004290BD0062909D01C
:1072600087210160064900200860784605490860CA
:10727000872038BD204603F08FFA38BD0CC00720A8
:1072800010C0072014C0072038B504466846FEF732
:10729000BFFB01060B4801D5006838BD9DF8001002
:1072A00004290BD0062909D0872101600649002056
:1072B0000860784605490860872038BD204603F0FD
:1072C0002DFB38BD0CC0072010C0072014C00720BC
:1072D00038B504466846FEF79BFB01060B4801D50E
:1072E000006838BD9DF8001004290BD0062909D08C
:1072F000872101600649002008607846054908603A
:10730000872038BD204603F0BBFB38BD0CC00720EA
:1073100010C0072014C0072038B505466846FEF7A0
:1073200077FB124C000617D49DF80000022809D004
:1073300087200F4920600020086078460D490860CA
:10734000872038BD002004F053FE000604D42846F0
:1073500003F08EFD000601D5206838BD01208DF8B0
:1073600000006846FEF74AFB38BD00000CC007204D
:1073700010C0072014C0072038B505466846FEF740
:1073800047FB1F4C000632D49DF8000010281FD088
:107390000CDC0C281CD004DC012819D002280DD1EB
:1073A00016E00D2814D00E2808D111E013280FD0B4
:1073B00014280DD015280BD0182809D08720114982
:1073C00020600020086078460F490860872038BD9B
:1073D0006846FEF724FB000609D46846FEF730FB3A
:1073E000000604D4284605F015FC000601D52068E7
:1073F00038BD08208DF800006846FEF7FFFA38BD5A
:107400000CC0072010C0072014C007202DE9F04150
:1074100086B002A8FEF7FCFA504C00067ED49DF818
:10742000080001274E4E0025082807D0092805D05E
:107430000A2874D0872006B0BDE8F08105F094FCDE
:10744000009031684FF00A080191042821D005DC32
:1074500048B1012809D0032829D118E0052802D015
:10746000822824D11FE0009560E06846FFF750F8BD
:10747000000670D401A8FFF75AF800066BD48DF807
:10748000088002A8FEF7BAFA000664D44EE008208D
:1074900000E009208DF8080002A8FEF7AFFA00907E
:1074A0003068019042E003290DD004290BD009F087
:1074B0003CFF03A8FEF7E8FF00064CD49DF80C0043
:1074C0000E2803D011E006F0F9FF2FE004A9622096
:1074D00014F002FA00063ED49DF81000C00704D054
:1074E0000120F9F7CBFC000635D40098822801D0A2
:1074F000922801D106F0E2FF6846FFF709F800067E
:1075000029D401A8FFF713F8000624D49DF8080039
:1075100009280BD08DF8088002A801E01BE00DE0DF
:10752000FEF76CFA15E000BFCDE900750098206009
:107530000199316079460B4A11607CE78120CDE9E1
:1075400000056846FEF7E4FF000604D401A8FEF734
:10755000EEFF0006E8D520686DE700000CC00720AC
:1075600010C0072014C007202DE9F04186B003A801
:10757000FEF78AFF364C000660D402A8FEF748FAF0
:1075800000065BD401A8FEF7CCFF000656D404A881
:10759000FEF7D7FF000651D49DF8080087272D4D30
:1075A0002D4E4FF000080A2801D0092835D106F0E9
:1075B00079FB000642D401980128684608D0FEF7FE
:1075C00038FA00063AD49DF80800092805D013E0DF
:1075D000FEF740FA000631D414E00198922801D059
:1075E000822802D113208DF800009DF80C00142889
:1075F00002D10C208DF800000198932802D10E20B2
:107600008DF800006846FEF7F9F9000616D49DF8DB
:107610000800092814D00A2808D027607846C5F841
:1076200000803060872006B0BDE8F0819DF80C0036
:107630000E2805D1FAF7ADFE000601D52068F2E765
:10764000019820600499296079463160EBE70000D9
:107650000CC0072010C0072014C0072038B505460D
:107660006846FEF7D5F9164C00061FD49DF80000B9
:107670000C2809D087201349206000200860784634
:1076800011490860872038BD6846FEF7C8F9000632
:107690000CD40D208DF800006846FEF7D1F90006E5
:1076A00004D4284603F0AAFC000601D5206838BDA2
:1076B00008208DF800006846FEF7A0F938BD0000EC
:1076C0000CC0072010C0072014C00720F0B585B0FB
:1076D00001A808F056FE344C000655D46846FEF763
:1076E00097F9000650D49DF8000002252F4E304F28
:1076F00013281ED00CDC0D281BD004DC012818D068
:1077000002280DD115E00E2813D0102808D143E02F
:1077100014280ED015280CD018280AD01B283BD0CE
:10772000872020600020306078463860872005B0D0
:10773000F0BD012004F05CFC000625D404A804F090
:10774000F7F8000622D59DF81000E8B1012809D00D
:10775000022810D0882020600920306078463860E8
:107760008820E4E7F8F756FD18208DF8000006E0C1
:10777000F8F765FD08E0F8F74DFD8DF80050684614
:10778000FEF73CF90006F3D52068D0E78DF80050ED
:107790006846FEF733F9CAE79220206078463560E4
:1077A00038609220C3E700000CC0072010C00720FB
:1077B00014C007202DE9F04385B0814602A808F0E7
:1077C000E0FD2C4C000645D40620F9F72CFF2A4D8D
:1077D0002A4E38B90420F9F726FF18B90120F9F725
:1077E00022FF80B16846FEF713F9000632D49DF8F7
:1077F000000000274FF0870802280ED00D2817D070
:10780000182829D114E091202060B1202860784602
:107810003060912005B0BDE8F08301A8FFF751F971
:10782000000617D416499DF804000978084213D1C0
:1078300001A9484603F01AFEA8B19DF8040048B11A
:10784000F8F7E8FC18208DF800006846FEF7D6F837
:10785000F8F7F5FC2068DDE7C4F8008078462F6073
:1078600030608720D6E702208DF800006846FEF7DA
:10787000C5F8CFE70CC0072010C0072014C00720B0
:107880001C040000F8B506466846FEF7C1F8504CE7
:10789000000650D49DF800004E4D132812D004DC91
:1078A00001280FD00E2804D10CE015280AD01B287F
:1078B00008D087202060002028607846464908606C
:1078C0008720F8BDFAF783F993281ED06846FEF7A3
:1078D000A6F800062FD49DF800001B2819D002201E
:1078E0008DF800006846FEF7ABF8000623D40120AF
:1078F00004F07EFB00061ED4304606F031FA50B18B
:107900008F280FD0922816D117E0F8F783FC0E20AD
:1079100019E01020E4E708208DF800006846FEF723
:107920006DF8F8BDF8F776FC2868072801D1142017
:1079300009E0F8F784FC2068F8BDF8F76BFC2868CC
:107940003128F6D116208DF800006846FEF756F86B
:10795000EFE72DE9FC4101A8F9F709FA1C4C0006F4
:107960000BD4BDF804001B4E1B4F002540B16946E7
:10797000622013F0B1FF000609D52068BDE8FC8144
:10798000812020607846356038608120F6E79DF8D8
:107990000000800703D5002110A02FF036F8F9F77A
:1079A000EBF930B1F8F736FC09F0BFFCF8F747FC0B
:1079B000E3E70F48018841F00201018001200AF04D
:1079C000B1F825607846356038600020D6E70000C1
:1079D0000CC0072010C0072014C007208493818B9F
:1079E000888A809220848E8A938C858D92800A006A
:1079F00002C00720F8B506460D466846FEF708F8AF
:107A00001C4C00062DD49DF80020132A19D008DC48
:107A1000012A16D0022A14D00E2A12D0102A06D11A
:107A20000FE0142A0DD0152A0BD0182A09D0872070
:107A300011492060002008607846104908608720BE
:107A4000F8BD6846FDF7EBFF00060AD46846FDF76F
:107A5000F7FF000605D42946304606F04BFB00062A
:107A600001D52068F8BD08208DF800006846FDF7B4
:107A7000C5FFF8BD0CC0072010C0072014C00720A8
:107A8000F8B506460D466846FDF7C2FF1D4C0006D8
:107A900027D49DF800101C4A1C48102911D004DC82
:107AA00002290ED00D2904D10BE0112922D014296E
:107AB00007D087212160002111607946016087206D
:107AC000F8BD6846FDF7ABFF00060AD46846FDF72F
:107AD000B7FF000605D42946304606F0C7FB00066E
:107AE00001D52068F8BD08208DF800006846FDF734
:107AF00085FFF8BD91212160A921116079460160BF
:107B00009120F8BD0CC0072010C0072014C007202A
:107B10003EB501A8FDF76BFF214C00063ED4684638
:107B2000FDF776FF000639D402A9012025F082FD79
:107B3000000633D49DF800001A4D022806D00E2806
:107B400004D0102802D00298C00705D004F082F8B3
:107B500080B1922822D114E09DF804208721124898
:107B600021600AB1042100E000212960794601600A
:107B700087203EBD10208DF800006846FDF73EFFCF
:107B80003EBD2868312809D1F8F744FB16208DF84E
:107B900000006846FDF732FFF8F751FB20683EBD54
:107BA0000CC0072010C0072014C0072038B50546B8
:107BB0006846FDF72DFF184C00061DD49DF8000007
:107BC000112809D0872015492060002008607846D8
:107BD00013490860872038BD124829680160696828
:107BE0004160A9688160342012F0A1FE000603D430
:107BF0002FF0B1F8000601D5206838BD284608F0FE
:107C0000EFFE10B109F091FBF6E702208DF80000BD
:107C10006846FDF7F3FE38BD0CC0072010C00720F2
:107C200014C0072094C807202DE9FC416846FDF7E1
:107C3000EFFE194C000622D49DF800000025174ED7
:107C4000174F052809D01D2820D0872020607846AE
:107C5000356038608720BDE8FC8101A90120FDF76F
:107C6000A8FF00060BD404F0B7F8000607D40120E3
:107C70008DF800006846FDF7C1FE000601D52068BA
:107C8000E9E7019800B1012009F010FC2560784671
:107C9000356038600020DEE70CC0072010C00720E8
:107CA00014C0072038B56846FDF7B2FE0E4C00063A
:107CB00011D49DF80000072809D087200B492060C7
:107CC0000020086078460A490860872038BD04F023
:107CD000ABF8000601D5206838BD01208DF8000002
:107CE0006846FDF78BFE38BD0CC0072010C007208A
:107CF00014C0072038B504466846FDF789FE010622
:107D00000A4801D5006838BD9DF80010032909D044
:107D1000872101600649002008607846054908600F
:107D2000872038BD204604F005FA38BD0CC0072076
:107D300010C0072014C0072038B504466846FDF778
:107D400067FE01060A4801D5006838BD9DF800109D
:107D5000032909D087210160064900200860784680
:107D600005490860872038BD204604F05BFA38BD1D
:107D70000CC0072010C0072014C0072038B50446E7
:107D80006846FDF745FE01060A4801D5006838BD82
:107D90009DF80010032909D08721016006490020C1
:107DA0000860784605490860872038BD204604F001
:107DB000B1FA38BD0CC0072010C0072014C007203E
:107DC00038B504466846FDF723FE0106204801D574
:107DD000006838BD9DF8001001290BD0022909D098
:107DE000872101601B490020086078461A49086015
:107DF000872038BD204604F00BFC38BD38B504465A
:107E00006846FDF705FE0106114801D5006838BD3A
:107E10009DF8001001290FD0032910D004290ED09D
:107E200005290CD0872101600A49002008607846A6
:107E300009490860872038BD0121204605E009F086
:107E4000CEFA2EF088FF0021084604F05BFC38BD16
:107E50000CC0072010C0072014C007202DE9F843EC
:107E600080466946012025F0E5FB104C00060DD444
:107E700000980F4E0F4FC0074FF0000509D00022A9
:107E80000121404604F0CAFC000609D52068BDE87F
:107E9000F883872020607846356038608720F6E7D1
:107EA00025607846356038600020F0E70CC0072078
:107EB00010C0072014C0072038B504464FF000401A
:107EC000FDF73AFB000602D51648006838BD20468B
:107ED000FDF71FFE00061FD4A01CFDF72BFE0006B9
:107EE0001AD4201DFDF737FE000615D409F0D6FE82
:107EF000000602D509F019FA0EE06846FDF7E0FD2C
:107F0000000609D46846FDF7D3F9000604D4684694
:107F1000FDF7CCFD000602D5FDF709FC38BDFDF7E5
:107F200071FB38BD0CC007202DE9F04188B001A8D5
:107F3000FDF75DFD384C00065ED49DF80400374F18
:107F4000374E48B1912020609C20306078463860E0
:107F5000912008B0BDE8F08106A9012025F06AFB58
:107F6000000649D406984FF00005C00746D0684681
:107F7000FDF74EFD00063FD46846FDF750FD0006B4
:107F80003AD46846FDF75CFD000635D408208DF82C
:107F900000006846FDF732FD00062DD44FF00108C1
:107FA0008DF8088002A8FEF765FA000624D40320A5
:107FB0008DF80C0003A8FDF768FD00061CD41949D4
:107FC0000220087014482560FEF7A2FA000613D4B8
:107FD00013483560FEF7ABFA00060DD4ADF81080FB
:107FE00004A8FEF76EFA000606D4ADF8145005A8F2
:107FF000FEF778FA000608D52068AAE787202060F7
:108000007846356038608720A3E72560784635607C
:10801000386000209DE700000CC0072014C0072036
:1080200010C0072000C007202DE9FF47064668461C
:1080300003F0A7FFA14C000663D4BDF800004FF485
:10804000B46148433178C1EB011100EB81007178D4
:10805000451802A8FEF735FD000652D498499DF850
:108060000800DFF860920978DFF85CA208424FF060
:1080700086074FF0170817D06946022006F052FC19
:1080800000063ED401A9032006F04CFC000638D4BB
:10809000BDF80000BDF80410C0EB001000EB40007C
:1080A00001EB401085421DD303A8FAF77BFA0006C6
:1080B00027D49DF80C00F8B16846FEF787F9000652
:1080C0001FD401A8FEF792F900061AD4BDF80000EB
:1080D000BDF80410C0EB001000EB400001EB4010B5
:1080E000854209D227607946C9F800808620CAF8FF
:1080F000001004B0BDE8F087304626F026F80006F0
:1081000001D52068F5E703F0EBFFF2E72DE9FF4723
:1081100081466946532013F0DFFB684C000629D4E2
:108120009DF8000000F004008DF8000001A8FDF7A4
:108130006FFC00061ED49DF80400624D624E0027BD
:10814000DFF88881102817D009DC022814D00D2808
:1081500019D091210E287DD00F2806D19AE0112840
:108160000AD0192815D01A2813D003A8FAF71AFA3A
:10817000000670D52068BCE74846FFF755FF05E0CC
:1081800088F800700FE0484625F0DFFF0006F1D4C4
:10819000F6E74846FFF748FF0028EBD198F80000C3
:1081A000C246022805D0276078462F603060002044
:1081B0009FE79DF8000020B14D2012F0B8FB0006AB
:1081C000D8D4484625F05CFF0006D3D4404999F83E
:1081D000028088683F4A8B681B1A9342FBD348464B
:1081E00025F04EFF0006C5D499F80210414507D18D
:1081F000822020600520286078463060822078E761
:1082000003218AF8001034494FF0010801A881F8D1
:108210000080FDF71FFC0006ACD401A8FDF7EEFBC3
:108220000006A7D40420F9F78FFA0006A2D49DF81F
:10823000000020B1012009F075FC00069AD402A9C3
:10824000532013F049FB000694D49DF8080010F069
:10825000010001E01BE024E08DF8080008D00120B7
:1082600009F060FC000685D408F0B6FF000681D452
:108270009DF8080020B1012009F054FC000686D4C6
:10828000C4F8008078462F603060012031E7A020DC
:10829000216001E0D2202160286078463060912082
:1082A00027E79DF80C108720206011B1042028607A
:1082B00000E02F607846306087201AE70CC0072066
:1082C0001C04000010C0072014C007205EC1072056
:1082D00000000940E0C8100062C107202DE9FE43FC
:1082E000054601A8FEF7EDFBAB4C00062BD49DF82C
:1082F0000400AA4EAA4F4FF086084FF01A09A8B101
:10830000A848007848B16946022006F00BFB000639
:1083100019D4BDF8000085421CD36846F9F76AFB02
:10832000000610D4BDF80000854213D302A8FAF766
:1083300039F9000607D49DF8080098B16846FEF7A1
:1083400045F8000602D52068BDE8FE83BDF80000B0
:10835000854207D2C4F800807846C6F8009038609D
:108360008620F1E7002020603060784638600020E9
:10837000EAE72DE9F14F88B000278DF8047003A9D2
:108380000898F8F789FBBDF80C0048F26901834DA5
:10839000834E814C401E4FF086094FF0140A8842EC
:1083A00005D300BFC4F80090C5F800A05EE001A9A5
:1083B000532013F091FA00067ED49DF8040000F0DB
:1083C00004008DF804006846FDF722FB0006F3D494
:1083D0009DF80000102820D009DC02281DD00D28AF
:1083E0001BD091210E2868D00F2808D198E01128C1
:1083F00013D0192811D01A280FD01C280DD006A888
:10840000FAF7D0F8000657D49DF8181087200029F5
:1084100020607CD0042028608AE0BDF80C00FFF7C3
:108420005DFFDFF8848138B3862845D188F8007075
:108430009DF800001C2810D01A283DD019283BD0E8
:108440006846FDF7ECFA000636D41C208DF80000D3
:108450006846FDF7D3FA00062ED40220F9F761F939
:10846000000629D41A20C4F80090286078463060AD
:10847000862009B0BDE8F08F02A825F032FE000684
:108480004FF0010B07D54FF4FA60ADF808008DF8F6
:108490000AB08DF80BB005A902A8F8F7FDFABDF8EF
:1084A0000C10BDF8140098F800208142404610D905
:1084B000012A08D0418001E05EE02EE088F800B09B
:1084C000C4F800B062E042888A4204D088F80070A4
:1084D00068E7012AF7D0089825F058FE00064BD42B
:1084E0004FF0020988F800909DF8040048B13A2046
:1084F00012F01DFA00063FD4012009F013FB00061C
:108500003AD40220F9F720F9000635D400E00EE055
:108510009DF800001C280FD018E0A020216001E089
:10852000D22021602860784630609120A1E72F603A
:108530007846306087209CE76846FDF77AFA0006A7
:108540001AD46846FDF75AFA000615D403F0C8FDA0
:108550009DF80000192807D01A2805D02760784612
:108560002F603060002084E79DF8040050B13E2069
:1085700012F0DDF9000601D520687AE700210BA092
:108580002EF043FA88F80090C4F800B078462F60C7
:10859000306001206DE700000CC0072010C00720EC
:1085A00014C007201C0400005EC10720200A200A16
:1085B000200A200A200A200A200A200A00000000BF
:1085C000F0B5054641799E4C9E4F9F4E8FB0862058
:1085D00009B1042902D92060062005E0297909B1F2
:1085E0001E2907D920600520386078463060862033
:1085F0000FB0F0BD6988288803F05AFC00067DD4CE
:1086000068796946FDF72AFD000677D4BDF80010A9
:108610000020A1F57F42FF3A71D0064600906846DF
:10862000FDF765FB000669D46846FDF791FF00067B
:1086300064D4012769463846FDF78CFB00065DD4FB
:108640007F1CFFB2112FF5D36846FDF7ADFB000686
:108650007ED46846FDF7B9FB000679D40127694648
:108660003846FDF79AFA000672D47F1CFFB20B2F32
:10867000F5D3012769463846FEF707F8000667D4A8
:108680007F1CFFB2112FF5D36846FDF74AFD0006A7
:108690005ED46846FDF76AFD000659D46846FDF7CA
:1086A00090FA000654D46846FDF7ADFA00064FD4A0
:1086B0006846FDF761FA00064AD40127009669462C
:1086C0003846FDF78EFF000642D47F1CFFB2052F0F
:1086D000F5D9ADF800606846FDF71AFB000637D4FF
:1086E0006846FDF726FB000632D46846FDF77AFAA5
:1086F00000062DD46846FDF797FA01E028E029E04E
:10870000000625D40096012669463046FDF736FB63
:1087100000061DD4761CF6B2112EF5D32846FDF7BF
:10872000F8F9000614D4A81CFDF704FA00060FD4CB
:10873000281DFDF710FA00060AD4012009F0F2F90D
:10874000000605D44FF00040FCF7F6FE000608D501
:1087500020684DE78B2121603860784630600846FC
:1087600046E701248DF800406846FDF78EF90006C3
:1087700033D436480470681DFDF7A8FA00062CD4DF
:108780006846FDF79DF9000627D46846FCF790FD82
:10879000000622D46846FDF789F900061DD4684614
:1087A000FDF79FF9000618D46846FCF75AFD00064D
:1087B00013D46846FDF78BF900060ED46846FDF722
:1087C000A1F9000609D46846FCF772FD000604D43E
:1087D0006846FDF78DF9000602D5FCF7A8FF07E70C
:1087E00008F044FE000624D48DF8014068798DF825
:1087F000020008F069FA00061BD4684607F0A6F9E3
:10880000000616D4684608F007FB000611D4FCF7F2
:10881000E0FE00060DD4684607F0C3F9000608D450
:10882000684608F024FB000603D4FCF7DEFE0006D1
:1088300002D508F07AFDD0E7FCF7E4FED8E60000A8
:108840000CC0072010C0072014C0072000C007205C
:1088500070B5057A724E96B00446102D0AD986205E
:10886000704930600320086078466F4908608620B0
:1088700016B070BD0DB90125257260680F902146B4
:108880000FA8FCF77EFC000605D44FF00040FCF773
:1088900053FE000601D53068EAE76846FDF731FA75
:1088A000000652D40FA96846FCF7F5FA00064CD42E
:1088B0006846FDF71CFA000647D46846FDF732FA11
:1088C000000642D4BDF80000401CADF80000684628
:1088D000FDF71EFA000638D469462846FDF746FA29
:1088E000000632D40FA96846FCF7D5FA00062CD44E
:1088F00069462846FDF72EFA000626D46946284622
:10890000FDF749FA000620D421466846FCF7FDFA37
:1089100000061AD469462846FDF730FA000614D43A
:1089200004F10800FDF762FA00060ED42046FDF7B8
:108930006EFA000609D4201DFDF77AFA000604D469
:108940000FA8FDF786FA000602D5FCF7F0FE8FE7C8
:1089500001202DF0EBFD000658D409F01CF80006AC
:1089600054D40D208DF80500207A8DF8130060682E
:10897000CDF807002068CDF80B000F98CDF80F0058
:108980002A4905A833F00EFF0DF10600FDF7A8F9FE
:1089900000063BD401A807F0D9F8000636D401A898
:1089A00008F03AFA000631D4012007F0ECFD000689
:1089B0002CD46846FEF785F8000627D49DF8000001
:1089C00090B11B48007878B111A8FDF789F900062D
:1089D0001CD48DF85050206812900F98139011A855
:1089E00006F061FB000611D4FCF7F3FD00060DD480
:1089F00001A807F0D6F8000608D401A808F037FA55
:108A0000000603D4FCF7F1FD000602D508F08DFC4A
:108A10009BE7064900200870FCF7F4FD28E70000FA
:108A20000CC0072010C0072014C00720D6C807209C
:108A30001C04000070B5057A744E96B00446102DE3
:108A40000AD986207249306003200860784671494F
:108A50000860862016B070BD05B9012560680F90CA
:108A600021460FA8FCF78DFB000605D44FF000400F
:108A7000FCF762FD000601D53068EBE76846FDF7BC
:108A800040F9000662D40FA96846FCF725FA0006F3
:108A90005CD46846FDF72BF9000657D46846FDF70D
:108AA00052F9000652D4BDF80000401CADF8000099
:108AB0006846FDF73EF9000648D46846FDF752FDCA
:108AC000000643D40FA96846FCF7E5F900063DD43B
:108AD0006846FDF73DFD000638D469462846FDF797
:108AE00045F9000632D40FA96846FCF7F5F90006EF
:108AF0002CD469462846FDF72DF9000626D4694690
:108B00002846FDF748F9000620D421466846FCF7C0
:108B10001DFA00061AD469462846FDF72FF900060B
:108B200014D404F10800FDF761F900060ED42046C4
:108B3000FDF76DF9000609D4201DFDF779F900064F
:108B400004D40FA8FDF785F9000602D5FCF7EFFD68
:108B500080E708F000FF00064FD40E208DF80500D6
:108B6000207A8DF813006068CDF807002068CDF8F2
:108B70000B000F98CDF80F00274905A833F012FE1F
:108B80000DF10600FDF7ACF8000636D401A806F09A
:108B9000DDFF000631D401A808F03EF900062CD410
:108BA0006846FDF78EFF000627D49DF8000090B1BF
:108BB0001A48007878B111A8FDF792F800061CD485
:108BC0008DF85050206812900F98139011A806F05D
:108BD000BAFA000611D4FCF7FCFC00060DD401A87B
:108BE00006F0DFFF000608D401A808F040F90006EF
:108BF00003D4FCF7FAFC000602D508F096FBA5E7C3
:108C0000054900200870FCF7FDFC23E70CC0072095
:108C100010C0072014C00720D6C807201C0400007D
:108C200030B504460079544D91B008B110280AD9E6
:108C30008620524928600320086078465049086021
:108C4000862011B030BD4FF00040FCF775FC0006E7
:108C500001D52868F5E76846FDF753F8000636D4D5
:108C600021466846FCF738F9000630D46846FDF71F
:108C70003EF800062BD420796946FDF777F8000608
:108C800025D421466846FCF727F900061FD4207931
:108C90006946FDF75FF8000619D4201DFDF71DF9A0
:108CA000000614D42046FDF707F900060FD46846E5
:108CB000FDF740FA00060AD421466846FCF7EBF8B7
:108CC000000604D46846FDF72CFA000602D5FCF72E
:108CD0002EFDB6E708F01FFE000647D408208DF8E9
:108CE00005000025CDF806500DF10B00FDF7CCF87E
:108CF00000063BD46846FDF7D8F8000636D4BDF828
:108D00000000ADF80C008DF80A502068CDF80E0078
:108D100001A806F01BFF000628D401A808F07CF883
:108D2000000623D46846FDF7CCFE00061ED49DF84D
:108D3000000048B11348007830B120680F900FA8A8
:108D400006F054FA000611D4FCF743FC00060DD4DB
:108D500001A806F026FF000608D401A808F087F84D
:108D6000000603D4FCF741FC000602D508F0DDFA4A
:108D7000ADE7FCF747FC64E70CC0072010C00720F4
:108D800014C007201C04000030B504460079694D6A
:108D900093B008B110280AD98620674928600320BB
:108DA0000860784665490860862013B030BD4FF0F2
:108DB0000040FCF7C1FB000601D52868F5E70EA8C6
:108DC000FCF79FFF000650D421460EA8FCF763F87D
:108DD00000064AD40EA8FCF78AFF000645D4207985
:108DE0000EA9FCF7C3FF00063FD421460EA8FCF7EE
:108DF00052F8000639D420790EA9FCF7ABFF000623
:108E000033D40FA8FDF760FC00062ED49DF83C007B
:108E100088B10EA9FDF746FC000626D421460EA80F
:108E2000FCF75AF8000620D40EA99DF83C00FDF787
:108E30002CFC000619D40EA8FDF77CF9000614D40A
:108E400021460EA8FCF748F800060ED40EA8FDF740
:108E500068F9000609D4201DFDF73FF8000604D488
:108E60002046FDF729F8000602D5FCF760FC9CE7D8
:108E700008F011FD000656D404208DF8010010A959
:108E80004C2012F029FD00064DD49DF840008007CB
:108E900002D49DF83C0020B9684606F057FE000653
:108EA00041D49DF840009DF83C1000F00100401EA8
:108EB000084204D1684607F0AFFF000633D40EA87D
:108EC000FDF7FFFD00062ED49DF8380048B11C4880
:108ED000007830B12068119011A806F0B1F90006B1
:108EE00021D4FCF776FB00061DD49DF840008007D6
:108EF00002D49DF83C0020B9684606F052FE0006F8
:108F000011D49DF840009DF83C1000F00100401E77
:108F1000084204D1684607F0AAFF000603D4FCF714
:108F200064FB000602D508F000FA9EE7FCF76AFB36
:108F30003BE700000CC0072010C0072014C007202A
:108F40001C04000030B504460079544D91B008B1BE
:108F500010280AD9862052492860032008607846E4
:108F600050490860862011B030BD4FF00040FCF73A
:108F7000E3FA000601D52868F5E76846FCF7C1FE6C
:108F8000000636D421466846FBF785FF000630D43C
:108F90006846FCF7ACFE00062BD420796946FCF746
:108FA000E5FE000625D421466846FBF774FF00065F
:108FB0001FD420796946FCF7CDFE000619D4201D88
:108FC000FCF78BFF000614D42046FCF775FF000663
:108FD0000FD46846FDF7D4F800060AD42146684647
:108FE000FBF759FF000604D46846FDF7BFF80006FA
:108FF00002D5FCF79CFBB6E708F023FC000647D43B
:1090000007208DF805000025CDF806500DF10B0066
:10901000FCF73AFF00063BD46846FCF746FF000623
:1090200036D4BDF80000ADF80C008DF80A50206869
:10903000CDF80E0001A806F089FD000628D401A88D
:1090400007F0EAFE000623D46846FDF73AFD000665
:109050001ED49DF8000048B11348007830B1206854
:109060000F900FA806F019F9000611D4FCF7B1FA19
:1090700000060DD401A806F094FD000608D401A84E
:1090800007F0F5FE000603D4FCF7AFFA000602D5A0
:1090900008F04BF9ADE7FCF7B5FA64E70CC0072020
:1090A00010C0072014C007201C04000070B504463F
:1090B0000079684E92B0032508B1102809D986209E
:1090C000306065480560784664490860862012B0C3
:1090D00070BD4FF00040FCF72FFA000601D5306854
:1090E000F5E70EA8FCF70DFE000650D421460EA8A9
:1090F000FBF7F2FE00064AD40EA8FCF7F8FD0006C6
:1091000045D420790EA9FCF731FE00063FD4214654
:109110000EA8FBF7E1FE000639D420790EA9FCF772
:1091200019FE000633D40FA8FDF7CEFA00062ED4A0
:109130009DF83C0088B10EA9FDF7B4FA000626D4CC
:1091400021460EA8FBF7C8FE000620D40EA99DF804
:109150003C00FDF79AFA000619D40EA8FDF710F8A6
:10916000000614D421460EA8FBF7B6FE00060ED466
:109170000EA8FCF7FBFF000609D4201DFCF7ADFE8E
:10918000000604D42046FCF797FE000602D5FCF743
:10919000CEFA9CE708F015FB000655D48DF8015077
:1091A00010A94C2012F098FB00064DD49DF8400009
:1091B000800702D49DF83C0020B9684606F0C6FC42
:1091C000000641D49DF840009DF83C1000F00100DD
:1091D000401E084204D1684607F01EFE000633D444
:1091E0000EA8FDF76EFC00062ED49DF8380048B19D
:1091F0001B48007830B12068119011A806F077F86C
:10920000000621D4FCF7E5F900061DD49DF84000C6
:10921000800702D49DF83C0020B9684606F0C1FCE6
:10922000000611D49DF840009DF83C1000F00100AC
:10923000401E084204D1684607F019FE000603D418
:10924000FCF7D3F9000602D508F06FF89FE7FCF7AA
:10925000D9F93CE70CC0072010C0072014C0072034
:109260001C04000010B5044692B04FF00040FCF71B
:1092700063F9000603D54348006812B010BD0FA87B
:10928000FCF73FFD000626D40FA8FCF76AFE000697
:1092900021D40F980E9021460EA8FBF71DFE000664
:1092A00019D40EA8FCF723FD000614D40EA8FCF771
:1092B00085FD00060FD421460EA8FBF7ECFD000645
:1092C00009D40EA8FCF770FD000604D42046FCF774
:1092D00037FE000602D5FCF72AFACEE708F051FA6D
:1092E000000648D408208DF801000F98CDF8020040
:1092F0000DF10700FCF70CFE00063CD40EA8FCF7AD
:1093000018FE000637D4BDF83800ADF8080000207C
:109310008DF806002068CDF80A00684606F016FCB5
:10932000000628D4684607F077FD000623D40EA86F
:10933000FDF7C7FB00061ED49DF8380048B112485F
:10934000007830B12068109010A805F04FFF00069B
:1093500011D4FCF73EF900060DD4684606F021FC56
:10936000000608D4684607F082FD000603D4FCF727
:109370003CF9000602D507F0D8FFACE7FCF742F94C
:109380007BE700000CC007201C04000030B5044639
:1093900093B04FF00040FCF7CFF8564D000619D4BB
:1093A0000EA8FCF7AEFC000631D40EA8FCF7D9FDE0
:1093B00000062CD421460EA8FBF76DFD000626D42E
:1093C0000EA8FCF794FC000621D40FA8FDF77CF949
:1093D000000602D5286813B030BD9DF83C00C8B126
:1093E0000EA9FDF75FF9000611D421460EA8FBF780
:1093F00073FD00060BD40EA99DF83C00FDF745F95E
:10940000000604D42046FCF79BFD000611D5FCF7AE
:109410008EF9E0E70EA8FCF7D1FC0006F7D4214650
:109420000EA8FBF759FD0006F1D40EA8FCF7BCFC12
:10943000E6E708F086F9000656D404208DF801000E
:1094400010A94C2012F048FA00064DD49DF84000B7
:10945000800702D49DF83C0020B9684606F076FBF0
:10946000000641D49DF840009DF83C1000F001003A
:10947000401E084204D1684607F0CEFC000633D4F3
:109480000EA8FDF71EFB00062ED49DF8380048B14B
:109490001948007830B12068119011A805F0D0FE6D
:1094A000000621D4FCF795F800061DD49DF8400075
:1094B000800702D49DF83C0020B9684606F071FB95
:1094C000000611D49DF840009DF83C1000F001000A
:1094D000401E084204D1684607F0C9FC000603D4C8
:1094E000FCF783F8000602D507F01FFF8FE7FCF7B3
:1094F00089F870E70CC007201C04000030B5044652
:1095000091B04FF00040FCF717F8444D000656D4D8
:109510000FA8FCF7F6FB000626D40FA8FCF721FDE8
:10952000000621D40F980E9021460EA8FBF7B3FC3D
:10953000000619D40EA8FCF7DAFB000614D40EA816
:10954000FCF74DFC00060FD421460EA8FBF7A3FC48
:10955000000609D40EA8FCF738FC000604D4204607
:10956000FCF7EEFC000603D5FCF7E1F811B030BDC6
:1095700008F087F800064AD40EA8FDF7A2FA000604
:1095800045D49DF8380048B12548007830B12068AE
:10959000109010A805F081FE000638D407208DF841
:1095A00001000F98CDF802000DF10700FCF7B0FCA8
:1095B000000604D40EA8FCF7BCFC000601D5286800
:1095C000D4E7BDF83800ADF8080000208DF806009B
:1095D0002068CDF80A00684606F0B8FA000616D4EE
:1095E000684607F019FC000611D4FBF7F2FF0006ED
:1095F0000DD4684606F0D5FA000608D4684607F090
:1096000036FC000603D4FBF7F0FF000602D507F096
:109610008CFEA9E7FBF7F6FFA8E700000CC00720C7
:109620001C04000010B5044692B04FF00040FBF758
:1096300083FF000603D55548006812B010BD0EA880
:10964000FCF75FFB00062ED40EA8FCF78AFC000690
:1096500029D421460EA8FBF73FFC000623D40EA810
:10966000FCF745FB00061ED40FA8FDF72DF80006F9
:1096700019D49DF83C00C8B10EA9FDF713F80006F7
:1096800011D421460EA8FBF727FC00060BD40EA927
:109690009DF83C00FCF7F9FF000604D42046FCF7D7
:1096A0004FFC000611D5FCF742F8C6E70EA8FCF700
:1096B00096FB0006F7D421460EA8FBF70DFC00062A
:1096C000F1D40EA8FCF781FBE6E707F0BAFF00062D
:1096D00056D403208DF8010010A94C2012F0FCF89C
:1096E00000064DD49DF84000800702D49DF83C0050
:1096F00020B9684606F02AFA000641D49DF84000D9
:109700009DF83C1000F00100401E084204D168465C
:1097100007F082FB000633D40EA8FDF7D2F900064D
:109720002ED49DF8380048B11948007830B120682F
:10973000119011A805F0DBFD000621D4FBF749FFCD
:1097400000061DD49DF84000800702D49DF83C001F
:1097500020B9684606F025FA000611D49DF84000AD
:109760009DF83C1000F00100401E084204D16846FC
:1097700007F07DFB000603D4FBF737FF000602D598
:1097800007F0D3FD8FE7FBF73DFF56E70CC007203E
:109790001C04000000B58FB04FF00040FBF7CCFE7A
:1097A000000603D51B4800680FB000BD07F029FF75
:1097B000000626D410208DF801000EA8FCF7A1FAAF
:1097C00000061ED40E98CDF80200684606F0BEF9D9
:1097D000000616D4684607F01FFB000611D4FBF7FD
:1097E000F8FE00060DD4684606F0DBF9000608D442
:1097F000684607F03CFB000603D4FBF7F6FE0006C4
:1098000004D507F092FDFBF792FFCDE7FBF7FAFED8
:10981000CAE700000CC00720F0B5734D070091B0F7
:10982000288802D040F0200001E040F0100028809D
:109830004FF00040FBF780FE6C4E000671D40FA87D
:10984000FCF74EFA000668D469469DF83C00FCF728
:1098500005FC000661D4BDF800006946401CADF867
:1098600000009DF83C00FCF7ECFB000655D4684670
:10987000FCF726F9000650D46846FBF72BFD0006DE
:109880004BD46846FCF712F9000646D46846FCF74C
:1098900028F9000641D46846FBF7F7FC00063CD4E3
:1098A0006846FCF714F9000637D46846FCF72AF935
:1098B000000632D46846FBF70DFD00062DD468463D
:1098C000FCF716F9000628D4002468460094FCF73B
:1098D0000EFA00067AD46846FDF7F3F8000602D5C2
:1098E00007F023FD19E002202CF020FE000614D41E
:1098F00038003F4F0DD09DF8000028B1387818B1DE
:1099000004F0DCFD000608D407F046FE000604D48F
:1099100011E007F041FE000604D5FBF708FF11B087
:10992000F0BD53E09DF8000028B1387818B104F07C
:10993000C5FD0006D4D410A96A2012F098F80006DC
:1099400044D49DF8400010F002008DF8400002D091
:10995000742010F0ECFF8DF800406846FCF7B6F973
:109960000006BDD48DF800406846FCF78EF800066E
:10997000B6D46846FCF75DF80006B1D49DF8000047
:10998000022806D18DF800406846FCF726F800064C
:10999000A6D402208DF8050007F096F900069FD4A2
:1099A00001A806F0D3F800069AD4FBF712FE0006D1
:1099B00096D401A806F0F5F8000691D4FBF715FE41
:1099C00000068DD4FBF71EFE000601D53068A6E721
:1099D000288820F0B000288006483460046078466B
:1099E0000549086000209AE702C007200CC0072044
:1099F0001C04000010C0072014C00720FE4909887D
:109A000001807047FC4949880180704730B58FB0AC
:109A100005460B208DF801000EA8FCF762F8F74C04
:109A2000000630D4BDF83800ADF80A000EA8FCF7E7
:109A300047F8000627D40E98CDF8060028798DF84F
:109A40000C002888ADF802006888ADF8040068466C
:109A500006F07CF8000616D4684607F0DDF900062B
:109A600011D4FBF7B6FD00060DD4684606F099F850
:109A7000000608D4684607F0FAF9000603D4FBF79D
:109A8000B4FD000602D520680FB030BDDC490020CF
:109A9000206008607846DB4908600020F4E72DE983
:109AA000F34F9BB007461C99002011900870D249D3
:109AB0003888DFF84CB30880788848803879CF4DF3
:109AC000862408B11E2804D905212C60CBF800108B
:109AD00012E0388848F6AD61142688421DD878888F
:109AE0004FF01708B0F5B46F0DD32C607846C54918
:109AF000CBF80080086002E07946C2480160862009
:109B00001DB0BDE8F08F05A8FCF70DF800067CD469
:109B10003888BDF81410884203D22C60CBF800605E
:109B2000EAE70DD105A8FCF70FF80006EFD4788816
:109B3000BDF81410884203D22C60CBF80080DBE71C
:109B400002A8FCF723F80006E1D405A8FCF7D9F831
:109B50000006DCD405990298814209D08C20286047
:109B600000207946CBF80000A64801608C20C7E7AA
:109B7000022006F008FD0006C9D4012004F073FF9E
:109B80000006C4D44FF00040FBF7D6FC0006BED45C
:109B90006846FCF7A5F800067DD405A8FCF7B1F8E7
:109BA0000006F9D4059898B102A99DF80000FCF7C9
:109BB00029FA0006F0D405A902A8FBF7FBF8000675
:109BC000EAD402A99DF80000FCF70FFA0006E3D4DE
:109BD00005A8FCF7C7FC0006DED4059898B102A9D9
:109BE0009DF80000FCF7D2FC0006D5D405A902A818
:109BF000FBF7E0F80006CFD402A99DF80000FCF7BF
:109C0000B8FC0006C8D402A900E0D9E09DF8000025
:109C1000FCF70EFA0006BFD4BDF8080002A9401CEC
:109C2000ADF808009DF80000FCF7F5F90006B3D484
:109C300005A8FCF777F80006AED4BDF8140098B17B
:109C400002A99DF80000FCF799FB0006A4D405A921
:109C500002A8FBF794F900069ED402A99DF8000023
:109C6000FCF77FFB000697D405A8FCF76CF800060C
:109C700092D4BDF81400A8B102A99DF80000FCF729
:109C800093FB000688D405A902A8FBF778F9000623
:109C900087D402A900E08AE29DF80000FCF777FB78
:109CA000000687D401208DF80400C0B205A9FCF796
:109CB0005DF8000684D40598B8B19DF8041002AA96
:109CC0009DF80000FCF7E6F9000685D405A902A876
:109CD000FBF770F8000688D49DF8041002AA9DF8DE
:109CE0000000FCF7C7F9000685D49DF8040005A91B
:109CF000FCF751F8000685D40598B8B19DF804101A
:109D000002AA9DF80000FCF7E1F900068FD405A92E
:109D100002A8FBF79FF8000689D49DF8041002AA58
:109D20009DF80000FCF7C5F9000685D49DF80400F5
:109D3000401CC0B28DF804001028B6D905A8FCF765
:109D40003DF8000688D4059E4FF000089EB102A998
:109D50009DF80000FCF73EFA000684D405A902A88D
:109D6000FBF728F800068DD402A99DF80000FCF747
:109D700024FA000686D405A8FCF731F8000687D43B
:109D800005984FF00009B0F1000A13D002A99DF820
:109D90000000FCF735FA00068CD405A902A8FBF7F1
:109DA00009F8000686D402A99DF80000FCF71BFA0A
:109DB00000068AD401A90B2011F08EFD000601D502
:109DC00028689DE69DF80400012801D0032823D1CE
:109DD00005A8FBF796FF000686D402AA01219DF88C
:109DE0000000FCF78FF9000685D405A902A8FAF750
:109DF000E1FF00068AD407E064C107200CC00720F9
:109E000010C0072014C0072002AA01219DF80000FD
:109E1000FCF768F9000688D49DF80400022803D0F6
:109E2000042801D0062873D146EA0A0048EA09014D
:109E300008436ED086EA0A0188EA0900014368D027
:109E400000200990BAEB060179EB080005D2B6EBC9
:109E50000A0A68EB0904012004E0BAEB060A69EB80
:109E6000080400201A900020814680460646012002
:109E70008DF80400C0B205A9FBF778FF00068BD46B
:109E800005999DF8040019EB010948EB060805A99E
:109E9000FBF781FF000685D4059810B10998401C96
:109EA00009909DF80400401CC0B28DF804001028F1
:109EB000E0D9002610208DF80400C0B205A9FBF7F8
:109EC00055FF000688D40598049030434BD0049881
:109ED000AAFB003204FB00200AFB06015FEA5802DD
:109EE0004FEA3900181851414A46434632F036F9D4
:109EF000BAEB000A049A64EB0104B9EB02091A9A5E
:109F000068EB060832B1049A101A66EB010604E009
:109F100082E056E0049A10184E4109990590491EB6
:109F200009919DF8041002AA9DF80000FCF7EAF8D8
:109F30000006A4D405A902A8FAF73CFF00069ED4A7
:109F40009DF8041002AA9DF80000FCF7CBF800066B
:109F500095D400BF9DF80400401E10F0FF008DF85E
:109F60000400AAD158E05AEA0400F3D059EA0800E4
:109F7000F0D19DF8040005A9FBF70DFF00068AD477
:109F800005980028E6D01A9848B1092028600020DA
:109F9000CBF800007846FE4908600920B0E5099832
:109FA00000EBD070421012EB0A0044EBE271099A08
:109FB0004FEAE27332F0D2F8BAEB000A64EB010424
:109FC000A8E701208DF80400C0B205A9FBF7CEFE7A
:109FD0000006AED40598B8B19DF8041002AA9DF809
:109FE0000000FCF78FF80006A3D405A902A8FAF731
:109FF000E1FE00069DD49DF8041002AA9DF8000021
:10A00000FCF770F8000694D49DF80400401CC0B220
:10A010008DF804001028D7D901248DF8044000BF22
:10A020009DF8040005A9FCF73DFB000687D40598C0
:10A03000B8B19DF8041002AA9DF80000FCF716FBC9
:10A04000000685D405A902A8FAF7B4FE000696D446
:10A050009DF8041002AA9DF80000FCF7F7FA00062C
:10A060008DD49DF80400401CC0B28DF80400112866
:10A07000D6D305A8FCF75EF80006AAD4059898B1D7
:10A0800002A99DF80000FCF768F80006A1D405A914
:10A0900002A8FAF78FFE00069BD402A99DF80000E3
:10A0A000FCF74EF8000694D405A8FCF769F8000602
:10A0B0007DD4059898B102A99DF80000FCF774F8CA
:10A0C000000674D405A902A8FAF774FE00066ED43F
:10A0D00002A99DF80000FCF75AF8000667D48DF835
:10A0E000044000BF9DF8040005A9FBF762FD0006CF
:10A0F0005DD40598B8B19DF8041002AA9DF800003F
:10A10000FCF797F8000652D405A902A8FAF752FE08
:10A1100000064CD49DF8041002AA9DF80000FCF73C
:10A1200078F8000643D49DF80400401CC0B28DF8B6
:10A1300004000B28D6D305A8FBF7E3FD000636D4B0
:10A14000059898B378883C21B0FBF1F0401CC1B26F
:10A150008DF8041002AA9DF80000FCF789F80006AB
:10A1600025D405A902A8FAF725FE00061FD49DF8FC
:10A17000041002AA9DF80000FCF76AF8000616D445
:10A18000397902AA9DF80000FCF791F800060ED478
:10A1900005A902A8FAF70EFE000608D4397902AA2A
:10A1A0009DF80000FCF773F8000600D400E087E09B
:10A1B0008DF804409DF8040005A9FCF71FFA00067D
:10A1C0007ED49DF8041002AA9DF80000FCF72FFA37
:10A1D000000675D405A902A8FAF7ECFD00066FD4B5
:10A1E0009DF8041002AA9DF80000FCF710FA000682
:10A1F00066D49DF80400401CC0B28DF80400052808
:10A20000D8D902A90120FBF738FC000658D405A9CB
:10A210000120FBF7CEFC000652D49DF80000012877
:10A2200014D002280DD003280BD004280ED088208B
:10A2300002212860CBF8001079465548016088203B
:10A240005EE405A902A8FAF72FFF03E005A902A81A
:10A25000FAF7EFFE00067AD402A90120FBF701FC11
:10A26000000674D4012006F08EF900066FD413A8FE
:10A27000FCF727FC00066AD446499DF84C004FF0D5
:10A2800092060978084267D016A9032006F0FEF866
:10A2900000065CD418A9052004F044FB000656D43F
:10A2A000052216A918A832F051FA88B1FBF73FFA37
:10A2B000422010F03CFB08202CF092FD312000E001
:10A2C0001BE02E60CBF800007846314908605CE066
:10A2D00012A9002004F026FB000638D49DF848009F
:10A2E00080062FD507F038F9000604D43846FFF76A
:10A2F0008DFB000602D507F018F828E03888ADF885
:10A3000028007888ADF82A0038798DF82C0014A937
:10A310000AA805F019F8DBF8000028280FD02878E3
:10A320000006E8D414A8FBF72DFE0006E3D415A818
:10A33000FBF739FE0006DED41C98047015E00120FE
:10A340001190EFE705A8FBF7DCFC000602D5FBF750
:10A35000EEF90CE4059840B907F0FEF80006CAD4FF
:10A360003846FFF753FB0006C5D48DF8044001A81A
:10A37000FBF733FB0006BED4119868B128212E608C
:10A38000CBF80010794602480160922019E50000E0
:10A3900014C007201C040000FBF734F911E500008D
:10A3A000F8B5054646793B4C3B4A3C4B86200EB1FE
:10A3B000022E02D92060072005E02E790EB11E2E54
:10A3C00006D9206005201060784618608620F8BD08
:10A3D00029B16988288801F06BFD000641D4002767
:10A3E0000126009769463046FBF7D7FB000638D4B4
:10A3F000761CF6B20B2EF5D36846FBF7E2FB00069F
:10A400002FD46846FBF7FFFB00062AD46846FBF70B
:10A41000B3FB000625D4ADF800706846FBF7E2FBFD
:10A4200000061ED46846FBF7FFFB000619D4284639
:10A43000FBF76FFB000614D4A81CFBF77BFB0006A0
:10A440000FD4281DFBF787FB00060AD4012007F074
:10A4500069FB000605D44FF00040FBF76DF80006DD
:10A4600001D52068F8BD02208DF800006846FBF792
:10A470000CFB000607D40A4901200870681DFBF791
:10A48000A3FD000602D5FBF752F9F8BDFBF7BAF8B9
:10A49000F8BD00000CC0072010C0072014C0072022
:10A4A00000C007201CB54FF00040FBF745F8000640
:10A4B00002D5174800681CBD07F084FC00061ED4B6
:10A4C00000248DF800406846FBF7DFFA000616D43A
:10A4D0008DF8044001A8FBF777FD00060FD468460D
:10A4E000FBF7A7FA00060AD49DF8000002280BD15A
:10A4F0008DF800406846FBF770FA000604D506F0B8
:10A5000014FFFBF714F91CBDFBF77CF81CBD000021
:10A510000CC007202DE9F04F054600799A4C9B4E60
:10A520009B4F93B04FF086084FF0050B08B11E28E3
:10A5300004D9C4F80080C6F800B017E0288848F6AF
:10A54000AD614FF01409884205D900BFC4F80080FE
:10A55000C6F800900AE068884FF0170AB0F5B46FAB
:10A560000AD300BFC4F80080C6F800A0784638605F
:10A57000862013B0BDE8F08F02A8FBF7D4FA0006DE
:10A5800015D42888BDF808108842DFD309D102A865
:10A59000FBF7DAFA00060AD46888BDF8081088428A
:10A5A000E0D34FF00040FAF7C7FF000601D520685E
:10A5B000DFE76846FBF712FD00067CD402A8FBF734
:10A5C000E5FA000677D4029898B103A99DF8000037
:10A5D000FBF789FE00066ED402A903A8FAF7EAFB8E
:10A5E000000668D403A99DF80000FBF76FFE000683
:10A5F00061D403A99DF80000FBF78BFE00065AD436
:10A60000BDF80C0003A9401CADF80C009DF800003B
:10A61000FBF772FE00064ED40120804602A9FBF72C
:10A62000C8FA000647D40298A8B103AA41469DF88B
:10A630000000FBF787FE00063DD402A903A8FAF745
:10A64000B9FB000637D403AA41469DF80000FBF78A
:10A6500069FE00062FD408F10100C0B280460A2826
:10A66000DCD903A90120FBF708FA000623D402A9CC
:10A670000120FBF79EFA00061DD49DF800004FF064
:10A68000880801280BD0022803D00220C4F80080DB
:10A690001DE002A903A8FAF707FD04E00BE002A9F8
:10A6A00003A8FAF7C6FC000605D403A90120FBF7AE
:10A6B000D8F9000602D5FBF73AF85AE79DF80000F2
:10A6C000012809D002280AD00920C4F8008030608F
:10A6D0007846386088204CE78DF815B002E00620F7
:10A6E0008DF8150002A8FBF7FCF9000642D4BDF86E
:10A6F0000800401CADF81E0002A8FBF7E1F90006B7
:10A7000038D40298401CCDF81A0002A8FBF7D7FAFB
:10A7100000062FD4029808901E490DF1250032F052
:10A7200041F828798DF824002888ADF8160068884B
:10A73000ADF8180006F0C8FA00061BD405A805F00D
:10A7400005FA000616D405A806F066FB000611D42B
:10A75000FAF73FFF00060DD405A805F022FA00061F
:10A7600008D405A806F083FB000603D4FAF73DFFE2
:10A77000000602D506F0D9FD9DE7064900200870C5
:10A78000FAF740FFF5E600000CC0072010C00720D4
:10A7900014C00720D6C8072030B5044600785C4DA9
:10A7A00091B008B10A280AD986205A4928600420A5
:10A7B0000860784658490860862011B030BDA0680E
:10A7C0000E90211D0EA8FAF7DCFC000605D44FF010
:10A7D0000040FAF7B1FE000601D52868EDE70FA8A2
:10A7E000FBF7F9F9000650D40EA90FA8FAF753FBAE
:10A7F00000064AD40FA8FBF7E4F9000645D40FA8D9
:10A80000FBF7FAF9000640D4BDF83C00401CADF857
:10A810003C000FA8FBF7E6F9000636D420780FA914
:10A82000FBF7C7F9000630D40EA90FA8FAF733FBDF
:10A8300000062AD420780FA9FBF7AFF9000624D42C
:10A840000FA8FBF7A3F900061FD40EA90FA8FAF76B
:10A8500022FB000619D40FA8FBF78EF9000614D4CA
:10A860002046FBF7F2F900060FD4201DFBF70AFA89
:10A8700000060AD404F10800FBF70DFA000604D420
:10A880000EA8FBF712FA000602D5FAF750FF94E77C
:10A8900007F0A1F8000635D410A8FBF700F9000670
:10A8A00030D49DF84000022803D107F09FFA00063B
:10A8B00028D49DF84000012827D109208DF80100F7
:10A8C00020788DF802000E98CDF80300684605F058
:10A8D0003DF9000616D4684606F09EFA000611D42B
:10A8E000FAF777FE00060DD4684605F05AF900061F
:10A8F00008D4684606F0BBFA000603D4FAF775FEE2
:10A90000000602D506F011FDBFE7FAF77BFE54E71B
:10A910000CC0072010C0072014C0072030B5044623
:10A920000078544D91B008B10A280AD986205249BE
:10A93000286004200860784650490860862011B0DD
:10A9400030BDA0680E90211D0EA8FAF71AFC000673
:10A9500005D44FF00040FAF7EFFD000601D5286856
:10A96000EDE70FA8FBF737F9000650D40EA90FA8A2
:10A97000FAF7B2FA00064AD40FA8FBF722F900064C
:10A9800045D40FA8FBF738F9000640D4BDF83C00C9
:10A99000401CADF83C000FA8FBF724F9000636D4A4
:10A9A00020780FA9FBF705F9000630D40EA90FA8EF
:10A9B000FAF792FA00062AD420780FA9FBF7EDF8EF
:10A9C000000624D40FA8FBF7E1F800061FD40EA957
:10A9D0000FA8FAF781FA000619D40FA8FBF7CCF8F4
:10A9E000000614D42046FBF730F900060FD4201DD2
:10A9F000FBF748F900060AD404F10800FBF74BF90D
:10AA0000000604D40EA8FBF750F9000602D5FAF7A9
:10AA10008EFE94E706F0FFFF000624D40A208DF88E
:10AA2000010020788DF802000E98CDF803006846EA
:10AA300005F08CF8000616D4684606F0EDF900061D
:10AA400011D4FAF7C6FD00060DD4684605F0A9F842
:10AA5000000608D4684606F00AFA000603D4FAF79E
:10AA6000C4FD000602D506F060FCD0E7FAF7CAFD87
:10AA700065E700000CC0072010C0072014C00720A5
:10AA800030B504460078564D91B008B10A280AD96D
:10AA9000862054492860042008607846524908609E
:10AAA000862011B030BDA0680E90211D0EA8FAF7C7
:10AAB00068FB000605D44FF00040FAF73DFD0006A4
:10AAC00001D52868EDE70FA8FBF7A7F8000650D4DA
:10AAD0000EA90FA8FAF7DFF900064AD40FA8FBF772
:10AAE00092F8000645D40FA8FBF7A8F8000640D45A
:10AAF000BDF83C00401CADF83C000FA8FBF794F8F3
:10AB0000000636D420780FA9FBF753F8000630D49E
:10AB10000EA90FA8FAF7E0F900062AD420780FA9A9
:10AB2000FBF73BF8000624D40FA8FBF72FF800062C
:10AB30001FD40EA90FA8FAF7CFF9000619D40FA851
:10AB4000FBF71AF8000614D42046FBF77EF800063F
:10AB50000FD4201DFBF796F800060AD404F1080074
:10AB6000FBF799F8000604D40EA8FBF79EF8000640
:10AB700002D5FAF7DCFD94E706F06DFF000629D454
:10AB800011208DF801000FA8FBF725F8000621D44D
:10AB90000F98CDF802000E98CDF80600684604F034
:10ABA000D5FF000616D4684606F036F9000611D423
:10ABB000FAF70FFD00060DD4684604F0F2FF000618
:10ABC00008D4684606F053F9000603D4FAF70DFDE1
:10ABD000000602D506F0A9FBCBE7FAF713FD60E704
:10ABE0000CC0072010C0072014C007202DE9F04F2B
:10ABF00085B06846FAF7FBFEF84F00060ED49DF8C4
:10AC00000000DFF8DC93DFF8DCA30024012809D082
:10AC100001A90120FBF7F6F9000607D5386805B051
:10AC2000BDE8F08F3C60C9F800401CE18DF80040A1
:10AC30000DF104029DF800009DF80410135C401C07
:10AC4000C0B219448DF804108DF800000528F1D326
:10AC50001046FAF7AEF900067DD4A0460494ADF88C
:10AC60000C400124E04EDFF884B3254630780228FA
:10AC700005D000EB40000BEBC00040688047E8B215
:10AC8000054601A9FBF7B1F90006E5D401A928465C
:10AC9000FBF76FFC0006DFD403A92846FBF7BBF9DE
:10ACA0000006D9D403A92846FBF7CBF90006D3D474
:10ACB00003A92846FBF755FB00064CD403A92846F8
:10ACC000FBF765FB000646D48DF800409DF80010A8
:10ACD00001AA2846FBF7CEF900063CD49DF80010E7
:10ACE00004AA2846FBF7E5F9000634D49DF80010C5
:10ACF00001AA2846FBF7F6F900062CD49DF80000BF
:10AD0000401CC0B28DF800001028DFD901A92846E8
:10AD1000FBF753FA00061ED401A92846FBF763FA95
:10AD2000000618D48DF800409DF8001001AA2846AE
:10AD3000FBF76FFA00060ED49DF80000401CC0B26D
:10AD40008DF800000A28EFD98DF800409DF800101A
:10AD500001AA284600E073E0FBF77AFA00066FD4F8
:10AD60009DF80000401CC0B28DF800001828EDD9F5
:10AD70008DF800409DF8001001AA2846FBF787FADD
:10AD800000065DD49DF80000401CC0B28DF80000A4
:10AD90001E28EFD98DF800409DF8001001AA284622
:10ADA000FBF735FC00064BD49DF80000401CC0B2F8
:10ADB0008DF800000528EFD98DF800409DF80010AF
:10ADC00001AA2846FBF742FC000639D49DF8000092
:10ADD000401CC0B28DF800001028EFD901A9284608
:10ADE000FBF7AEF900062BD401A92846FBF7CFF9F3
:10ADF000000625D46D1CEDB2042D7FF637AF254635
:10AE00003078022805D000EB40010BEBC100406810
:10AE10008047E0B2044601A9FBF758FA00060FD4B8
:10AE200003A92046FBF768FA000609D428468DF8E6
:10AE30000050C1B201AA2046FBF774FA000602D501
:10AE4000FAF775FCEBE69DF80000401CC0B28DF8E7
:10AE500000000A28EDD9641CE4B2022CD0D9C7F84E
:10AE60000080C9F8008079460020CAF80010D6E6B4
:10AE7000F0B504460179594D594E5A4F91B086208C
:10AE800009B11E2902D9286005200DE0218848F665
:10AE9000AD62914202D92860142005E06188B1F5C5
:10AEA000B46F07D32860172030607846386086205A
:10AEB00011B0F0BD0FA9022005F03BFD000615D42E
:10AEC000BDF83C00A0B104F045FD00060ED4464894
:10AED0000678012E04D0012006F024FE000605D4D9
:10AEE0004FF01040FAF728FB000609D52868DFE785
:10AEF000912028608A203060784638609120D7E71A
:10AF0000FFF774FE000620D401F0EAF800061CD416
:10AF10002046FBF752FA000617D4A01CFBF75CFA98
:10AF2000000612D4201DFBF768FA00060DD401209C
:10AF30008DF800006846FAF750FD000605D4694612
:10AF40002B2010F0C9FC000602D5FAF7F0FBAFE7A2
:10AF50009DF80000C00701D16079E8B3012E49D007
:10AF60006846FAF7ADFD000633D46846FAF7A0F953
:10AF700000062ED46846FAF799FD000629D406F09B
:10AF800051F9000625D41A490220087012208DF8C4
:10AF900005006946042005F079FA000619D4BDF8C9
:10AFA0000000401CADF8060020798DF810002088C4
:10AFB000ADF808006088ADF80A006846FAF780FD31
:10AFC000000606D40098039001A804F0EAFD0006EC
:10AFD00010D506F0AAF9B8E70CE000000CC0072075
:10AFE00010C0072014C00720CAC30720CCC3072005
:10AFF00000C00720FAF706FB5AE70000F8B505463F
:10B000000379384C3849394A86200BB11E2B02D9B6
:10B01000206005200EE02B8848F6AD671426BB4261
:10B0200002D920600E6006E06B88B3F5B46F06D3DA
:10B03000206017200860784610608620F8BD2C49F3
:10B040000120FAF7DFFF000640D42A490220FAF770
:10B05000D9FF00063AD42846FAF75BFD000635D43E
:10B06000A81CFAF767FD000630D4281DFAF773FD17
:10B0700000062BD4002568460095FBF749FA000628
:10B0800024D468460095FBF752FA00061ED48DF8CA
:10B0900000606846FBF7EEF9000617D40120ADF812
:10B0A00000006846FBF70DFA00060FD469461C2025
:10B0B00010F012FC000609D49DF8000040B1ADF874
:10B0C00000506846FAF703FD000601D52068F8BD78
:10B0D000032009498DF80000022008706846FAF73D
:10B0E000D4FCF8BD0CC0072010C0072014C00720F6
:10B0F00078C107207DC1072000C007202DE9FC4151
:10B100004FF00040FAF718FA4C4C00067ED468461F
:10B11000F9F75BFF00062AD401273E46F0B2054648
:10B120006946FAF79EFC000621D46D1CEEB20B2E88
:10B13000F4D3002568460095FAF7B8FC000616D44B
:10B14000ADF800506846FAF7C2FC00060FD4684616
:10B150000095FAF7CDFC000609D4ADF80070022086
:10B16000C0B206466946FBF796F9000605D506F01B
:10B17000DCF8FAF7DCFABDE8FC81761CF0B21B289B
:10B18000EED92F4F04226946384625F035F80006DF
:10B190004ED42C4E0098B04227D004226946381D68
:10B1A000009525F034F8000642D42548042269466B
:10B1B000083025F02CF800063AD4214804226946CC
:10B1C0000C3025F024F8000632D41D4804226946CC
:10B1D000103025F01CF800062AD4042269463846AF
:10B1E000009625F014F8000622D41548042269467A
:10B1F0001430009525F00BF8000619D410480422ED
:10B200006946183025F003F8000600E010E00FD47E
:10B210000B48042269461C3024F0F9FF000607D4CD
:10B22000074804226946203024F0F1FF000601D5CA
:10B230002068A0E7FAF7E6F99DE700000CC00720B8
:10B2400004000020CEFAADDEFEB56846F9F7B1FE87
:10B25000284C000640D400270125ADF808702E4682
:10B26000F0B206466946FAF7C0FE000634D402A9D9
:10B270003046FAF7D0FE00062ED402A93046FAF77F
:10B28000E0FE000628D402A93046FBF76AF8000663
:10B2900022D402A93046FBF77AF800061CD469468E
:10B2A0003046FAF78AFF000616D469463046FAF7A8
:10B2B0009AFF000610D4761CF6B2042ED0D9E8B25C
:10B2C00005466946FBF702F8000605D402A92846A0
:10B2D000FBF712F8000601D52068FEBD6D1CEDB22B
:10B2E000022DECD9044827600760784603490860BE
:10B2F0000020FEBD0CC0072010C0072014C007208E
:10B300007CB506466846F9F754FE0D4D000607D495
:10B3100001246A4631462046FAF79AFF000601D515
:10B3200028687CBD641CE4B2052CF2D305490020DA
:10B330002860086078460449086000207CBD000051
:10B340000CC0072010C0072014C007207CB506469B
:10B350006846F9F72EFE0D4D000607D401246A4613
:10B3600031462046FAF793FF000601D528687CBDD8
:10B37000641CE4B2052CF2D3054900202860086063
:10B3800078460449086000207CBD00000CC00720FE
:10B3900010C0072014C00720FEB507466846F9F71D
:10B3A00008FE144D000617D40026012402966A46B2
:10B3B00039462046FAF75EFE00060DD402AA394649
:10B3C0002046FAF776FE000606D46A46394620463D
:10B3D000FAF788FE000601D52868FEBD641CE4B2B9
:10B3E000052CE4D304482E600660784603490860C3
:10B3F0000020FEBD0CC0072010C0072014C007208D
:10B400002DE9FC4107466846F9F7D3FD144E0006C6
:10B4100015D401252C46E0B204466A463946FAF7AF
:10B42000F8FE00060BD4641CE4B2052CF3D3E8B29A
:10B4300004466A463946FAF775FF000602D53068B9
:10B44000BDE8FC81641CE5B2032DF0D30549002062
:10B45000306008607846044908600020F0E700008A
:10B460000CC0072010C0072014C007202DE9F04FA2
:10B4700097B080464FF000098A4681F80090052079
:10B4800003F0F1FAFC4C00067ED4FF2005F07BF8B7
:10B490000006F9D415A8FBF714FB0006F4D469469E
:10B4A000002004F036FF0006EED4BDF8000090271F
:10B4B000F24DF34E192802D301202760E1E06946DE
:10B4C000022005F036FA0006DED4BDF8000090B187
:10B4D000EC480DF12C0B007800287CD06946012047
:10B4E00004F017FF0006CFD4BDF80000402805D3B4
:10B4F00003202760C5E00C202760C2E014A90020CB
:10B5000003F010FA0006BFD49DF85000010902D0E4
:10B5100004202760B5E001070BD5400709D4872038
:10B5200020607846C5F800903060872017B0BDE8ED
:10B53000F08F03A9052003F0F5F90006A4D46946AD
:10B54000032004F0A3FF00069ED42068052805D040
:10B55000052203A9684631F0F9F8D0B19DF85000F2
:10B5600000077DD56946002004F090FF00068BD4CB
:10B5700003A90B2003F0D6F9000685D40C2203A9F9
:10B58000684631F0E3F800E08EE028B1052027603E
:10B5900077E00720276074E003A90C2003F0C2F9CC
:10B5A000000691D4062208F1060103A831F0CEF876
:10B5B00010B10620276064E003A9112003F0B2F95E
:10B5C000000671D40622414603A831F0BFF818B135
:10B5D0000820276055E0D4E069460E2003F0A2F968
:10B5E000000661D403A800F0CCFC00065CD4BDF8D2
:10B5F0000000BDF80C10884207D963200FF097F9BE
:10B60000000651D4092027603BE003A9F5F7A9F90A
:10B610009DF80C00694600F5FA60ADF82C009DF825
:10B620000D008DF82E009DF80E008DF82F000F20D4
:10B6300003F078F9000637D4BDF800103C20B1FBC8
:10B64000F0F28DF83020B1FBF0F200FB12108DF813
:10B6500031008DF8329003A9102003F063F900E067
:10B6600023E0000620D46946042004F00FFF000602
:10B670001AD4BDF80000BDF80C10884206D00A208C
:10B68000276028607846306090204FE769460620A2
:10B6900003F048F9000672D4BDF80C00BDF80010A4
:10B6A000401C8142EBD110E069E003F0F5F900287D
:10B6B0007FF46FAF0BF1040022F0E2FC00065ED4D1
:10B6C0000BA822F00EFD000659D404F083F9000601
:10B6D00055D40BF10701002004F0D8FE00064ED42B
:10B6E000D8F80610CDF83F10B8F80A00ADF84300BE
:10B6F000D8F80010CDF84510B8F80400ADF84900AE
:10B7000013A9042004F0C2FE000638D4D8F80610AD
:10B710000791B8F80A00ADF82000D8F80010CDF86D
:10B720002210B8F80400ADF82600D8F80C000A90F2
:10B7300006A90BA8F5F7B0F9BDF84C00ADF81A0052
:10B7400006A8FAF7E6F9000619D49DF830109DF81E
:10B750003100C1EB011100EB8100ADF8000068463B
:10B76000FAF7E8F900060AD44748FAF7F4F90006B0
:10B7700005D44FF00040F9F7DFFE000604D520683D
:10B78000D4E60BF1040097E706F012FA00066ED437
:10B7900006A806F022FA000669D49DF850000007BA
:10B7A00007D43848007820B10BA803F083F90006CD
:10B7B0005DD4344F4FF001088AF800803878D8B152
:10B7C00003F0FBFB000652D40121304806F033FAA7
:10B7D00000060AD5F4F71EFD02F070FEF4F72FFD07
:10B7E00005F0A3FDF9F7A3FFC9E703F022FC00066B
:10B7F0003DD420680028E7D0112005F050F800065D
:10B8000035D406A9002005F05AF800062FD4387860
:10B8100058B107A9052003F085F8000627D406A92A
:10B82000012005F04CF8000621D4122005F037F86D
:10B8300000061CD49DF8540050B36846FAF740F94E
:10B84000000614D46846F9F733FD00060FD46846A5
:10B85000FAF72CF900060AD4FBF74FF9000606D4D4
:10B860004F468AF80090F9F7CDFE00065AD505F04C
:10B870005CFDF9F75CFF59E60CC0072010C00720FB
:10B8800014C007201C04000071C3072008C707204C
:10B89000FFE747468DF800806846FBF72BF9000666
:10B8A000E5D4ADF81090CDF80C908DF81290B84614
:10B8B00038468DF80070C0B203A9FAF7D2F8000636
:10B8C000D5D49DF80000401CC0B28DF800000A28B5
:10B8D000F1D94F4603A8CDF80C90FAF7E7F8000627
:10B8E000C5D403A80397FAF703F90006BFD4ADF84F
:10B8F0000C7003A8FAF7EBF80006B8D44046ADF890
:10B900000C808DF80080C0B203A9FAF7C4FD0006D0
:10B91000ADD49DF80000401CC0B28DF800001B287B
:10B92000F1D999E7276078462F6030600020FDE567
:10B930002DE9F04796B0002180460170052003F004
:10B9400092F8C04C00067DD4FF2004F01CFE0006D7
:10B95000F9D415A8FAF74BF80006F4D49DF8540072
:10B96000B94EBA4D48B1912020609C20286078469D
:10B970003060912016B0BDE8F0876946012004F0E0
:10B98000C8FC0006DFD4BDF800009027402802D391
:10B990000320276027E06946022004F0CAFF000662
:10B9A000D1D4BDF80000E0B103F076F80006CAD4A7
:10B9B00028684FF002094FF0920A232809D00FA9F6
:10B9C000002002F0AFFF0006BDD49DF83C00000946
:10B9D0000BD0C4F800A07846C5F8009030609220E3
:10B9E000C8E70C202760286061E003A9052002F069
:10B9F00099FF0006A7D46946032004F047FD00061E
:10BA0000A1D420684FF0070A28B90522694603A887
:10BA100030F09CFE98B39DF83C0000077DD5694648
:10BA2000002004F033FD00068DD403A90B2002F0A2
:10BA300079FF000687D40C2203A9684630F086FE01
:10BA400020B100E0A6E005202760CCE769460E2083
:10BA500002F068FF000695D403A800F092FA0006F1
:10BA600090D4BDF80000BDF80C10884208D06320C7
:10BA70000EF05DFF000685D409202760B3E713E0D0
:10BA80006946042004F002FD000689D403A91020B1
:10BA900002F048FF00067DD4BDF80000BDF80C1090
:10BAA0004FF00A0A884206D02760C5F800A0784601
:10BAB000306090205EE76946062002F033FF000602
:10BAC00068D4BDF80C00BDF80010401C8142EBD1D9
:10BAD00003A90C2002F026FF00065BD46946012072
:10BAE00004F0D4FC000655D40622694603A830F0C1
:10BAF0002DFE10B10620276075E703A9112002F082
:10BB000011FF000646D46946022004F0BFFC00067F
:10BB100040D4062203A9684600E005E030F016FE96
:10BB200030B1082027605EE702F0B6FF0028BBD1E5
:10BB300006AD281D22F0A4FA00067BD406A822F048
:10BB4000D0FA000676D4E91D002004F09FFC000620
:10BB500070D40DF12B01012004F098FC000669D48B
:10BB60000DF13101022004F091FC000662D40EA90F
:10BB7000042004F08BFC00065CD4BDF83800ADF85E
:10BB8000420010A906A8F4F787FF11A9052002F0CA
:10BB9000C9FE00E04EE000064CD44FF00040F9F73B
:10BBA000CBFC000646D406F02AF8000639D49DF8EE
:10BBB0003C00000704D406A802F07CFF000630D445
:10BBC000012188F8001003F0F8F9000629D4204D6F
:10BBD00001211F4806F02FF800060AD5F4F71AFBDA
:10BBE00002F06CFC00061CD4F4F729FB2078000658
:10BBF00017D403F01EFA000613D495F8400000286D
:10BC0000E6D1112004F04BFE00060AD410A9012051
:10BC100004F055FE000604D4122004F040FE000695
:10BC200004D505F082FBF9F782FDA3E6F9F7EAFCFB
:10BC3000000601D520689DE688F80090012005F0F7
:10BC400071FF97E60CC0072014C0072010C0072022
:10BC500008C707202DE9F0438BB007A9012021F088
:10BC6000E9FC594C000645D4684602F0C2FD0006C6
:10BC700040D408A9032004F009FC544DDFF850819A
:10BC8000000616D40027052208A903A830F05EFD9F
:10BC900080B142200EF04BFE00062BD49220206093
:10BCA0003120794628609220C8F800100BB0BDE81A
:10BCB000F08301279DF811004FF0000641074FF077
:10BCC000870903D4C4F800902E606DE0400654D577
:10BCD00006A8F9F79DFE000674D49DF818000E28FA
:10BCE00001D0002FEED060200EF021FE000602D51C
:10BCF00005F01BFB66E002F0CFFE000662D468464A
:10BD000000F03FF900065DD40DF1020000F01DF9CE
:10BD1000000657D41E208DF80400684602F036FF56
:10BD200000064FD48DF800606846F9F756FE00060D
:10BD300048D4684602F0DFFC000643D4BDF800009A
:10BD4000401E80B203F006F900063BD4214D0121CC
:10BD5000204805F070FF000606D5F4F75BFA02F004
:10BD6000ADFBF4F76CFA2DE003F063F9000629D47B
:10BD700095F840000028EAD11BE00798C00707D0DB
:10BD80008DF800606846F9F728FE00061AD410E026
:10BD90006846F9F72CFE000614D49DF8000040B167
:10BDA0000420C4F80090286079468720C8F8001065
:10BDB0007CE733200EF0BBFD000603D402F059FFF0
:10BDC000000695D4206871E70CC0072010C007203A
:10BDD00014C0072008C7072038B54FF00040F9F716
:10BDE000ABFB104D000617D400248DF800406846C8
:10BDF000F9F76CFF000606D48DF800406846F9F7A5
:10BE000044FE000602D5F9F792FC38BD684600945E
:10BE1000F9F76DFF000601D5286838BDF9F7F2FB88
:10BE200038BD00000CC007201CB54FF00040F9F7EA
:10BE300083FB000602D51D4800681CBD01A8FAF767
:10BE4000CDF800062CD46846F9F73AFE000627D450
:10BE50006846F9F72DFA000622D46846F9F726FE5F
:10BE600000061DD46846F9F73CFE000618D4684663
:10BE7000F9F7F7F9000613D46846F9F728FE00062B
:10BE80000ED400248DF8044001A8FAF79DF80006AE
:10BE900006D48DF800406846F9F7F7FD000602D594
:10BEA000F9F745FC1CBDF9F7ADFB1CBD0CC0072024
:10BEB0002DE9FC5F9B4D9C4E9C4C894607004FF042
:10BEC00086084FF0140A03D048F6AD60874204D9C3
:10BED000C4F80080C5F800A008E04FF0170BB9F5D2
:10BEE000B46F08D3C4F80080C5F800B0784630605D
:10BEF0008620BDE8FC9F01A8FAF768FA00060BD47B
:10BF0000BDF804003F1A4FF4B4604743E0D46846DC
:10BF1000FAF76CFA000601D52068EAE7BDF80010D0
:10BF2000A9EB0100C019DDD40021B0F5B46F06DB28
:10BF30008A2020607846296030608A20D9E7216015
:10BF40007846296030600020D3E738B5044668465B
:10BF500022F096F80106754801D5006838BD9DF8B5
:10BF600000209DF80110C2EB021201EB820121803A
:10BF7000002101606B48016078466B490860002031
:10BF800038BD38B50446684622F0ABF8000602D545
:10BF90006648006838BD21466846F4F77DFD38BD27
:10BFA0007CB50025ADF800506846FFF7CEFF5F4C2A
:10BFB000000604D401A8FFF7E4FF000601D52068BD
:10BFC0007CBDBDF80010BDF80400FFF771FF5549B6
:10BFD000554A38B19120206088200860784610606A
:10BFE00091207CBD256078460D60106000207CBDEE
:10BFF0002DE9FE43DFF8388181464A4E98F800006B
:10C00000494F4A4C002510B188F8005062E069465B
:10C010003D200FF02CFD000651D49DF80000E8B340
:10C02000012188F8001001A8FFF78FFF000646D411
:10C0300002A8FFF7A6FF000641D4BDF80800BDF82E
:10C040000410C0EB001000EB400001EB401801A809
:10C05000FAF79FFB000632D402A8FAF789FB000624
:10C060002DD4BDF80800BDF80410C0EB001000EBA3
:10C07000400001EB40109DF80010C1EB011100EBF6
:10C080008101414526D8B9F1000F1BD062200EF086
:10C090004EFC000613D46946532000E01AE00FF06E
:10C0A0001BFC00060BD49DF8000010F002008DF878
:10C0B000000007D0012005F035FD000602D52068FC
:10C0C000BDE8FE8387202060052030607846386018
:10C0D0008720F5E725607846356038600020EFE777
:10C0E0001CB56846FFF731FF104C00060ED401A8BE
:10C0F000FFF747FF000609D401A8FAF72FFB000657
:10C1000004D46846FAF73BFB000601D520681CBD45
:10C110000449002020600860784603490860002038
:10C120001CBD000010C0072014C007200CC0072051
:10C1300068C1072010B5044690B04FF00040F9F7F1
:10C14000FBF9000603D53648006810B010BD201D6D
:10C15000FAF725FA000617D404F10800FAF730FAC6
:10C16000000611D4207A0FA9FAF748FA00060BD47A
:10C17000211D0FA8F8F78FFE000605D4207A0FA91D
:10C18000FAF72FFA000602D5F9F7D1FADDE70EA982
:10C190004B200FF0A1FB00063CD49DF83800C007EF
:10C1A00003D005F078FC000634D413208DF801008C
:10C1B000207A8DF802006068CDF803009DF8380001
:10C1C000800704D5684603F0C1FC000622D49DF820
:10C1D0003800C00704D0684604F01EFE000619D4DB
:10C1E000F9F7F7F9000615D49DF83800800704D553
:10C1F000684603F0D6FC00060CD49DF83800C00752
:10C2000004D0684604F033FE000603D4F9F7EDF9D4
:10C21000000602D505F089F8B6E7F9F7F3F994E7D7
:10C220000CC0072010B5044690B04FF00040F9F75D
:10C2300083F9000603D53648006810B010BD201DF4
:10C24000FAF7ADF9000617D404F10800FAF7B8F9C7
:10C25000000611D4207A0FA9FAF7D0F900060BD402
:10C26000211D0FA8F8F738FE000605D4207A0FA983
:10C27000FAF7B7F9000602D5F9F759FADDE70EA982
:10C280004B200FF029FB00063CD49DF83800C00776
:10C2900003D005F020FC000634D414208DF80100F2
:10C2A000207A8DF802006068CDF803009DF8380010
:10C2B000800704D5684603F049FC000622D49DF8A7
:10C2C0003800C00704D0684604F0A6FD000619D463
:10C2D000F9F77FF9000615D49DF83800800704D5DA
:10C2E000684603F05EFC00060CD49DF83800C007D9
:10C2F00004D0684604F0BBFD000603D4F9F775F9D5
:10C30000000602D505F011F8B6E7F9F77BF994E7D6
:10C310000CC0072070B594B0002604468DF8446028
:10C320004079B74DA0B111A8F9F76AFD000674D4A1
:10C330009DF8440008B110280AD98620B149286028
:10C34000032008607846B0490860862014B070BDAC
:10C350004FF00040F9F7F0F80006E8D460790028C3
:10C3600075D06846F9F7CDFC00066CD4A07921465B
:10C370000028684652D0F8F7AFFD000663D468463F
:10C38000F9F7B5FC00065ED469469DF84400F9F75C
:10C39000EDFC000657D4A07921460028684640D01D
:10C3A000F8F79AFD00064ED469469DF84400F9F767
:10C3B000D1FC000647D411A8F9F78FFD000642D43E
:10C3C0002046F9F779FD00063DD420796946FAF751
:10C3D00069F900067FD421466846F8F75CFD00063F
:10C3E00079D420796946FAF750F9000673D4A07918
:10C3F0000028684618D0F9F79DFE00066BD4214648
:10C400006846F8F748FD000665D46846F9F789FEE6
:10C41000000660D405F055F973E0BFE0F8F73BFD86
:10C42000ABE7F8F738FDBDE7F9F7AAFE000652D4EE
:10C4300021466846F8F72FFD00064CD46846F9F708
:10C4400095FEE5E703E046E004F06FFF43E010A847
:10C45000F9F757FC00063ED410A8F9F782FD000654
:10C4600039D410980090A07921460028684635D02C
:10C47000F8F732FD00062ED46846F9F738FC0006BE
:10C4800029D42046F9F75CFD000624D4A0790028C1
:10C49000684626D0F9F792FC00061CD4214668466F
:10C4A000F8F7F9FC000616D46846F9F77DFC00069B
:10C4B00011D420796946FAF7F5F800060BD4214625
:10C4C0006846F8F7E8FC000605D420796946FAF7D3
:10C4D000DCF8000613D5F9F72AF937E7F8F7DBFCA3
:10C4E000C8E7F9F77CFC0006F5D421466846F8F762
:10C4F000D2FC0006EFD46846F9F767FCD7E705F0F1
:10C5000000F90006A0D4A079A8B108208DF8050094
:10C5100020798DF80A00617901A871B1CDF8066023
:10C52000C01DF9F7B1FC00068ED46846F9F7BDFCD2
:10C53000000689D40EE00720E8E71099CDF8061030
:10C54000C01DF9F7E5FC000628D46846F9F7F1FCB0
:10C55000000623D4BDF80000ADF80C002068CDF82B
:10C560000E000FA94C200FF0B7F9000616D49DF865
:10C570003C00800704D501A803F0E8FA0006C1D406
:10C580009DF83C00C00704D001A804F045FC00065B
:10C59000B8D46846FAF795FA000601D52868D5E6BA
:10C5A0009DF8000060B11948007848B120681290E9
:10C5B000A079002812A820D002F018FE0006A1D40D
:10C5C000F9F707F800069DD49DF83C00800704D5D4
:10C5D00001A803F0E6FA000694D49DF83C00C007D9
:10C5E00004D001A804F043FC00068BD4F8F7F1FF57
:10C5F000000687D4F9F706F8A8E602F04EFEDDE75C
:10C600000CC0072010C0072014C007201C04000025
:10C6100071B581B04FF00040F8F78EFF7A4C0006FC
:10C620003CD403208DF800006846F9F72EFA000686
:10C6300062D419208DF800006846F9F71BFF000648
:10C640005AD472490220087001A91920F9F723FF72
:10C65000000623D4012005F065FA00064CD403F04F
:10C6600056FC000648D4BDF8040003F0B6FB0006F3
:10C6700042D420680025052807D0654E03F094FCBD
:10C68000000639D42068D8B913E0F9F750F800064D
:10C6900004D401202AF0BAF8000601D520687CBD38
:10C6A000812020605B48056078465B4908608120F6
:10C6B0007CBD7078062803D0052801D00B28DDD179
:10C6C0002AF049FB000617D401202AF09FF8000643
:10C6D00012D4012005F026FA00060DD48DF8005082
:10C6E0006846F9F7D2F9000606D48DF8005068467E
:10C6F000F9F7C0FE000602D5F9F719F87CBDF8F786
:10C7000081FF7CBD2DE9F843064689464FF0004085
:10C71000F8F712FF3C4C00066CD496B103208DF85C
:10C7200000006846F9F7B1F9000622D419208DF807
:10C7300000006846F9F79EFE00061AD4334902202D
:10C7400008706846F9F7CDF9000653D469461920F8
:10C75000F9F7A1FE00064DD4012005F0E3F900062B
:10C7600007D404F09CFC000603D404F0AAFC0006E5
:10C7700003D5F8F7DCFFBDE8F8832068254FDFF824
:10C780009880002505280FD1F8F7D1FF000631D495
:10C7900001202AF03BF800062CD481202060794645
:10C7A0003D60C8F80010E6E704F0D0FC000606D4AF
:10C7B00020680028F8D02AF0CEFA000602D504F04E
:10C7C000B4FDD6E7F8F71EFF000613D4A6B148461D
:10C7D00005F0A8F900060DD48DF800506846F9F769
:10C7E00054F9000606D48DF800506846F9F742FE69
:10C7F000000601D52068BEE7256079463D6000202F
:10C80000C8F80010B7E700000CC0072000C00720E0
:10C81000A0C8072010C0072014C007202DE9FC4144
:10C820002F4C90460F460026C0B3FAF71AF940B1D4
:10C83000F3F7F0FC00212BA02AF0E7F8F3F7FFFC58
:10C8400043E08DF800606846F9F7B8F86846F9F7F4
:10C85000C4F802208DF800006846F9F7F1F80006E8
:10C8600033D46846F9F7DBF800062ED46846F9F7AA
:10C87000C5F8000629D40120ADF80400054601A939
:10C880002846F9F708FE00061FD46D1C1B2DF6D9AB
:10C8900003F0A0F8FEF732FC000616D4C7B14046FC
:10C8A0000FF0D4FC000610D400200EF0CAFF0006E2
:10C8B0000BD40EF00DF920B900200EF069FB000634
:10C8C00003D4F4F7FEFB000602D52068BDE8FC8126
:10C8D0000B482660066078460A4908600020F5E7A4
:10C8E0000CC007208EE8A8A1AAA020A8ADA8E6A8A1
:10C8F000A0ABA8A7A0E6A8A8208E87930A000000F6
:10C9000010C0072014C007202DE9F0418AB0BB48B1
:10C91000F8F75BFBBA48F8F758FB06A8FAF7D1F826
:10C92000B84C000652D49DF818000527B64EDFF823
:10C93000DC82002510B307A912200EF0CDFF0006FF
:10C9400044D408A92E200EF0C7FF00063ED405A847
:10C95000F9F79AFD000639D49DF81C10C80705D0D8
:10C960009DF814000E2812D0142810D09DF8140041
:10C970000F2803D19DF82000800708D4276079464E
:10C9800035600520C8F800100AB0BDE8F081A04F5E
:10C99000880715D5002003F05AFD000616D4694615
:10C9A000002003F018FD000610D4BDF8021002208C
:10C9B00003F037FD000609D4BDF80200788008E0D6
:10C9C0000021022003F02DFD000601D52068DBE7E1
:10C9D0007D803D702560794635600020C8F80010E4
:10C9E000D2E72DE9F04F89B04FF00005854CDFF814
:10C9F0001C82854F06008DF814504FF0050B04D0B3
:10CA0000012E02D0022870D09DE0DFF804A24FF082
:10CA100000096946022003F0DEFC20B1052830D071
:10CA200093287DD152E09AF8000060B1BAF8021064
:10CA3000BDF80220481C824211D0022003F0F1FC14
:10CA4000000674D44AE001218AF80010BAF80210F6
:10CA5000BDF802204B1C9A42EFD1AAF80220684888
:10CA600001A9F8F754FB000661D464480DF10901EF
:10CA7000F8F74DFB00065AD4BDF80210AAF80210D0
:10CA80002CE0012E1FD105A8F8F7B1FF00064ED407
:10CA90009DF81400B8B106A90120F9F7B3FA000611
:10CAA00045D406A95648F8F732FB00063FD406A93C
:10CAB0000220F9F7A7FA000639D406A94F48F8F77B
:10CAC00026FB000633D48AF8005034E0BAF802108E
:10CAD000491CAAF802103868082828D109F1010970
:10CAE000B9F1640F95DB2EE0FFE705A8F8F77FFFAB
:10CAF00000061CD49DF81400E8B106A90120F9F73E
:10CB000081FA000613D406A93D48F8F700FB000699
:10CB10000DD406A90220F9F775FA000607D400E043
:10CB200005E006A93548F8F7F2FA00060BD52068AB
:10CB300009B0BDE8F08FC4F800B079463D6005202B
:10CB4000C8F80010F4E7256079463D600020C8F879
:10CB50000010EDE72DE9F04F83468DB08A46084678
:10CB6000F8F733FA5846F8F730FA0AA8F9F7A9FFA8
:10CB7000244C000630D49DF82800DFF89080224F26
:10CB8000002578B3002003F062FC000624D4694637
:10CB9000002003F020FC00061ED4BDF80210022085
:10CBA00003F03FFC000617D405AE0DF11D0905A9E1
:10CBB000022003F010FC206810B193280FD015E07C
:10CBC000311D5846F8F7A3FA000605D449465046E9
:10CBD000F8F79DFA000606D520680DB0A9E7386879
:10CBE0000828E4D002E020680528E0D125607946D5
:10CBF0003D600020C8F80010EFE70000A7C1072043
:10CC0000A0C107200CC0072010C0072014C00720B7
:10CC10006AC107202DE9F84F054600794C4C4D4F6D
:10CC2000DFF83481862608B11E2802D90520266047
:10CC30004AE0288848F6AD614FF0140A884203D9CB
:10CC40002660C7F800A040E068884FF0170BB0F5E9
:10CC5000B46F03D32660C7F800B036E06846F9F732
:10CC6000B5FB000667D42888BDF80010401A4FF4C1
:10CC7000B46148435FEA0009E2D46846F9F7B6FBBD
:10CC8000000658D46888BDF80010411A11EB090F4E
:10CC9000E0D432490120F9F7B5F900064BD4304908
:10CCA0000220F9F7AFF9000645D468790F380D284E
:10CCB00008D2DFE800F0101010101007101010104C
:10CCC0000710100008202660386079468620C8F8D2
:10CCD0000010BDE8F88F2846F8F71BFF00062AD49D
:10CCE000A81CF8F727FF000625D4281DF8F733FF06
:10CCF000000620D4681DF9F7BDFB00061BD40025F3
:10CD000068460095F9F704FC000614D468460095BF
:10CD1000F9F70DFC00060ED40120ADF800006846BE
:10CD2000F9F7CFFB000606D4ADF800506846F9F7D6
:10CD3000D9FB000601D52068CBE7032009498DF80F
:10CD40000000022008706846F8F79FFEC1E7000067
:10CD50000CC0072010C0072014C0072078C107208E
:10CD60007DC1072000C007202DE9F04F91B005A834
:10CD7000F9F78AFBFA4C00067ED46846F9F7ABFB5C
:10CD80000006F9D4DFF8DCA34FF010014FF00209E0
:10CD90009AF800004FF0000802074FF0010734D561
:10CDA0009DF81400A0F10E020E2A6DD2DFE802F009
:10CDB00007070F0F0F1C076C6C6C6C6C6C0F8AF8FC
:10CDC00002008DF8141009E0ADF800905CE0BDF8A9
:10CDD0000010032958D1401C8DF8140005A8F9F75C
:10CDE00049FB0006C8D4EFE7BDF8000003284BD18B
:10CDF0009AF802008DF81400554605A8F9F73AFB99
:10CE00000006B9D4ADF800903CE0554640063BD54D
:10CE10009DF814000E2804D00F2802D0102833D11A
:10CE200015E0BDF80020042A2ED18AF802008DF802
:10CE3000141005A8F9F71EFB00069DD41420ADF8C8
:10CE400000006846F9F73DFB000695D41CE0BDF8EC
:10CE50000000032818D1ADF800706846F9F742FBCE
:10CE6000A8788DF8140005A8F9F704FB000688D40B
:10CE70000420ADF8000000E05DE26846F9F721FB10
:10CE80000006AFD485F800809DF81420B64DB74E4B
:10CE900088214FF0640B4FF010401C2A72D2DFE85B
:10CEA00012F07100BB046406640664066406420660
:10CEB00042064206420642064206420642061C005E
:10CEC0001C000E031604AB0382040C059F069F068C
:10CED0009F069F067100A304C102BDF800200A2A24
:10CEE0007BD007DCDAD2DFE802F04D1A51F29CBEAB
:10CEF000D4E3F4FADFF878B25A2A67D008DC0B2AB8
:10CF00007ED00C2A7DD0392A7CD0402A3AD117E233
:10CF10005B2A78D0642A77D0B42AF7D124E09149EB
:10CF200012200EF0D9FC000687D49AF800100120D8
:10CF300001F048018AF8001004F0F4FD000684D4E2
:10CF40009DF814000E280DD1694662200EF0C4FC35
:10CF500000068CD49DF80000C00703D0F3F778FFDB
:10CF6000000684D4B4202DE07E496920491C0EF0CF
:10CF7000B3FC000685D49AF80100000603D504F03E
:10CF800081FE60E2D5E2ADF80090F7E004F07DFEAE
:10CF90000006C9D40EA92E200EF09EFC0006C3D4B4
:10CFA0009DF814000E2805D00F2810D19DF83800E8
:10CFB00080070CD5FFF7A8FC0006B5D4206805282B
:10CFC00005D00A20ADF80000D8E006E000E104201A
:10CFD00041E200BFADF80070F5E30020FFF701FD6E
:10CFE0000006A1D42068002872D00EA92E200EF0D1
:10CFF00073FC000698D49DF814000E280BD004E0B2
:10D0000083E05CE0D5E033E1BEE00F28DFD19DF89E
:10D0100038008007DBD56B200DF089FC00068ED42C
:10D02000D5E70FA969200EF022FD000687D49DF8F0
:10D030003C00C00603D404F0AAFE000689D468466A
:10D04000F9F75AFA000684D4BDF80000042801D28A
:10D05000401CF4E3ADF800706846F9F743FA0006A7
:10D0600088D40520AEE704F08FFE000691D4684610
:10D07000F9F742FA00068CD4BDF800000228E7D385
:10D08000ADF800706846F9F72DFA000687D406203F
:10D0900098E704F082FE00068FD46846F9F72CFA70
:10D0A00000068AD4BDF800000428D1D3072089E700
:10D0B0001B200DF03CFC000693D40C2082E704F00A
:10D0C00060FE00068DD408207CE708E001E020E047
:10D0D00057E004F053FE00068CD4092072E704F0F8
:10D0E0004AFE000686D40EA92E200EF0F5FB00069F
:10D0F00095D49DF814000E2805D00F287ED19DF8F8
:10D10000380080077AD50B205CE70220FFF769FC26
:10D110006FE204F0C3FD000688D40EA92E200EF0A5
:10D12000DBFB00068AD49DF814000E2805D00F28DA
:10D130007DD19DF83800800779D50E4D01206F8193
:10D1400029F0F4F900068BD456200DF0F0FB000610
:10D1500086D4A5F80A90022029F0E8F9F3E300004C
:10D160000CC0072070C1072010C0072014C0072082
:10D170000000094000DD0720ADF800B06846F9F76F
:10D18000A0F911B0BDE8F08F29F0B6FD000688D4F3
:10D190002068052804D09DF814000E2807D079E1F6
:10D1A000C4F800807846C5F8008030602FE35A202C
:10D1B00008E7F8F7C1F9000684D4FDF717FD00066B
:10D1C0007ED4F8F71FFA75E32760C5F8008025E1E3
:10D1D0006846F9F776FC000684D49DF8000038B361
:10D1E000FD484FF05B09007800283FF4CCAE68465C
:10D1F000F8F71FFC00068FD4F84800E066E20078DC
:10D20000D8B19DF800001B2817D06846F9F709F936
:10D21000000687D46F46B81CF9F714F9000692D4BB
:10D22000381DF9F720F900068DD4684601E079E34E
:10D230007BE001F0ABFC000685D46946042003F0D6
:10D2400025F9000684D4BDF80000401C80B201F02E
:10D2500081FE50B192286ED1F2F7DCFF13208DF8D9
:10D2600000006846F8F7DBFBF7E3ADF80090FEE25C
:10D27000D948007828B30121D94804F0DCFC000625
:10D2800085D401F0D6FE000696D4D54890F840002B
:10D29000002885D16846F8F7CCFB00068CD49DF8B1
:10D2A00000000E283DD06846F9F7BBF8000693D47D
:10D2B000DAF8081001919AF80C108DF8081001E0C6
:10D2C000F2E039E0DAF80D10CDF809109AF8110003
:10D2D0008DF80D0004200DF1020103F0D7F80006CF
:10D2E00089D4BDF80200401CADF80200112003F003
:10D2F000D6FA00068DD46946022003F0E0FA000653
:10D3000087D4122003F0CBFA000688D4022003F061
:10D310009EF8000688D46946022003F05CF80006F7
:10D320008AD4FEF7DDFE000686D4DBF80810402024
:10D33000CAF8041046E683E2A94981F84080A9E7CB
:10D34000DBF80810DAF80400081AA649884203D26C
:10D35000A548007801289CD1C1468DF80080684618
:10D36000F8F73BFB00068BD4B84638460DF11C0B92
:10D37000C7B269463846F8F745FE000684D4C7EBC5
:10D38000C70101EB0B0AAAF107013846F8F70EFBBB
:10D3900000068CD4AAF107006946F7F7B8FE00062C
:10D3A00085D47F1CF8B20428E2D907A8F8F7F4FA6C
:10D3B000000695D406A8F9F784FB000690D49DF8E2
:10D3C000180018B9F9F799FB000689D469461220AC
:10D3D0000EF082FA00068DD49DF8000040070AD5B1
:10D3E0006846F7F7F2FD000684D469460120F8F795
:10D3F00038FB000684D4694662200EF06DFA000600
:10D4000088D49DF80000C00704D00020F3F736FD53
:10D41000000685D4C4F80080C5F8009078463060D6
:10D420000120AEE6BDF80020392A35D006DC012AFD
:10D430007ED0022A0AD0032A7BD123E0642A61D05D
:10D44000822AF9D10FE000068DD49CE504F01DFC82
:10D45000000688D48220ADF800006846F9F731F85C
:10D4600000068BD4B6E504F095FC000686D4684629
:10D47000F9F742F800068CD4BDF800000428FFF448
:10D48000E7ADFDE304F00AFC000689D429F017FC9F
:10D49000000685D4392095E5F8F74EF8000688D4C3
:10D4A000FDF7A4FB00067DD5F8F741F969E6000613
:10D4B00084D461E6206805287FF486AE70E6BDF866
:10D4C0000020172A79D011DC142A1CD009DC012A8B
:10D4D000AED0022AAFD104F0D8FB000684D41420C9
:10D4E000B9E7152A4AD0162AA6D12BE01B2A3FD02D
:10D4F0007CDC182A5BD0192A1ED01A2A9CD176E02F
:10D50000642A99D1C1E304F02AFC00069CD4684641
:10D51000F8F7F2FF000697D4BDF800001028AED34C
:10D52000ADF800706846F8F7DDFF00068CD401E026
:10D53000DBE0DBE0192045E504F005FC000688D4BB
:10D5400016203FE504F011FC00068AD46846F8F77F
:10D55000D3FF000685D4BDF8000010288FD3ADF8A6
:10D5600000706846F8F7BEFF000684D41B2029E54A
:10D5700004F0EFFB000688D4152023E504F0F2FB4D
:10D58000000686D46846F8F7B7FF000687D4BDF8D2
:10D5900000001028C3D3ADF800706846F8F7A2FF6A
:10D5A000000601E035E108E082D418200AE504F025
:10D5B000CDFB000692D4172004E504F0D9FB000649
:10D5C0008CD46846F8F798FF000687D4BDF80000B1
:10D5D0001028A4D31A20F5E41C04000082C10720FF
:10D5E00008C7072040420F00CAC307207FE004F0AD
:10D5F000B3FB00068AD443E3BDF800201F2A42D0C3
:10D6000009DC012A71D0022A0AD0032A3FF415AF9F
:10D610001E2A6BD10AE0202A1FD0212A67D148E0B8
:10D6200004F033FB00068AD41E2014E704F07FFBCD
:10D63000000684D46846F8F75FFF000685D4BDF87D
:10D64000000018287FF604ADADF800706846F8F7C2
:10D6500049FF000689D42020B4E404F06EFB0006E4
:10D6600089D46846F8F748FF000684D4BDF8000066
:10D670001828E7D9ADF800706846F8F733FF0006C0
:10D6800084D41F209EE404F055FB00068CD4684629
:10D69000F8F732FF000687D4BDF800001828D1D96A
:10D6A000ADF800706846F8F71DFF000688D4212009
:10D6B00088E404F045FB000687D46846F8F71CFFB1
:10D6C000000697D4BDF800001828BBD9D8E2BDF8F1
:10D6D0000020292A43D00BDC012A06D0022A0CD0D4
:10D6E000032A93D0282A01D10DE0E0E019E16BE094
:10D6F0002A2A1ED02B2A67D147E004F0C6FA00067A
:10D7000091D42820A7E604F006FB00068BD46846D7
:10D71000F8F7F2FE000686D4BDF800001E2891D965
:10D72000ADF800706846F8F7DDFE000686D42A20C2
:10D7300048E404F0F6FA00068CD46846F8F7DCFEFC
:10D74000000687D4BDF800001E2892D9ADF80070FD
:10D750006846F8F7C7FE000672D4292032E404F0C8
:10D76000DDFA00066CD46846F8F7C6FE000667D4FA
:10D77000BDF800001E2892D9ADF800706846F8F791
:10D78000B1FE00065CD42B201CE404F0CDFA0006A8
:10D7900056D46846F8F7B0FE000651D4BDF8000034
:10D7A0001E2892D96CE2BDF80020372A0DD02ADC61
:10D7B000012A7CD0022A7FF43EAE04F066FA00060D
:10D7C0003ED4372047E68DE11DE004F0A1FA0006C3
:10D7D00036D46846F8F790FE000631D4BDF8000054
:10D7E0002028FFF435AC4BE2BDF80020382A0ED0DB
:10D7F00009DC012A5BD0022ADDD104F046FA0006DA
:10D800001ED438202EE4392A7FF47AAE44E6002074
:10D81000B7E4F7F7F7FE4AE6BDF800003E2816D059
:10D8200006DC012843D002280BD0032879D13FE041
:10D830003F2877D0402827D0642872D10DE04FE1EF
:10D8400071E004F022FA00066DD43E200AE404F0F0
:10D85000A7FA000667D43F2004E429F04DFA000639
:10D8600061D4206805283FF429AE402081E0684655
:10D87000F8F727FE000656D4042020607846C5F845
:10D880000080306004207CE4FDF738FC00064AD4B8
:10D890000327ADF800706846F8F713FE000642D47F
:10D8A00027607846C5F800803060032069E443E1D2
:10D8B00004F0F4F9000636D486E4BDF80000092827
:10D8C00052D00FDC2DD2DFE800F02C1F2FF93F0BD8
:10D8D00009070500FFF7FDBBFFF7EABBFFF7D9BB60
:10D8E000FFF7C1BB52287DD007DC0C283FF4E7AB23
:10D8F000502841D0512814D197E0532873D0542890
:10D9000072D064280DD1C0E1E34912200DF0E4FF8C
:10D91000000608D49AF8001001F008018AF80010F7
:10D920000AE172E159E17FE08AF8008004F0ADF984
:10D93000000679D4ADF800706846F8F7D3FD00060C
:10D9400072D4042034E446E104F021FA00066BD4DA
:10D950006846F8F7D1FD000666D4BDF8000004283B
:10D96000FFF476AB052076E504F005FA00065BD4FB
:10D970005020ADF800007AE76846F8F75AF800063C
:10D9800052D49DF800000E2833D06846F8F749FDC0
:10D99000000649D4DAF8081001919AF80C108DF8B5
:10D9A0000810DAF80D10CDF809109AF811008DF86A
:10D9B0000D0004200DF1020102F068FD000633D4D1
:10D9C000BDF80200401CADF80200112002F067FF14
:10D9D000000629D46946022002F071FF000623D414
:10D9E000122002E03AE051E069E002F058FF000640
:10D9F0001AD4694612200DF06FFF000614D49DF86A
:10DA0000000040070AD56846F7F7DFFA00060BD496
:10DA100069460120F8F725F8000605D4FDF714FC47
:10DA2000000601D4512016E57CE06846F8F764FD55
:10DA3000000677D4BDF80000C0B20546FDF7ACFC87
:10DA400000066FD4102D49D3ADF800706846F8F782
:10DA500049FD000666D452206CE4FBE06846F8F706
:10DA60004BFD00065ED4BDF80000C5B22846FDF7A8
:10DA7000C7FC000656D40A2D30D3ADF800706846B6
:10DA8000F8F730FD00064DD4532053E46846F8F70C
:10DA900033FD000646D4BDF80000C0B20546FDF7D0
:10DAA00055FC00063ED41E2D18D3ADF80070684614
:10DAB000F8F718FD000635D454203BE424E068460E
:10DAC000F8F71AFD00062DD4BDF80000C5B22846AF
:10DAD000FDF716FC000625D4182D07D26D1CE8B200
:10DAE000ADF800006846F8F7FDFC9AE48DF8008078
:10DAF0006846F7F772FF000614D4FEF7F1FA000645
:10DB000010D4FEF701FF74E50120FEF76AFF00065E
:10DB100008D420680028E8D004F0C0F8000601D43A
:10DB2000FFF70BBB7FE0BDF80000012804D00228FE
:10DB300006D0632869D109E0012003F0F3FF82E4F5
:10DB400004F0A3F800066ED46320A4E4534890F8D0
:10DB5000400000283FF4B0AE0221504804F06BF8BA
:10DB6000000660D401F065FA5BE4BDF800005C28B3
:10DB700029D006DC012812D002281ED0032844D167
:10DB80003CE05D2812D05E287FF4BBAE44480078AC
:10DB900000283FF45AAC3C200CF0C9FE53E40120AD
:10DBA00003F0C0FF000675D45D2074E43B200CF048
:10DBB000BEFE00066ED45E206DE404F066F800063A
:10DBC00068D45C2067E402F0F5FD000662D42068AA
:10DBD000052855D072E400065CD429F070F866E49C
:10DBE000BDF8000079281FD00BDC012814D00328D1
:10DBF000CAD1012028F00AFE00064BD404F04EF8EA
:10DC0000E9E77A281BD07B282DD021607846C5F81B
:10DC100000903060882004E4012003F083FF0006B8
:10DC200038D4792037E417E05D200CF080FE000640
:10DC300030D402F06CF900062CD47A202BE402F0E8
:10DC4000B3F90028C6D0052807D0F2F7E3FA01207F
:10DC500028F0DCFDF2F7F3FA1CE029F030F80006BA
:10DC600018D47B2017E429F047F8000612D4206866
:10DC70000528AFD09DF81400172803D0182801D02C
:10DC8000032008E401F066FEB3E429F035F800064D
:10DC90007FF510AC206809E470C1072008C7072091
:10DCA0001C0400003EB54FF00040F7F745FC2B4C3C
:10DCB000000609D401A8F8F7E7FB000647D4684638
:10DCC000F8F72FFC000601D520683EBD009800063D
:10DCD0002ED49DF804000E2808D10120ADF80800CC
:10DCE00002A91A20F8F7D7FB000630D46846F7F7E8
:10DCF000E7FE00062BD46846F7F7DAFA000626D4CA
:10DD00006846F7F7D3FE000621D469469DF8040063
:10DD1000F8F7CEFB00061AD46846F7F7A2FA000619
:10DD200015D469469DF80400F8F7B5FB00060ED43B
:10DD300000248DF800406846F8F79CFB000606D4E6
:10DD40008DF800406846F7F7A0FE000602D5F7F709
:10DD5000EEFC3EBDF7F756FC3EBD00000CC00720B0
:10DD60002DE9F04F05460079D84CD94FD94E93B0E4
:10DD70004FF0860808B11E2804D90520C4F8008099
:10DD8000306017E0288848F6AD614FF0140B8842E8
:10DD900005D900BFC4F80080C6F800B00AE0688862
:10DDA0004FF0170AB0F5B46F0AD300BFC4F8008073
:10DDB000C6F800A078463860862013B0BDE8F08F22
:10DDC00008A8F8F703FB00067CD42888BDF82010CB
:10DDD000401A4FF4B46148435FEA0009DAD408A856
:10DDE000F8F704FB0006EFD46888BDF82010411A4C
:10DDF00011EB090FDAD4B8494FF0000A012081F87D
:10DE000000A0B649F8F7FEF80006DDD4B4490220B8
:10DE1000F8F7F8F80006D7D4052002F0B4FB0006A6
:10DE2000D2D408A8F8F74DFE0006CDD49DF8200006
:10DE30004FF0010B00287DD0AA4800780028FAD0C6
:10DE400000F0FCFE0BA9052000F06CFD0006BBD421
:10DE50000FA9032002F01AFB0006B5D405220FA972
:10DE60000BA82EF073FC78B142200CF060FD000688
:10DE7000AAD4012003F056FE9220206031203060A9
:10DE800078463860922098E700F006FE00069BD4A2
:10DE900090480068232809D13F200CF048FD000677
:10DEA00092D49148018821F0020101800BA9002041
:10DEB00000F038FD000687D49DF82C00400602D5FE
:10DEC000012001E0A3E00020804608A9042002F020
:10DED000DDFA000687D40BA9062000F023FD00061A
:10DEE00093D4BDF82000BDF82C60401C864201D1BF
:10DEF000012000E000208146B8F1000F13D1B9F1F4
:10DF0000000F10D1761EB6B209A9304601F026FBEB
:10DF100000067CD4BDF824002880BDF82600688067
:10DF20009DF82800287108A9042002F0AFFA000625
:10DF30006DD400E06EE0BDF82000401CB04212D06D
:10DF40004E200CF0F4FC000661D4012003F0EAFD41
:10DF500000065CD48F2020605E480721016078466F
:10DF600038608F2029E701A9304601F057FA0006F2
:10DF70004DD48DF820A0012711A93846F8F742F8B2
:10DF8000000644D407EB870101A80144052211A82B
:10DF9000491F2EF0DBFB10B18DF820B005E07F1C8F
:10DFA000042FE9D99DF8200060B350480680452031
:10DFB0000CF0BDFC00067CD464200CF0B8FC00061C
:10DFC00077D4494801260DF10407018821F00201A8
:10DFD00001804248019901609DF808100171404894
:10DFE000DDF8091001609DF80D10017106EB860047
:10DFF000C1193046491FF7F7F8FF000659D4761CBF
:10E00000042EF3D958EA090004D0334900E050E067
:10E0100081F800B02846F7F77CFD000649D4A81C1B
:10E02000F7F788FD000644D4281DF7F794FD000695
:10E030003FD42846F8F7EBF900063AD4A81CF8F7C5
:10E04000F7F9000635D4281DF8F703FA000630D496
:10E05000681DF8F70FFA00062BD4554608A8CDF82E
:10E0600020A0F8F755FA000623D408A80895F8F779
:10E070005EFA00061DD4ADF820B008A8F8F721FA22
:10E08000000616D4ADF8205008A8F8F72BFA0006C1
:10E090000FD408A91C200DF01FFC000609D49DF820
:10E0A000200040B1ADF8205008A8F7F710FD000699
:10E0B00001D5206881E603200D498DF8200002205B
:10E0C000087008A8F7F7E1FC77E600000CC007200D
:10E0D00014C0072010C0072082C1072078C1072084
:10E0E0007DC107201C04000002C0072094C1072046
:10E0F00000C007202DE9F84306460D466846F8F7AC
:10E10000E0FC564C00067DD49DF800105448554A5A
:10E110004FF0000939B13179862309B11E290BD995
:10E120000521236019E087212160C0F8009078461E
:10E1300010600846BDE8F883318848F6AD674FF0B7
:10E140001408B94203D92360C0F8008006E0718842
:10E15000B1F5B46F06D317212360016078461060D3
:10E160008620E7E771790F46891F082969D2DFE821
:10E1700001F00404151523272B2FB5F800C069887A
:10E180008C4502D913212360E7E7072F04D0002232
:10E19000604600F094FE1DE00122F9E7B5F800C0EA
:10E1A00069888C45CFD8092F04D00022604600F042
:10E1B00029FE0FE00122F9E7288800F0BAFD09E006
:10E1C000286800F0EAFD05E0288800F0C3FE01E0C1
:10E1D00000F0F3FE000632D43046F7F79AFC000652
:10E1E0002DD4B01CF7F7A6FC000628D4301DF7F795
:10E1F000B2FC000623D4701DF8F73CF900061ED4CB
:10E200004D4600E01BE06846CDF80090F8F780F935
:10E21000000614D468460095F8F789F900060ED474
:10E220000120ADF800006846F8F74BF9000606D467
:10E23000ADF800506846F8F755F9000604D5206897
:10E2400078E70821236088E7032007498DF800005C
:10E25000022008706846F7F718FC6BE70CC007202F
:10E2600010C0072014C0072000C007202DE9F84384
:10E27000054688466846F8F724FC4D4C00067CD4D9
:10E280009DF800004B4E4C4F4FF0030928B12979FF
:10E290008620A9B1206005202CE04A200CF047FB25
:10E2A000000679D4012003F03DFC000674D48F20D1
:10E2B00020607846C6F8009038608F20BDE8F8836B
:10E2C000298848F6AD62914202D92060142011E0FD
:10E2D0006988B1F5B46F02D3206017200AE069792C
:10E2E00002290CD003290AD0042908D0052906D018
:10E2F000206008203060784638608620DEE740469F
:10E3000002F052F94FF0000898B1812844D14A2018
:10E310000CF00DFB00063FD4012003F003FC0006C7
:10E320003AD4812020607846C6F800803860812089
:10E33000C4E72846F7F7EDFB00062DD4A81CF7F735
:10E34000F9FB000628D4281DF7F705FC000623D4A6
:10E35000681DF8F78FF800061ED445466846CDF8CC
:10E360000080F8F7D5F8000616D468460095F8F74F
:10E37000DEF8000610D4012000E00DE0ADF800004A
:10E380006846F8F79EF8000606D4ADF800506846D7
:10E39000F8F7A8F8000601D520688FE707498DF83F
:10E3A0000090022008706846F7F76FFB86E70000D0
:10E3B0000CC0072010C0072014C0072000C0072091
:10E3C00070B5FA48002404704470C47001201FF036
:10E3D000E8FA0106F64801D5006870BDF54A916873
:10E3E00042F2107395686D1A9D42FBD30460F248A7
:10E3F00004607846F1490860002070BD2DE9F043C3
:10E400008DB0074639208DF82800EDA00024006863
:10E41000E74EDFF8A4830325A1460B908DF8245026
:10E4200009AB6A4602210BA81FF04FFAD8B1D8F801
:10E430000000052800D214B120280CD018E08DF877
:10E44000245009AB6A4601210AA81FF03EFA0006D3
:10E450000ED40124E2E708A9002000F063FA8DF849
:10E460002190002CDAD19DF82400022804D00BE082
:10E4700030680DB0BDE8F0839DF800008DF82000F5
:10E480009DF801008DF821009DF8200038709DF85E
:10E4900021007870CB489DF8201000F82A1F9DF8C5
:10E4A00021104170C14901208870C6F8009078465B
:10E4B000C249C8F8009008600020DAE71CB50620C1
:10E4C0008DF80000C0480178012059B1B7490022F9
:10E4D00001AB0A704A708DF80400012168461FF0F4
:10E4E000F4F91CBDB24A88211160B349086078462E
:10E4F000B249086088201CBD2DE9FC41054600207A
:10E5000005218DF80410B0498DF80000AA4E097855
:10E51000AA4FA74C89B1A549AA4A6B460870443A4C
:10E52000012101A81FF0D1F900060FD5F1F772FE05
:10E53000FFF7C4FFF1F783FE14E08820206001207C
:10E540003060784638608820BDE8FC8125B19DF8B0
:10E5500000006D1EA84207D19A499DF80000443979
:10E5600081F840002068EFE7922020602020306092
:10E57000784638609220E7E72DE9FF5F24208DF888
:10E58000080003A9002000F0CDF9894D00067DD4D4
:10E590009DF80C00884E894F00074FF0920804D474
:10E5A0002620C5F80080306046E0864A4FF0000B18
:10E5B0008DF804B001AB443A012102A81FF085F99F
:10E5C000000675D41920FFF797FF000670D47D4828
:10E5D0004FF0270944380178072902D0FFF76EFF72
:10E5E00026E0D0F801100167D0F805104167DFF888
:10E5F000D4A1D0F809100AF13C0A8167D0F80D20A7
:10E60000CAF80220427C8AF80620D0F81210C167AE
:10E61000C18A0446A0F880100F20FFF76DFF0006A6
:10E6200046D4FFF74BFF000642D42078082809D0D3
:10E63000C5F80080C6F8009078463860922004B093
:10E64000BDE8F09FD4F80610CAF80E106189AAF848
:10E650001210607B217BDFF86C8100EB0120A8F8B1
:10E660004800607800F00F01000900EB800001EB2A
:10E6700040008DF80000A07800F00F01000900EBC9
:10E68000800001EB40008DF8010000E010E0E07830
:10E6900000F00F01000900EB800001EB40008DF855
:10E6A000020008F144016846F2F7A7F9000601D517
:10E6B0002868C4E7607900F00F01000900EB8000D2
:10E6C00001EB4001207900F00F02000900EB80000F
:10E6D00002EB4000C0EB001001EB8001A8F84610EF
:10E6E00032490120C870C5F800B07846C6F800B0BD
:10E6F00038600020A3E72DE9F0438BB005463920B0
:10E700008DF8200031A04FF000080068284C2A4EF8
:10E710001B27C146CDF824008DF81C7007AB6A4654
:10E72000022109A81FF0D1F890B1306805283AD22B
:10E73000B8F1000F37D18DF81C9007AB6A46012164
:10E7400008A81FF0C2F800062DD44FF00108E3E737
:10E750009DF801009DF80010052300EB01202880A2
:10E760000622A91C0DF10200F2F776F800061AD471
:10E7700005230622E91D02A8F2F76EF8000612D45E
:10E780000523062205F10C010DF10E00F2F764F8E5
:10E79000000608D40523062205F1110105A8F2F7A9
:10E7A0005BF8000614D520680BB063E683C1072030
:10E7B0000CC007200000094010C0072014C007202B
:10E7C000070300004CC707201C04000007020000DC
:10E7D00016222946FE482EF034F8FE4901204870E2
:10E7E000C4F800907846FC49C6F800900860002004
:10E7F000DAE72DE9F04389B0044639208DF81C0092
:10E80000F6A04FF000080068F54DF64E1527C146FA
:10E81000CDF820008DF8187006AB6A46022108A8D2
:10E820001FF053F890B1306805285DD2B8F1000FA1
:10E830005AD18DF8189006AB6A46012107A81FF03F
:10E8400044F8000650D44FF00108E3E79DF80500B6
:10E8500000F00F01000900EB800001EB40008DF893
:10E8600014009DF8060000F00F01000900EB800085
:10E8700001EB40008DF815009DF8070000F00F0136
:10E88000000900EB800001EB40008DF81600211D0F
:10E8900005A8F2F7B2F89DF80900042300F00F0173
:10E8A000000900EB800001EB40019DF8080000F03A
:10E8B0000F02000900EB800002EB4000C0EB0010EB
:10E8C00001EB8000E080052221466846F1F7C4FF95
:10E8D000000609D404231A4604F108010DF10A00C8
:10E8E000F1F7BAFF000602D5286809B0C2E5DDF8E5
:10E8F0000E00E0609DF8120020749DF81300607413
:10E90000B3481422214614382EF022F8B1490120D0
:10E910000870C5F800907846AF49C6F800900860C6
:10E920000020E2E72DE9F047A94E0546A948143E2C
:10E93000DFF8B082DFF8A092A94F0C46052D05DC68
:10E940000078B0B93046FFF754FF06E00A2D07DC27
:10E95000407870B99E48FFF7CEFE000623D408E049
:10E96000112D04DCC07820B9FFF706FEF5E7122D63
:10E9700011D09748583800F18001132D6AD2DFE892
:10E9800005F01517191C2023282A2F32373D44493A
:10E990004E5255585E00807878BB8D481630FFF790
:10E9A0002DFD00064BD53868BDE8F087707C48E047
:10E9B000406C07E0B0F8480001E0B0F84A00208061
:10E9C00040E0C06C20603DE0016D216090F8540093
:10E9D00004E0B08A25E050F85A1F0BE0207131E0C6
:10E9E00050F85F1F06E0416E216090F86800F5E77F
:10E9F00050F8691F21600079F0E720E0016F216085
:10EA0000416F6160806FA0601CE0C16F2160B0F851
:10EA1000800012E0D1F8020020608879DEE7B6F8C5
:10EA2000440020800EE0B6F84600FAE7B6F8480049
:10EA3000F7E7D1F80E002060488AA08002E096F83F
:10EA40002B002070002038607946C8F80000C9F813
:10EA50000010A9E7922025213860C8F800107946F7
:10EA6000C9F80010A0E75B4AC3074FF0000100D0CF
:10EA700011708307002B01DA517000E000D0917013
:10EA8000400700D5D170564801605648016078466D
:10EA900051490860002070471CB501208DF8000026
:10EAA00051A06B46006801900022022101A81EF0CF
:10EAB0000CFF1CBD30B597B0044608208DF84C0003
:10EAC0004A4801250078002856D02022492168466E
:10EAD0002DF0ADFF8DF8005034F8031B444813AB04
:10EAE000085C8DF8010014F8011C4248415C8DF867
:10EAF00002102178415C8DF803106178415C8DF83B
:10EB00000410A178405C8DF805006068CDF806001F
:10EB1000A068CDF80A00E068CDF80E002069CDF8B5
:10EB20001200A08AADF81600D4F816000690608B8B
:10EB3000ADF81C00B4F81D003121000A8DF81E004C
:10EB4000607F8DF81F0010208DF820002AA0026839
:10EB5000CDF821204068CDF8250035201D4A8DF8DC
:10EB600029000020107050709070D07014AA684670
:10EB70001EF0ABFE17B030BD194988200860194857
:10EB800005607846144908608820F3E77FB504469D
:10EB9000164801250078A8B309208DF800002088C8
:10EBA00002A9F1F7DEFE9DF808101248415C8DF8CD
:10EBB00001109DF80910415C8DF802109DF80A10B3
:10EBC000405C8DF80300608801A9F2F71FF81AE095
:10EBD00060C7072083C1072014C007200701000079
:10EBE0000CC0072010C00720080100001C04000012
:10EBF0001EDD0300EEE40300465072696E742D358D
:10EC00003500000010E020798DF80600F84900205A
:10EC10000246087048708DF80C5003AB0721684617
:10EC20001EF053FE04B070BDF24988200860F2481F
:10EC300005607846F14908608820F3E71CB501209B
:10EC400039218DF80410EE498DF80000097831B1B2
:10EC50006B460022012101A81EF037FE1CBDE54ACB
:10EC600088211160E44908607846E44908608820FA
:10EC70001CBD1CB501200A218DF80410E0498DF857
:10EC80000000097851B1DA49002002460870487046
:10EC90006B46012101A81EF018FE1CBDD54A882133
:10ECA0001160D54908607846D449086088201CBDA9
:10ECB000FEB50E46002521218DF800108DF8085074
:10ECC000042329460DF10102F1F784FDC94C000629
:10ECD00025D402ABCB4A052168461EF0F6FD00069E
:10ECE0001DD4C84F35600020FFF706FC000616D47F
:10ECF000206848B1C048C149326892B125600560BA
:10ED0000784608600020FEBD39780B29EBD104233A
:10ED100003223146781DF1F79FFD0006E3D52068F8
:10ED2000FEBD92222260272202607846086092206F
:10ED3000FEBD2DE9FC41B249AF4EB04F0978AD4D53
:10ED4000C1B1A0218DF80010010A8DF801108DF8D5
:10ED50000200A748002401AB047011208DF80400C4
:10ED6000A84A032168461EF0B0FD00060AD52868AF
:10ED7000BDE8FC818820286001203060784638603A
:10ED80008820F5E79F48102180F8401004742C601B
:10ED90007846346038600020EAE7FEB59849964E20
:10EDA000964F0978934DD1B1A1218DF80010002420
:10EDB000042321460DF10102F1F70CFD00060CD4ED
:10EDC0008B4802AB8F4A047011208DF80800052192
:10EDD00068461EF07AFD000609D52868FEBD882029
:10EDE000286001203060784638608820FEBD854864
:10EDF000102180F8401004742C607846346038602C
:10EE00000020FEBD2DE9FF4188467D497A4E7B4FAB
:10EE10000978784D29B1A2218DF804105AB1042146
:10EE20000AE0882028600120306078463860882019
:10EE300004B0BDE8F08105218DF805106946F1F7B1
:10EE400090FD9DF80000704C6946205C8DF806002E
:10EE50009DF80100205C8DF807009DF80200205C01
:10EE60008DF808004046F1F77CFD9DF8000003ABEB
:10EE7000644A205C8DF809009DF801000821205C9F
:10EE80008DF80A009DF80200205C8DF80B005848B0
:10EE90000024047011208DF80C0001A81EF015FD4F
:10EEA000000601D52868C3E75648102180F84010B5
:10EEB00004742C607846346038600020B8E7FEB5F2
:10EEC0004F4B4D4D4D4E1B784A4C6BB142F20F7378
:10EED000984201D899420FD98620206013202860DB
:10EEE000784630608620FEBD8820206001202860A2
:10EEF000784630608820FEBDA2238DF800300AB12C
:10EF0000062200E007228DF80120020A8DF8022077
:10EF10008DF80300080A8DF8040035488DF80510B7
:10EF20000027077011208DF8080002AB354A062132
:10EF300068461EF0CAFC000601D52068FEBD3148B7
:10EF4000102180F840100774276078462F603060E9
:10EF50000020FEBD2DE9FC412949274E274F0978A5
:10EF6000244DB9B1A3218DF80010010A8DF80110CC
:10EF70008DF802001E48002401AB047011208DF8AA
:10EF80000400204A032168461EF09FFC000609D5B4
:10EF90002868EDE6882028600120306078463860D7
:10EFA0008820E5E61748102180F8401004742C6092
:10EFB0007846346038600020DAE62DE9FC41A42070
:10EFC0008DF804000E480C4E0C4F0078094DE8B146
:10EFD000074800246B46047011208DF80000094A90
:10EFE000012101A81EF071FC000617D52868BFE6B4
:10EFF00083C107200CC0072010C0072014C00720C1
:10F000001C04000008C70720EEE4030088202860E5
:10F0100001203060784638608820A9E6F848102141
:10F0200080F8401004742C6078463460386000200A
:10F030009EE62DE9FC4105208DF80400F148F24ED2
:10F04000F24F0078F24C98B1F24800256B460570FB
:10F050008DF80050EA4A012101A81EF036FC000696
:10F060000ED5F1F7D7F8FFF729FAF1F7E8F818E02D
:10F07000882020600120306078463860882077E65C
:10F080009DF8000048B1102807D092202060202071
:10F0900030607846386092206AE6D94981F84000AD
:10F0A0000D54206864E62DE9FF410446D548D84D4B
:10F0B000D5490278D548012782B12278012A14D097
:10F0C000022A14D0032A2ED0042A2ED086222A60A7
:10F0D00006220A60794601608620A9E688222A6015
:10F0E0000F60794601601046A2E6102000E0112072
:10F0F0008DF80000207B8DF801006E464FF000086F
:10F1000004234146B21C6068F1F764FB000608D492
:10F11000A0680523B21D44460021F1F75BFB000601
:10F1200005D5286884E61220E2E71320E0E7B94815
:10F130006A4603AB047044708DF80C700B211046C6
:10F140001EF0C3FB74E62DE9FF410446AD48B04D07
:10F15000AD490278AD4801279AB118228DF80020F8
:10F160002278012A14D0022A14D0032A2ED0042A8D
:10F170002ED086222A6006220A6079460160862007
:10F1800056E688222A600F607946016010464FE6F5
:10F19000102000E011208DF80100207B8DF8020086
:10F1A0006E464FF0000804234146F21C6068F1F7F8
:10F1B00011FB000608D4A0680523F21D4446002177
:10F1C000F1F708FB000605D5286831E61220E2E7D2
:10F1D0001320E0E78F4803AB0022047044708DF8E1
:10F1E0000C700C2168461EF070FB21E6FEB58549C7
:10F1F000874E0125097871B116218DF80010002481
:10F200000068052321460DF10102F1F7E3FA00063B
:10F210000AD53068FEBD882030607B48056078469E
:10F220007A4908608820FEBD7A4802AB002204704B
:10F2300044708DF80850062168461EF046FBFEBD5E
:10F24000FEB57049724E0125097889B118218DF8F3
:10F25000001016218DF801100024006805232146B6
:10F260000DF10202F1F7B6FA00060AD53068FEBDCC
:10F2700088203060644805607846644908608820CA
:10F28000FEBD644802AB0022047044708DF8085043
:10F29000072168461EF019FBFEBDFEB559495C4EBC
:10F2A0000125097871B117218DF80010002400683C
:10F2B000052321460DF10102F1F78CFA00060AD56B
:10F2C0003068FEBD882030604F48056078464F4961
:10F2D00008608820FEBD4F4802AB002204704470D5
:10F2E0008DF80850062168461EF0EFFAFEBDFEB507
:10F2F0004449474E0125097889B118218DF800103D
:10F3000017218DF8011000240068052321460DF116
:10F310000202F1F75FFA00060AD53068FEBD8820C8
:10F320003060394805607846384908608820FEBD5D
:10F33000384802AB0022047044708DF80850072151
:10F3400068461EF0C2FAFEBD2DE9F04104462D4884
:10F350002D4E2E4F00782E4D86B08846F0B3208873
:10F3600002A9F1F7FEFA19208DF800009DF80810A7
:10F370002948415C8DF801109DF80910415C8DF819
:10F3800002109DF80A10405C8DF80300608801A906
:10F39000F1F73CFC20798DF806001E48002405ABEF
:10F3A0000470447008208DF8140003AA07216846F1
:10F3B0001EF08BFA000610D404231A46414603A817
:10F3C000F1F74AFA000608D40423032208F10401E5
:10F3D00004A8F1F741FA00060CD500E002E0286825
:10F3E00006B026E588202860012030607846386025
:10F3F0008820F5E72C607846346038600020EFE71D
:10F4000008C707201C04000010C0072014C00720F4
:10F410000CC0072083C10720EEE403002DE9FC5F48
:10F420000D469A499A4C9B4E09789B4F00295BD018
:10F4300023218DF80010010A8DF801108DF80200CB
:10F440004FF000098DF8049001AB944A03216846FF
:10F450001EF03BFA000643D4DFF840820020FFF79D
:10F460004BF800063CD498F8401029B198F80000F9
:10F47000092801D01028F1D1FFF720F800062FD479
:10F4800098F84010404671B3027805F10A0A092A3B
:10F4900005F10F0B4FF005034FF00602294637D058
:10F4A000C01CF1F7D9F900061AD47C4805230622BE
:10F4B000691D0930F1F7D0F9000611D4774805230A
:10F4C000062251460F30F1F7C7F9000608D47348F9
:10F4D0000523062259461530F1F7BEF9000635D549
:10F4E0002068BDE8FC9F07E0882020600120306094
:10F4F000784638608820F4E7142128462DF09FFADA
:10F500009220206027203060784638609220E8E71B
:10F5100008F10100F1F7A0F90006E1D40523062265
:10F52000691D08F10700F1F797F90006D8D45B4888
:10F530000523062251460D30F1F78EF90006CFD48F
:10F5400056480523062259461330C5E7C4F80090F3
:10F550007846C6F8009038600020C2E72DE9FE43E7
:10F560000F464A494A4DDFF82C810978DFF8289187
:10F5700029B323218DF80010010A8DF801108DF8B0
:10F58000020000268DF8086002AB444A0321684659
:10F590001EF09BF900060FD4404C0020FEF7ACFF94
:10F5A000000609D494F8400010B120780E28F4D158
:10F5B000FEF784FF00060BD52868BDE8FE8388208F
:10F5C00001212860C8F800107946C9F80010F4E756
:10F5D00094F84000F0B3E07800F00F01000900EB70
:10F5E000800001EB40008DF80400207900F00F014D
:10F5F000000900EB800001EB40008DF80500607908
:10F6000000F00F01000900EB800001EB40008DF8D5
:10F610000600394601A8F1F7F0F9E07900F00F0192
:10F62000000900EB800001EB4001A07900F00F021F
:10F63000000900EB800002EB4000C0EB001001EB82
:10F6400080007880207A38712E607946C8F8006092
:10F65000002000E002E0C9F80010AEE73E60922012
:10F66000BE8027212860C8F800107946C9F800102C
:10F67000A3E71021016006490020086005490860E1
:10F680007846054908600020704700001C0400000F
:10F690000CC0072010C0072014C0072008C707208F
:10F6A000F0B54178FD4AFE4BFE4C962509B119296B
:10F6B00003D902201560186015E005260E2916D022
:10F6C00006DC052913D0062911D00D2904D10EE03E
:10F6D0000F290CD019290AD0F34F0078795C8842A1
:10F6E00009D015601E60784620609620F0BD007835
:10F6F000801E3528F5D20020106018607846206002
:10F700000020F0BD2DE9F04F0120E44AE44BE54C28
:10F710000225E54F4FF036094FF00E0A4FF00D0B62
:10F720004FF006084FF00A0E4FF0070C03261A2878
:10F730006AD2DFE800F0691112171A25292D313538
:10F74000393D4115154552560D5A5E62211D6645DB
:10F7500087F812B01320EAE77E70BD700320E6E759
:10F7600035212EE0FD700420E1E73D710520DEE744
:10F7700087F817801820DAE787F816801720D6E771
:10F7800087F805900620D2E787F806900720CEE795
:10F7900087F807A00820CAE787F808A00920C6E76D
:10F7A00087F809C00A20C2E787F80AC00B20BEE725
:10F7B00087F80BB00C20BAE787F80CE00D20B6E70D
:10F7C00000213954401C1928B1D90020106018605C
:10F7D000784620600020BDE8F08F87F81080112067
:10F7E000A5E787F811E01220A1E787F813C01420DD
:10F7F0009DE787F814C0152099E705217975162033
:10F8000095E73E76192092E78F20106078461E60BB
:10F8100020608F20DFE72DE9F04F95B04FF0405882
:10F820004046012213A9CDF8388020F0E5FC9B4C1E
:10F8300000066AD408F10100012212A90E9020F0FE
:10F84000DBFC000661D499494FF00109962781F845
:10F8500000909DF84C00924D924EFF2805D05728FD
:10F860000AD04846276028600FE09DF84800FF282E
:10F87000F7D107202760F6E79DF848004FF0030A0C
:10F88000802807D02760C5F800A078463060962011
:10F8900015B0A0E70EA8F6F727FF000635D410A88C
:10F8A000F6F733FF000630D4404620F0BCFCA0F150
:10F8B000010850460E994FF0060AB0EB117FE1D1D6
:10F8C00021F070414145DDD2109AB0EB127FD9D1C1
:10F8D00022F070404045D5D20229D3D30228D1D39B
:10F8E000DFF8CCB110990E9888422AD002226946DE
:10F8F00020F082FC000608D49DF80000FF2806D006
:10F900006846FFF7CDFE000603D52068C0E78DF8F6
:10F91000009010990E98884207D29DF8002002446A
:10F920008A4202D9052027609DE79DF8001008440F
:10F9300020F070410E904145A4D8D3D1CDF838B015
:10F94000D0E74FF0000020602860784630604FF02C
:10F9500000009DE7FEB54FF040573C46384620F08A
:10F9600062FC54494618204620F063FC0546684670
:10F97000F6F7CBFE494C000621D40098B84219D0C6
:10F9800020F0704101F56C312A4601A800912CF05D
:10F99000C9FE0199491C6943B14201D3B81C03E077
:10F9A000A1F56C3141F0405000906846F6F7A3FE97
:10F9B000000604D46846F6F78DFE000601D52068DF
:10F9C000FEBD374900202060086078463549086050
:10F9D0000020FEBD1CB53548304C007888B122F0BF
:10F9E00065F808B1344800E03448009048F2570008
:10F9F000ADF80400022201A9009820F008FC0006DE
:10FA00000BD42B4800906846F6F764FE000604D439
:10FA10006846F6F770FE000601D520681CBD204937
:10FA200000202060086078461E49086000201CBD48
:10FA30001E48007870472DE9FC4106460D464FF000
:10FA4000405020F0F0FB441E1848144F4FF00008BF
:10FA5000007860B16846F6F747FE000604D401A8B6
:10FA6000F6F753FE000607D53868BDE8FC81C6F8F6
:10FA70000080C5F8008009E0A41E2C60DDE90010BC
:10FA8000401A306002D52968084430600449C7F83C
:10FA900000807846C1F80080024911E00CC00720C0
:10FAA00010C0072014C007209CC7072088C107206A
:10FAB00002000030FFAF030000B003B0009005B0BB
:10FAC00008600020D1E71CB500200090019001A93A
:10FAD0006846FFF7B0FF000603D4009808B1002085
:10FAE0001CBD01201CBD2DE9FC4180460024FB48C3
:10FAF000009401940078FA4EFA4FFB4D38B101A9F9
:10FB00006846FFF798FF000608D52868ADE705208E
:10FB100028607846346038600520A6E7DDE90010EB
:10FB2000411A08EBC80000EB4000B1EB400F07D2D0
:10FB3000962028600420306078463860962094E74C
:10FB40002C6078463460386000208EE710B540782D
:10FB5000E54C0B281AD008DC01280ED0022815D05D
:10FB600009280CD00A2806D109E00C280ED010284C
:10FB700005D0112803D0182002E0782000E00F20E3
:10FB8000FFF7B1FF000603D5206810BD0C20F7E792
:10FB9000D3490020206008607846D24908600020E0
:10FBA00010BD2DE9F04F044693B04FF0405020F0C7
:10FBB0003AFBA0F1010AC948C94FDFF82883007851
:10FBC000C94E002500287DD011A949200BF084FEE4
:10FBD000000678D49DF84400032873D0022811D180
:10FBE00060781A286ED2DFE800F08E0D0D0D0D0D35
:10FBF0000D0D0D8E8E0D8E0D0D8E0D8E0D0D0D8E2F
:10FC00000D0D8E0D2046FFF7A1FF00066FD4607822
:10FC100008B1192809D99620306003207946386048
:10FC20009620C8F8001013B0D5E5DFF8C0920E2872
:10FC30000ED006DC052817D0062815D00D2804D1D3
:10FC400006E00F2855D0192853D019F8000018E005
:10FC500004F110002CF0CAFD242802D984F8345095
:10FC6000242099F80D100AE004F111002CF0BEFDDB
:10FC7000242802D984F83550242099F80510243816
:10FC8000084420706846F6F740FD00062FD400981F
:10FC900020F07041AAEB01092178834649450DD92E
:10FCA000FF22362101A82CF0C2FE4A4601A958467F
:10FCB00020F0ADFA00061AD48D4800902278214633
:10FCC000009801E01FE012E020F0A1FA00060ED437
:10FCD00020780099084420F070410090514501D1EE
:10FCE000834800906846F6F706FD00060BD530689D
:10FCF00099E7A01C2CF07AFD242802D984F826501C
:10FD00002420C01CBDE7356079463D600020C8F85E
:10FD1000001088E72DE9F84F07464FF0405020F0DB
:10FD200082FADFF8B8B1461E6F4C9BF80000DFF88E
:10FD3000B081DFF8B09100254FF0050AF0B16846B8
:10FD4000F6F7E3FC000631D4DBF8043000998B426F
:10FD500014D03622394618461CE0DBF80410584609
:10FD6000491CCBF8041021F07041B14201D1604927
:10FD70004160DBF804000099884209D1C4F800A072
:10FD80007946C8F800500520C9F80010BDE8F88F82
:10FD90003622394620F030FA000607D43878FF289A
:10FDA000DBD03846FFF77CFC000601D52068EDE784
:10FDB0003978DBF804201144CBF8041021F07041AD
:10FDC000B14202D14A49CBF8041025607946C8F8FF
:10FDD00000500020C9F80010D8E72DE9F14FDFF8F6
:10FDE000FC800027404C98F800003D4D3D4E90B0FF
:10FDF000B9464FF0050A00286FD00EA8F6F785FC2B
:10FE0000000637D44FF0405020F00DFAA0F1010B5E
:10FE100070E00222694620F0EFF900062AD49DF82E
:10FE20000000FF2814D09DF8011005291DD00629D7
:10FE30001BD00B2919D0D8F804204146104420F0DB
:10FE40007042C8F804005A4517D0D8F8040016E0EC
:10FE5000D8F80400401C20F07042C8F804005A454D
:10FE600048D12348C8F8040044E06846FFF752FF31
:10FE7000000610D5206811B0ADE41D48486020F0A0
:10FE80007041594507D996202060062028607846A1
:10FE900030609620EFE79DF80100012803D0052887
:10FEA00001D0062804D19DF80020D8F804108F1A3C
:10FEB000052803D0062801D00B281BD1BDF80A1055
:10FEC0001098814216D1C8F80470C4F800907846A2
:10FED000C5F8009030600020CDE710E088C1072011
:10FEE00010C0072014C007200CC007209CC70720A3
:10FEF00002000030D8F804000E99884289D1C4F875
:10FF000000A07846C5F8009030600520B3E7F0B552
:10FF1000BD48BE4EBE4F0078BE4C87B00025A8B38A
:10FF2000B948001DF6F7E0FB00062CD401A826F026
:10FF300081FE000627D4694621200BF098FD0006BB
:10FF400021D49DF80000ADF8040069461F200BF095
:10FF50008EFD000617D49DF80000ADF80A00694632
:10FF600026200BF084FD00060DD49DF80000ADF8AE
:10FF70000C0026F0F0FE000605D4002101A826F0B2
:10FF8000D5FB00060AD5206807B0F0BDFFE70520C5
:10FF900020607846356038600520F5E725607846B2
:10FFA000356038600020EFE72DE9F843964E974F13
:10FFB000DFF85C823078974C002560B16846F6F730
:10FFC00063FA000663D47078B8B126F095FE000697
:10FFD00009D575705BE00520206079463D60C8F862
:10FFE0000010BDE8F8832068052854D08648001D1D
:10FFF000F6F770FB00064AD47570DFF81C9286484D
:020000040001F9
:10000000FFF788FE000642D42068D8B99DF80000AA
:1000100017281AD0152818D0192816D099F80100D9
:100020001A28ECD2DFE800F00D0E0E0E0E0E0E0EAA
:100030000E0D0D0E0D0E0E0D0E0D0E0E0D0D0E0EE7
:100040000D0EDCE720680528CBD05B200AF06FFCA2
:1000500000061CD499F80100062809D004DC022807
:1000600006D0052817D103E00B2801D0122812D1A1
:100070005C200AF05CFC000609D49DF800001728FB
:1000800001D0182807D126F01AFE000601D52068F5
:10009000A7E701207070256079463D600020C8F810
:1000A00000109EE770B5054657480021574A03786F
:1000B0005748584C8EB0002B3ED0AB0B3CD057A0CD
:1000C00026F0A3FC000634D4002159A026F09DFCA4
:1000D00000062ED4280411D5FFF719FF000628D4F6
:1000E000FFF762FF20680028FAD026F034FE0006F1
:1000F0001FD4012026F08AFB00061AD453200AF0F0
:1001000016FC000615D4012001F00CFD000610D4E9
:10011000FFF760FC00060CD40F256E468DF80150E9
:100120003EA1B01C2CF03EFB6846FFF73AFD0006EE
:1001300008D520680EB070BD21601160794601605D
:100140000020F7E78DF8015039A1B01C2CF02AFBF4
:100150006846FFF726FDEDE72DE9F05F2A4C1646CD
:100160008B464FF0010A012803D0606810F0405F11
:1001700005D1254884F802A0001DF6F7B5FADFF88E
:100180008C80DFF88C90234DA07801280DD1224F70
:100190002148FFF7BFFD000613D42868052813D0B7
:1001A00078781528F4D01828F2D025483146C0892F
:1001B0003060A278584607F08BFE07000DD0052F5F
:1001C0000BD02868BDE8F09F9120AD212860C8F8C9
:1001D00000107946C9F80010F4E758463168F0F786
:1001E00068FD67B184F802A030680028CCD00020F8
:1001F00028607946C8F80000C9F80010E2E7A07846
:10020000401CA070F0E7000088C1072010C0072044
:1002100014C007200CC00720A0C807208E98888132
:100220008A80208693908D808B80208A8B0A0000A4
:1002300086E3E0ADA0AB20AEE7A8E9A5AD0A0000DB
:1002400000DD07202DE9FF47022003901DF0BEFBD3
:100250000024FD48FD4EDFF8F89344708460254685
:1002600003274FF03208C4608DF804708DF80550F4
:1002700003AB02AA022101A8CDF800801DF06BFC9F
:10028000000603D5306804B0BDE8F0879DF808008B
:100290009DF8091000EB012009EB45016D1C8886D3
:1002A000032DE1D3EB48346004607846EA490860E6
:1002B0000020E8E7E64A02EB4000808E0880E34930
:1002C00000200860E34908607846E34908600020A0
:1002D000704708B569460220FFF7ECFF0106DB48CE
:1002E00001D5006808BDBDF80030DA49DA4AB3F537
:1002F0007A7F07D2932303600B2008607846106052
:10030000184608BD0023036078460B60106018464D
:1003100008BD2DE9FF418846CB4D02210391012400
:10032000E968CB4A8440C94F0C4202EB40061CD11D
:1003300004218DF804108DF805003220009003ABE5
:1003400002AA022101A81DF006FC000603D53868A8
:1003500004B0BDE8F0819DF808009DF8091000EB9D
:1003600001207087E8680443EC60718FA8F80010E2
:10037000B8490020386008607846B7490860002016
:10038000E6E73EB5044641208DF804000C200290BB
:100390003220009002AB2246012101A81DF0DBFBB8
:1003A0000106AA4801D500683EBDA7498A6842F007
:1003B00080028A60A64922681439CA6362680A64A6
:1003C000A2684A6400210160A24801607846A249FF
:1003D000086000203EBD0EB570B101280ED0022885
:1003E0001DD09A49882008609A490D2008607846F7
:1003F0009949086088200EBD102200E00522121DD8
:10040000019209228DF808208DF8090032200A4651
:10041000009001AB022102A81DF09DFB0EBD0A2237
:10042000EDE70EB50022029210228DF804208DF81F
:1004300005008DF80610080A8DF80700322001AA81
:10044000009002AB042110461DF085FB0EBD38B5AF
:1004500004466946FFF75DFF7C4A000601D5106837
:1004600038BDBDF8001039B1491E89B2ADF8001091
:100470002046FFF7D6FF38BD0520764910600020E2
:100480000860784674490860052038BD2DE9FE4FA4
:100490000D466D496E4E81466E4FDFF8BC81143EAD
:1004A0006A4C88684FF0930A4FF0070BB9F1050FBB
:1004B00059D2DFE809F0301818034F008946800749
:1004C00042D40120FFF7C3FF98BB614901201431DA
:1004D000FFF781FF000643D4D9F8081041F002016C
:1004E000C9F8081030E0C0070DD1FFF7B0FF00BB1E
:1004F00057490020FFF76FFF000631D4524881684A
:1005000041F001018160B9F1050F2CD2DFE809F05B
:100510000A12161C2200000604D46846FFF731FFB9
:1005200000061DD4F06B2860306C6860706CA860A9
:1005300022E015E0B0692860B08B03E0D6F81E0019
:100540002860708CA88017E0F06A286096F8300068
:10055000287111E029460220FFF7DBFE00060BD5CB
:100560002068BDE8FE8FC4F800A07946C7F800B047
:100570009320C8F80010F4E7002020607946386026
:10058000C8F80010EDE730498A6882438A60CA687B
:100590008243CA602D49002008602E4908607846D1
:1005A0002D490860002070472DE9F04F264D0422A8
:1005B00089B08046284F0026DFF89890234C2846C3
:1005C0006A704FF0860A4FF0010B022909D0032907
:1005D00007D0042922D0052920D00821C4F800A082
:1005E00043E0067003291FD01CE01748A97017309C
:1005F000F4F7EBFC14481030F4F7E7FC1248124D06
:1006000000781E3590B1A5F800B0B8F80010A980A8
:10061000A5F802B0B8F80200E8801FE080F800B04A
:10062000052901D00021E0E70121DEE7B8F800004C
:100630002880AE80B8F802106980EE8088420DD91B
:100640001321C4F800A010E090C107200CC00720BF
:10065000CAC7072010C0072014C00720A888E9884F
:1006600088420AD91421C4F800A07846C9F80010BD
:100670003860862009B0BDE8F08F69460220FFF798
:1006800048FE000669D4DFF814844FF0810A98F818
:10069000000020B92888BDF8001088426CD828884E
:1006A000401E81B20220FFF7BCFE000679D402A9E9
:1006B0000220FFF790FE206838B105280AD0932861
:1006C000D8D1D9F800100829D4D198F8001079B100
:1006D00020B10DE098F80000F0BB11E0BDF8083043
:1006E000AA88934204D3BDF80A002880AB8010E0AA
:1006F0000143DCD1BDF80800A88098F8000040B99B
:100700006888BDF80010884200D90846ADF800009E
:100710006880BDF80000401E81B20220FFF781FE14
:1007200000063ED402A90220FFF755FE206828B13A
:1007300093289FD1D9F8001008299BD198F8001070
:1007400061B158B9BDF80820EB889A4206D8BDF8C7
:100750000A00688090B219E00EE022E0014313D055
:10076000BDF80000401E80B2ADF80000298881422B
:10077000CFD998F8000050B1C4F800A07846C9F865
:1007800000603860812075E7BDF80800E88028889F
:10079000401E81B2A8F804100220FFF742FE0006B6
:1007A00001D5206866E726607846C9F800603860A1
:1007B00000205FE72DE9F047B84DDFF8E492DFF85D
:1007C000E4826878B84C002720B1032819D00428A7
:1007D0000FD107E0052020607946C8F80070C9F8FD
:1007E000001051E54F200AF0A2F800064AD4032079
:1007F000687027607946C8F800700020C9F80010BA
:1008000042E50026A9490220FFF7E5FD932804D11F
:10081000D8F80000082835D10126A888401C80B2ED
:10082000A880A97836EA010110D052200AF07FF89A
:10083000000627D426F08FFA000623D481202060FA
:100840007946C8F80070C9F800101DE5216805292F
:1008500004D092491E314988814202D26F705020E3
:1008600017E08EB991498D48091D1030F4F74FFCFF
:10087000000607D48D49894809311730F4F747FC41
:10088000000601D52068FFE4A8780028B9D026B179
:100890005220BDE8F0470AF04AB85120F9E700B508
:1008A00087B0002106918DF80400322001AA009043
:1008B00006AB012110461DF04EF907B000BD70B522
:1008C00088B003004FF00000774D0E4607900ED021
:1008D000012B0ED0022B0ED08820724928600D20EB
:1008E000086078466E490860882008B070BD102402
:1008F00002E0052400E00A2401209840241DFFF7AF
:1009000042FE000601D52868EFE708208DF80400B4
:100910008DF80530224631460DF106002BF091FF8F
:10092000322001AA009007ABA11C10461DF013F95C
:10093000DBE77CB50C4605466946FFF7EAFC5A4BF7
:10094000000605D401A92846FFF7B4FC000601D52E
:1009500018687CBDBDF80400BDF80010401A208066
:10096000504900201860086078464D490860002012
:100970007CBD7FB5054615208DF808000420039046
:1009800032200C46009003AB01AA012102A81DF001
:10099000E2F80106444802D5006804B070BDBDF815
:1009A00004102980BDF806102180002101603D4817
:1009B000016078463A4908600020EEE70EB5022251
:1009C000029216228DF804208DF8050041F288303D
:1009D0000A46009002AB022101A81DF0BCF80EBD32
:1009E00000B587B00021059140218DF80410016801
:1009F000CDF805104168CDF809108068CDF80D00DC
:100A0000264801AA05AB816821F08001816032206F
:100A100000900D2110461DF09EF84EE770B58CB089
:100A2000064680208DF824001E200A9032200D46B4
:100A300000900AAB01AA012109A81DF08CF81A4CFC
:100A4000000608D4BDF8040028801C220DF1060120
:100A500030462BF0F6FE20680CB070BD3EB5044663
:100A60000220029081208DF80400322001AA00901B
:100A700002AB012110461DF06EF801060A4801D5AF
:100A800000683EBDBDF804102180002101600548CA
:100A9000016078460249086000203EBD90C10720F1
:100AA00014C0072010C007200CC00720B6C70720BD
:100AB000F0B54478FD49FE4AFE4BA2250CB1192C35
:100AC00003D902200D60106015E005260E2C16D00B
:100AD00006DC052C13D0062C11D00D2C04D10EE011
:100AE0000F2C0CD0192C0AD0F34F00783C5DA0429B
:100AF00009D00D60166078461860A220F0BD00781D
:100B0000801E3528F5D200200860106078461860F5
:100B10000020F0BD2DE9F04F0120E44AE44BE54C04
:100B20000225E54F4FF036094FF00E0A4FF00D0B3E
:100B30004FF006084FF00A0E4FF0070C03261A2854
:100B40006AD2DFE800F0691112171A25292D313514
:100B5000393D4115154552560D5A5E62211D6645B7
:100B600087F812B01320EAE77E70BD700320E6E735
:100B700035212EE0FD700420E1E73D710520DEE720
:100B800087F817801820DAE787F816801720D6E74D
:100B900087F805900620D2E787F806900720CEE771
:100BA00087F807A00820CAE787F808A00920C6E749
:100BB00087F809C00A20C2E787F80AC00B20BEE701
:100BC00087F80BB00C20BAE787F80CE00D20B6E7E9
:100BD00000213954401C1928B1D900201060186038
:100BE000784620600020BDE8F08F87F81080112043
:100BF000A5E787F811E01220A1E787F813C01420B9
:100C00009DE787F814C0152099E70521797516200E
:100C100095E73E76192092E78F20106078461E6097
:100C200020608F20DFE738B54FF0404000906846E5
:100C3000F5F772FD9D4C000604D46846F5F77DFD7E
:100C4000000601D5206838BD994900202060086061
:100C5000784698490860002038BD2DE9FC4120F015
:100C6000FBFF934E934F914D002438B393490120DD
:100C700008706846F5F75AFD000604D401A8F5F798
:100C800066FD000602D52868BDE8FC814FF04040B3
:100C90001FF0C9FA009A0C21401EB1EB127F0BD154
:100CA00022F07042824207D2019AB1EB127F03D147
:100CB00022F07041814201D3FFF7B5FF2C607846E6
:100CC000346038600020DFE7FEB54FF0404528462D
:100CD0001FF0A9FA7A49471828461FF0AAFA0646D3
:100CE0006846F5F734FD714C000621D40098A842FF
:100CF00019D020F0704101F50831324601A8009169
:100D00002BF010FD0198401C7043B84201D30095B0
:100D100004E0A0F5083040F0404000906846F5F748
:100D20000CFD000604D46846F5F7F6FC000601D574
:100D30002068FEBD5E4900202060086078465D495D
:100D400008600020FEBD5D48007870472DE9FC4139
:100D500005460C464FF040401FF065FA461E5748C6
:100D6000524F4FF00008007858B16846F5F7DEFCA6
:100D7000000604D401A8F5F7EAFC000606D5386899
:100D800082E7C5F80080C4F8008008E02660DDE94D
:100D90000010401A286002D52168084428604449A0
:100DA000C7F800807846C1F80080424908600020FA
:100DB0006AE72DE9FC4180460024404800940194F4
:100DC00000783B4E3B4F394D38B101A96846FFF7DB
:100DD000BDFF000608D5286856E70520286078463C
:100DE0003460386005204FE7DDE90010411A08EB58
:100DF000C80000EB4000B1EB400F07D2A2202860F2
:100E00000420306078463860A2203DE72C607846A8
:100E100034603860002037E710B54078234C0B2849
:100E20001AD008DC01280ED0022815D009280CD0D1
:100E30000A2806D109E00C280ED0102805D0112868
:100E400003D0182002E0782000E00F20FFF7B1FF68
:100E5000000603D5206810BD0C20F7E714490020D8
:100E600020600860784613490860002010BD2DE915
:100E7000F04F044693B04FF040401FF0D4F9471EA6
:100E80000E48DFF82C90DFF82CA00078074E0025E4
:100E900000287DD011A962200AF01EFD000678D43A
:100EA0009DF84400C00773D020460BE00CC007201B
:100EB00010C0072014C007200AC80720B8C10720A7
:100EC000FF1F0200FFF7A8FF000671D4607808B189
:100ED000192809D9A22003213060C9F800107946E9
:100EE000CAF8001013B07EE6DFF8D4820E280ED0C8
:100EF00006DC052817D0062815D00D2804D106E0F9
:100F00000F2857D0192855D018F8000018E004F120
:100F100010002BF06BFC242802D984F834502420D4
:100F200098F80D100AE004F111002BF05FFC242862
:100F300002D984F83550242098F805102438084444
:100F400020706846F5F703FC000631D4009821783C
:100F5000834620F07040A7EB000841450ED9FF22E0
:100F6000362101A82BF063FD424601A958461FF027
:100F70004EF900061CD44FF04040009022782146E4
:100F800000981FF044F9000612D42078009901E07F
:100F90001AE00DE00844009020F07040B84202D101
:100FA0004FF0404000906846F5F7C7FB00060BD5B0
:100FB000306897E7A01C2BF019FC242802D984F88C
:100FC00026502420C01CBBE735607946C9F8005084
:100FD0000020CAF8001085E72DE9F84F07464FF0CA
:100FE00040401FF020F9DFF8DCB1461E764C9BF83C
:100FF0000000DFF8D881DFF8D89100254FF0050A0E
:10100000F8B16846F5F7A3FB000632D4DBF80430EC
:1010100000998B4215D03622394618461DE0DBF880
:1010200004105846491CCBF8041021F07041B1421D
:1010300002D14FF040414160DBF804000099884242
:1010400009D1C4F800A07946C8F800500520C9F8B5
:101050000010BDE8F88F362239461FF0CDF80006A3
:1010600007D43878FF28DAD03846FFF721FD00068C
:1010700001D52068EDE73978DBF804201144CBF87E
:101080000410B14203D14FF04041CBF80410256069
:101090007946C8F800500020C9F80010D9E749483F
:1010A000007818B14748001DF5F740BB46490520B8
:1010B00008604649002008607846454908600520D8
:1010C00070472DE9F04FDFF8FC803F4C3F4E98F819
:1010D00000003F4F8FB000254FF0050978B30EA8F0
:1010E000F5F735FB00060DD44FF0404A50461FF08F
:1010F0009AF8A0F1010B1DE0022269461FF07CF86E
:10110000000602D520680FB06DE59DF80000FF28AD
:1011100005D025607846356038600020F3E7D8F8C0
:101120000400401C20F07042C8F804005A4501D168
:10113000C8F804A0D8F804000E998842DCD1C4F89D
:1011400000907846356038600520DCE72DE9F843EB
:101150001C4E1E4FDFF8788030781B4C002560B1A4
:101160006846F5F791F9000620D4707888B125F02B
:10117000C3FD000609D5757018E00520206079468A
:101180003D60C8F80010BDE8F883206805280FD03E
:1011900075701048FFF720FF000607D42068052867
:1011A000F1D06A2009F0C3FB000601D52068EAE708
:1011B000256079463D600020C8F80010E3E7000094
:1011C0000AC80720B8C107200CC0072010C007209C
:1011D00014C00720A0C8072038B55F2009F0A7FB7E
:1011E000964C000613D4532009F0A1FB00060ED440
:1011F0006846F4F765FC000609D46846F4F758F829
:10120000000604D46846F4F751FC000601D52068B6
:1012100038BD8B4900202060086078468949086005
:10122000002038BD10B5162009F081FB000602D55C
:101230008248006810BDBDE8104025F08CBDF0B5B7
:101240007F4F8FB03868092801D8D23000E0D22013
:101250007D4D6860492009F06AFB784C00061DD47A
:1012600019208DF80500686801AE009077A37AA276
:101270002521B01C2BF024F8304400258570F4F7AC
:10128000D4FA08B1F4F7A5F901A8FEF78AFC000624
:1012900004D401A8FFF7EBFD000602D520680FB0CB
:1012A000F0BDF4F7C2FA08B1F4F79FF9256078466B
:1012B00064493D6008600020F1E7F0B58FB0054655
:1012C000002125F0A2FB5D4C00061FD419208DF8EB
:1012D000010028462BF08AFA0C38074602466E4673
:1012E0002946B01C2BF0ADFAF01900258570F4F7F3
:1012F0009CFA08B1F4F76DF96846FEF752FC000657
:1013000004D46846FFF7B3FD000601D52068C6E7A0
:10131000F4F78BFA08B1F4F768F9494825600560DD
:101320007846484908600020B9E738B543484C4C36
:101330000068922801D0932816D1414800682028DF
:1013400009D004DC062806D008280DD103E028289F
:1013500001D02A2808D13C480178012902D12178FE
:1013600009073BD501210170EEF754FF022025F05B
:10137000DDF8207800070DD5432009F0D8FA0006E3
:101380002AD425F0E8FC000626D4208820F00800A6
:10139000208021E0694662200AF09EFA9DF8000054
:1013A000000701D425F0D7FC25F0E1FD002025F051
:1013B00030FC022025F0BAF8432009F0B8FA000604
:1013C00003D425F0C8FC000603D5208840F00800AF
:1013D0002080012025F01DFCEEF731FF38BD10B54F
:1013E0001F4C2078C0071ED125F0C1FD002025F03C
:1013F00010FC1C4988681C4A8B681B1A9342FBD35B
:10140000022025F093F86C2009F091FA000607D429
:1014100025F0A1FC000603D4208840F001002080C4
:10142000012025F0F6FB054900200860044908600A
:10143000784604490860002010BD00000CC0072059
:1014400010C0072014C00720C0C107208E988881D3
:101450008A80209D8A8B870025732025750A0000CD
:1014600002C0072000000940B0AD010038B50020DF
:1014700009F05DFAFE4C00060DD4694662200AF0C0
:101480002BFA000607D49DF80000000705D425F0CC
:1014900062FC000601D5206838BDF64900202060B6
:1014A00008607846F4490860002038BD38B5054624
:1014B000012000F037FBEE4C000611D469461420E1
:1014C0000AF00AFA00060BD49DF80000C10709D003
:1014D0006D1E0540680705D424F05BFF000601D5AA
:1014E000206838BDE3490020206008607846E24962
:1014F0000860002038BD38B5694662200AF0ECF972
:10150000DB4C000619D49DF80000000703D425F039
:1015100022FC000611D4D94D288840F00400288010
:10152000102009F004FA000607D49DF80000000717
:1015300005D425F010FC000601D5206838BD2888A8
:10154000CC4920F004002880002020600860784604
:10155000C9490860002038BD38B50F2009F0E7F907
:10156000C34C00060DD4694662200AF0B5F90006A6
:1015700007D49DF80000000705D425F0ECFB000619
:1015800001D5206838BDBB4900202060086078463E
:10159000B9490860002038BD70B5B848B84DB44CA2
:1015A0000078297800F02000084314D00E2009F0BC
:1015B000BEF9000603D425F0CEFB000601D5206855
:1015C00070BD0020AB492870206008607846AA49A9
:1015D0000860002070BD002025F01BFB0E2009F0E4
:1015E000A6F9000603D425F0B6FB000601D50120BC
:1015F0002870EEF70FFE012025F00BFBEEF71FFE23
:10160000DDE738B50D2009F092F9994C00060DD4AC
:10161000694662200AF060F9000607D49DF80000D0
:10162000000705D425F097FB000601D5206838BDDA
:10163000904900202060086078468F4908600020AB
:1016400038BD38B50C2009F072F9894C00060DD46C
:10165000694662200AF040F9000607D49DF80000B0
:10166000000705D425F077FB000601D5206838BDBA
:10167000804900202060086078467F49086000208B
:1016800038BD38B50B2009F052F9794C00060DD45D
:10169000694662200AF020F9000607D49DF8000090
:1016A000000705D425F057FB000601D5206838BD9A
:1016B000704900202060086078466F49086000206B
:1016C00038BD38B5592009F032F9694C00060DD4FF
:1016D000694662200AF000F9000607D49DF8000070
:1016E000000705D425F037FB000601D5206838BD7A
:1016F000604900202060086078465F49086000204B
:1017000038BD38B55A2009F012F9594C00060DD4ED
:10171000694662200AF0E0F8000607D49DF8000050
:10172000000705D425F017FB000601D5206838BD59
:10173000504900202060086078464F49086000202A
:1017400038BD38B50A2009F0F2F8494C00060DD42E
:10175000694662200AF0C0F8000607D49DF8000030
:10176000000705D425F0F7FA000601D5206838BD3A
:10177000404900202060086078463F49086000200A
:1017800038BD38B5092009F0D2F8394C00060DD41F
:10179000694662200AF0A0F8000607D49DF8000010
:1017A000000705D425F0D7FA000601D5206838BD1A
:1017B000304900202060086078462F4908600020EA
:1017C00038BD38B5072009F0B2F8294C00060DD411
:1017D000694662200AF080F8000607D49DF80000F0
:1017E000000705D425F0B7FA000601D5206838BDFA
:1017F000204900202060086078461F4908600020CA
:1018000038BD38B5082009F092F8194C00060DD4FF
:10181000694662200AF060F8000607D49DF80000CF
:10182000000705D425F097FA000601D5206838BDD9
:10183000104900202060086078460F4908600020A9
:1018400038BD38B5062009F072F8094C00060DD4F1
:10185000694662200AF040F8000607D49DF80000AF
:1018600000070FD425F077FA00060BD5206838BDA5
:101870000CC0072010C0072014C0072002C007209A
:10188000C8C10720A4490020206008607846A34909
:1018900008600020EBE738B5042009F048F8A04CB8
:1018A00000060DD4694662200AF016F8000607D437
:1018B0009DF80000000705D425F04DFA000601D57B
:1018C0002068D4E794490020206008607846934956
:1018D00008600020CBE738B5052009F028F8904CC7
:1018E00000060DD46946622009F0F6FF000607D411
:1018F0009DF80000000705D425F02DFA000601D55B
:101900002068B4E784490020206008607846834955
:1019100008600020ABE738B5032009F008F8804CD8
:1019200000060DD46946622009F0D6FF000607D4F0
:101930009DF80000000705D425F00DFA000601D53A
:10194000206894E774490020206008607846734955
:10195000086000208BE738B5022008F0E8FF704CE3
:1019600000060DD46946622009F0B6FF000607D4D0
:101970009DF80000000705D425F0EDF9000601D51B
:10198000206874E764490020206008607846634955
:10199000086000206BE738B5012008F0C8FF604CF4
:1019A00000060DD46946622009F096FF000607D4B0
:1019B0009DF80000000705D425F0CDF9000601D5FB
:1019C000206854E754490020206008607846534955
:1019D000086000204BE738B5132008F0A8FF504CF2
:1019E00000060DD46946622009F076FF000607D490
:1019F0009DF80000000705D425F0ADF9000601D5DB
:101A0000206834E744490020206008607846434954
:101A1000086000202BE738B5142008F088FF404C00
:101A200000060DD46946622009F056FF000607D46F
:101A30009DF80000000705D425F08DF9000601D5BA
:101A4000206814E734490020206008607846334954
:101A5000086000200BE738B5152008F068FF304C0F
:101A600000060DD46946622009F036FF000607D44F
:101A70009DF80000000705D425F06DF9000601D59A
:101A80002068F4E624490020206008607846234955
:101A900008600020EBE638B5572008F048FF204CDE
:101AA00000060DD46946622009F016FF000607D42F
:101AB0009DF80000000705D425F04DF9000601D57A
:101AC0002068D4E614490020206008607846134955
:101AD00008600020CBE638B5582008F028FF104CED
:101AE00000060DD46946622009F0F6FE000607D410
:101AF0009DF80000000705D425F02DF9000601D55A
:101B00002068B4E604490020206008607846034954
:101B100008600020ABE6000010C0072014C00720BA
:101B20000CC007207CB50546022024F0FFFC9E4C2B
:101B3000000625D49D4E3078800730D569465E205A
:101B400009F095FF00061BD401A9242009F08FFF9E
:101B5000000615D49DF80000632813D095B124F039
:101B60000CFF00060CD4362008F0E1FE000607D476
:101B700009F052FA000603D425F0EDF800060AD564
:101B800020687CBD352008F0D2FE0006F8D4002D78
:101B9000EED04B20E8E7308820F002003080844906
:101BA00000202060086078468249086000207CBDE3
:101BB00010B53B2008F0BBFE7B4C000607D47E48E6
:101BC000007830B13C2008F0B2FE000601D5206854
:101BD00010BDBDE810400120A4E710B50146142255
:101BE00076482AF02EFE382008F0A1FE000602D525
:101BF0006D48006810BDBDE8104025F0ACB810B5C8
